:020000040000FA
:100000008FEF48F0FFFFFFFF08D0FFFFFFFFFFFF6C
:10001000FFFFFFFFFFFFFFFF00D0E0CF02F1010174
:10002000D8CF01F1E8CF00F181509EB046EC39F015
:10003000F2B42DEC39F0A1B242EC39F09EBAECECFE
:1000400038F0F2B21BEC39F0F0B021EC39F000C11D
:10005000E8FF01C1D8FF02C1E0FF1000FFFFFFFF72
:10006000FFFFFFFFFFFFFFFFFFFFFFFFFFFFFFFFA0
:10007000FFFFFFFFFFFFFFFFFFFFFFFFFFFFFFFF90
:10008000FFFFFFFFFFFFFFFFFFFFFFFFFFFFFFFF80
:10009000FFFFFFFFFFFFFFFFFFFFFFFFFFFFFFFF70
:1000A000FFFFFFFFFFFFFFFFFFFFFFFFFFFFFFFF60
:1000B000FFFFFFFFFFFFFFFFFFFFFFFFFFFFFFFF50
:1000C000FFFFFFFFFFFFFFFFFFFFFFFFFFFFFFFF40
:1000D000FFFFFFFFFFFFFFFFFFFFFFFFFFFFFFFF30
:1000E000FFFFFFFFFFFFFFFFFFFFFFFFFFFFFFFF20
:1000F000FFFFFFFFFFFFFFFFFFFFFFFFFFFFFFFF10
:10010000001210180606080A0A0C0606080A060A53
:1001100006060808060E06060A0A08140C0A060A4D
:1001200008060606101010101010101010101010F5
:1001300010101010101010101010101010101010BF
:10014000101010101014161416120C140E1414148F
:100150000E180A0608080A060C0A08080808060607
:10016000040A0C120A0A0A060A0E140808061212D9
:10017000040E140806100E0C0606080606060606EF
:10018000080804040A16161614080A080806060ABF
:100190000808040A0E140A0C0A141010101010108B
:1001A000101010101010101010101010101010104F
:1001B00010101010101010101010140E120E08084D
:1001C00006141414141414141414141414141414FD
:1001D00014141414141414141414141414141414DF
:1001E0001414141414141414141414140A0A0A08F9
:1001F0000808080E0614100A100C06060606060863
:10020000020E0E080808060606060A0A0408040E6E
:100210001412140E0A0E0C100E0A0A0A0E0C10000C
:10022000FFFFFFFFFFFFFFFFFFFFFFFFFFFFFFFFDE
:10023000FFFFFFFFFFFFFFFFFFFFFFFFFFFFFFFFCE
:10024000FFFFFFFFFFFFFFFFFFFFFFFFFFFFFFFFBE
:10025000FFFFFFFFFFFFFFFFFFFFFFFFFFFFFFFFAE
:10026000FFFFFFFFFFFFFFFFFFFFFFFFFFFFFFFF9E
:10027000FFFFFFFFFFFFFFFFFFFFFFFFFFFFFFFF8E
:10028000FFFFFFFFFFFFFFFFFFFFFFFFFFFFFFFF7E
:10029000FFFFFFFFFFFFFFFFFFFFFFFFFFFFFFFF6E
:1002A000FFFFFFFFFFFFFFFFFFFFFFFFFFFFFFFF5E
:1002B000FFFFFFFFFFFFFFFFFFFFFFFFFFFFFFFF4E
:1002C000FFFFFFFFFFFFFFFFFFFFFFFFFFFFFFFF3E
:1002D000FFFFFFFFFFFFFFFFFFFFFFFFFFFFFFFF2E
:1002E000FFFFFFFFFFFFFFFFFFFFFFFFFFFFFFFF1E
:1002F000FFFFFFFFFFFFFFFFFFFFFFFFFFFFFFFF0E
:100300000000010F0019010F0002010F4102010F4F
:100310004102010F1423010F1441010F1423010F97
:10032000145F010F147D010F14B9010F7302010F47
:100330000018010F0000010F3202010F0A1E010F09
:100340000A37010F0A50010F0A69010F0A82010FD3
:100350001423010F2041010F205F010F209B010F8B
:100360000600010F3702010F0E02010F2802010FD4
:100370003202010F1423010F6400010F6419010FF1
:10038000644B010F6464010F0000010F2823010F6B
:100390002823010F2823010F2823010F2823010FF1
:1003A0002823010F2823010F2823010F2823010FE1
:1003B0002823010F2823010F2823010F2823010FD1
:1003C0002823010F2823010F2823010F2823010FC1
:1003D0002823010F2823010F2823010F2823010FB1
:1003E0002823010F2823010F2823010F2823010FA1
:1003F0002823010F2823010F2823010F2823010F91
:100400002823010F2823010F2823010F0023010FA8
:100410000041010F005F010F007D010F009B010FE4
:1004200000B9010F00D7010F0023010F0041010F98
:10043000005F010F007D010F009B010F00B9010F4C
:1004400000D7010F6696010F0000010F6CD8010F55
:100450006CD8010F6400010F0000010F0000010FB4
:100460000000010F0000010F0000010F0000010F4C
:100470000000010F0000010F0000010F0000010F3C
:100480000000010F2802010F1423010F147D010F3A
:10049000557D010F557D010F557D020F557D010FD3
:1004A0000000010F0A02010F0000010F0000010F00
:1004B0001423010F1441010F1402010F0000010F5A
:1004C000145F010F0A02010F0009010F557D020F91
:1004D0000012010F001B010F0024010F002D010F5E
:1004E0000036010F6432010F6419010F6432010FED
:1004F000644B010F6464010F6400010F6419010F64
:100500001441010F4141010F4141010F6432010FBC
:100510000A00010F0A19010F0A32010F0A4B010FDD
:100520006432010F557D010F6978010F693C010F9D
:100530004102010F149B010F2A48010F3C02010FD9
:100540003460010F3478010F644B010F0000010F7C
:100550000008010F0227010F0230010F557D010F26
:100560001441010F2823010F2823010F2823010F15
:100570002823010F2823010F2823010F2823010F0F
:100580002823010F2823010F2823010F2823010FFF
:100590002823010F2823010F2823010F2823010FEF
:1005A0002823010F2823010F2823010F2823010FDF
:1005B0002823010F2823010F2823010F2823010FCF
:1005C0002823010F2823010F2823010F2823010FBF
:1005D0002823010F2823010F2823010F2823010FAF
:1005E0002823010F0D02010F145F010F0201010FFB
:1005F0000230010F0000010F0000010F0000010F89
:100600000023010F0041010F005F010F007D010F6A
:10061000009B010F00B9010F00D7010F0023010F4C
:100620000041010F005F010F007D010F009B010FD2
:1006300000B9010F00D7010F0023010F0041010F86
:10064000005F010F007D010F009B010F00B9010F3A
:1006500000D7010F0023010F0041010F005F010FC0
:10066000007D010F009B010F00B9010F00D7010FA2
:100670000023010F0041010F005F010F007D010FFA
:10068000009B010F00B9010F00D7010F0023010FDC
:100690000041010F005F010F007D010F009B010F62
:1006A00000B9010F00D7010F0A02010F557D010F9C
:1006B000020C010F6419010F6400010F6400010FA7
:1006C0006419010F6400010F020C010F6464010F33
:1006D0001441010F021E010F147D010F1E02010FB4
:1006E0001423010F6419010F6432010F644B010FD1
:1006F0006464010F6400010F6432010F0000000FF9
:100700001423010F2802010F6923010F6923010F30
:100710006923010F0101010F41A8010F0730010BEF
:100720007887010F0227010F00D8010F0A08010F77
:100730000A10010F0000010F1802010F0023010F22
:100740000041010F007D010F009B010F145F010F9D
:100750001441010F145F010F147D010F149B010F51
:100760006432010F6400010F5A36010F145F010F4C
:10077000147D010F149B010FFFFFFFFFFFFFFFFF21
:10078000FFFFFFFFFFFFFFFFFFFFFFFFFFFFFFFF79
:10079000FFFFFFFFFFFFFFFFFFFFFFFFFFFFFFFF69
:1007A000FFFFFFFFFFFFFFFFFFFFFFFFFFFFFFFF59
:1007B0004275696C64696E67204D443220486173EC
:1007C000687D506C6561736520576169742E2E2EAB
:1007D0007D7D4865696E72696368735765696B6191
:1007E0006D70204F535443327D7D4D656E753F7D56
:1007F0004D656E753A7D4C6F67626F6F6B7D4761BB
:10080000732053657475707D5365742054696D65EC
:100810007D7D5265736574204D656E757D7D536574
:100820007475707D457869747D7D576169742E2E6D
:100830007D7D4D443220486173683A7D4465736123
:10084000747D496E746572666163657D537461720F
:10085000747D446174617D7D4865616465727D7DF0
:1008600050726F66696C657D446F6E652E7D436165
:100870006E63656C2052657365747D7D54696D652A
:100880003A7D446174653A7D53657420486F757292
:10089000737D52657365742E2E2E7D7D4C6F67625D
:1008A0006F6F6B7D437573746F6D2046756E6374E7
:1008B000696F6E7320497D7D5265736574204D6547
:1008C0006E757D7D5365742054696D653A7D4D6FFD
:1008D00072657D7D4465636F706C616E7D7D47617F
:1008E000736C6973747D4D6F72657D7D4578697435
:1008F0007D7D4E6F466C797D5374617274204469BE
:100900007665205B636D5D7D456E64204469766528
:100910002020205B636D5D7D456E642044656C61C5
:10092000792020205B735D7D506F776572204F6664
:10093000662020205B735D7D5072652D6D656E7540
:10094000202020205B735D7D76656C6F6369747910
:100950005B6D2F6D696E5D7D57616B652D757020C8
:10096000205B6D4261725D7D6D61782E537572669C
:100970002E5B6D4261725D7D474620646973706CC9
:10098000617920205B255D7D6D696E2E204F3220C0
:100990004469732E5B255D7D44697665206D656EC7
:1009A000757320205B735D7D53617475726174652E
:1009B000207820205B255D7D4465736174757261CC
:1009C000746520785B255D7D4E6F466C79205261A1
:1009D00074696F205B255D7D474620616C61726D97
:1009E000203120205B255D7D6E6F742075736564FA
:1009F000202020202020207D4465636F204F6666E4
:100A00007365745B646D5D7D70704F32206C6F77C1
:100A1000205B634261725D7D70704F322068696750
:100A2000685B634261725D7D73686F772070704FA1
:100A3000325B634261725D7D73616D706C696E677C
:100A4000207261746520207D44697669736F72201D
:100A500054656D702020207D44697669736F722023
:100A60004465636F6461747D44697669736F722055
:100A70004E6F74557365317D44697669736F72206A
:100A800070704F322020207D44697669736F722028
:100A9000446562756720207D44697669736F7220B2
:100AA0004E6F74557365327D73686F7720434E5374
:100AB000202020205B255D7D4C6F67626F6F6B206F
:100AC0006F6666736574207D4C6173742044656342
:100AD0006F2061745B6D5D7D456E642041706E6F4B
:100AE00065205B6D696E5D7D53686F77205662612E
:100AF0007474205B3D315D7D546869732070726F42
:100B00006772616D2069737D64697374726962755F
:100B100074656420696E207468657D7D686F70659A
:100B200020746861742069742077696C6C20626538
:100B30007D7D75736566756C2C20627574205749D0
:100B400054484F55547D414E592057415252414EC1
:100B500054593B20776974686F75747D6576656E4E
:100B60002074686520696D706C6965647D7D77614E
:100B70007272616E7479206F667D4D4552434841B3
:100B80004E544142494C495459206F727D7D46492B
:100B9000544E45535320464F5220417D50415254AC
:100BA0004943554C415220505552504F53452E7D8C
:100BB0005365652074686520474E552047656E650E
:100BC00072616C7D5075626C6963204C6963656EFF
:100BD000736520666F727D7D6D6F726520646574CC
:100BE00061696C733A7D7777772E6865696E726993
:100BF0006368737765696B616D702E64657D4465AC
:100C0000636F73746F707D7D6D2F6D696E7D4E6F38
:100C10002053746F707D4465636F73756D7D446997
:100C2000766574696D657D7D44657074687D46691F
:100C3000727374204761733F7D7D44656661756C96
:100C4000743A7D7D4D696E757465737D4D6F6E74FC
:100C50006820207D446179202020207D59656172C3
:100C60002020207D536574207D7D47617323207D86
:100C70005965737D43757272656E743A7D7D5365F7
:100C8000747570204D656E753A7D437573746F6D24
:100C90002046756E6374696F6E73497D4465636F3A
:100CA000747970653A7D5A482D4C3136204F437D1A
:100CB0004761756765202020207D47617567657DE8
:100CC0005A482D4C31362043437D41637469766523
:100CD000204761733F207D7D4761732053657475A4
:100CE00070202D204761736C6973747D4465707446
:100CF00068202B7D4465707468202D7D4261636B94
:100D00007D7D43435220536574506F696E74204D4E
:100D1000656E757D43435220536574506F696E74E0
:100D2000204D656E757D5350237D426174746572EC
:100D30007920496E666F7D7D426174746572792099
:100D4000496E666F726D6174696F6E7D4379636C15
:100D500065733A7D41706E6F657D4C61737420439D
:100D60006F6D706C6574653A7D7D4C6F77657374DB
:100D70002056626174743A7D4C6F7765737420619C
:100D8000743A7D7D546D696E3A7D546D61783A7D1B
:100D9000536574204761737D4F32202B7D7D4F3228
:100DA000202D7D7D4865202B7D7D4865202D7D7D16
:100DB000457869747D7D44656C6574657D7D4465A9
:100DC0006275673A7D7D4F4E207D4F46467D446576
:100DD0006C2E20616C6C7D7D556E657870656374DA
:100DE00065642072657365742066726F6D7D4469F9
:100DF00076656D6F64652120506C65617365206850
:100E0000656C707D616E64207265706F72742074A1
:100E10006865204465627567207D496E666F726DF6
:100E20006174696F6E2062656C6F77217D7D4261B0
:100E3000696C6F75747D41706E6F65202020207D18
:100E400044657363656E747D537572666163657D19
:100E5000517569743F7D4D6F72657D7D436F6E6620
:100E600069726D3A7D7D4D656E7520323A7D4361C4
:100E70006E63656C7D7D4F4B217D53746F70776120
:100E8000742E7D7D4E4F5420555345442121212100
:100E9000217D4E4F542055534544212121212121AC
:100EA00021212121217D4E6F742075736564217D80
:100EB0004E6F7420757365642121217D4C31362D70
:100EC0004746204F437D437573746F6D2046756EA2
:100ED0006374696F6E7349497D7D4746204C6F7717
:100EE0002020202020205B255D7D47462048696723
:100EF0006820202020205B255D7D436F6C6F72236E
:100F00002042617474657279207D436F6C6F722327
:100F1000205374616E646172647D436F6C6F7223E1
:100F200020446976656D61736B7D6E6F7420757397
:100F30006564202020202020207D53686F77207357
:100F40006563732E205B3D315D7D6E6F742075731C
:100F50006564202020202020207D6E6F7420757312
:100F60006564202020202020207D4176722E2044A0
:100F700065707468205B3D315D7D6E6F74207573A4
:100F80006564202020202020207D6E6F74207573E2
:100F90006564202020202020207D6E6F74207573D2
:100FA0006564202020202020207D6E6F74207573C2
:100FB0006564202020202020207D6E6F74207573B2
:100FC0006564202020202020207D6E6F74207573A2
:100FD0006564202020202020207D6E6F7420757392
:100FE0006564202020202020207D6E6F7420757382
:100FF0006564202020202020207D6E6F7420757372
:101000006564202020202020207D6E6F7420757361
:101010006564202020202020207D6E6F7420757351
:101020006564202020202020207D6E6F7420757341
:101030006564202020202020207D6E6F7420757331
:101040006564202020202020207D6E6F7420757321
:101050006564202020202020207D6E6F7420757311
:101060006564202020202020207D6E6F7420757301
:101070006564202020202020207D6E6F74207573F1
:101080006564202020202020207D6E6F74207573E1
:101090006564202020202020207D6E6F74207573D1
:1010A0006564202020202020207D6E6F74207573C1
:1010B0006564202020202020207D6E6F74207573B1
:1010C0006564202020202020207D6E6F74207573A1
:1010D0006564202020202020207D437573746F6D6F
:1010E0002046756E6374696F6E732049497D53683D
:1010F0006F77204C6963656E73657D7D4E6F7420DC
:10110000557365642121212121212121217D4E4F0B
:1011100054205553454421212121217D70704F32A7
:10112000202B7D7D70704F32202D7D7D44696C2E8B
:101130007D7D4465636F747970653A205A482D4C03
:101140003136204F437D466F72204F70656E2043CD
:101150006972637569742020207D446976657273B5
:101160002E20537570706F7274732035207D547209
:10117000696D69782047617365732E2020202020D7
:10118000207D436F6E66696775726520796F757231
:1011900020676173207D696E204761737365747584
:1011A00070206D656E752E20207D436865636B2011
:1011B000434631312026204346313220217D44658B
:1011C000636F747970653A204761756765202020E8
:1011D000207D4469766574696D652077696C6C2043
:1011E000626520696E7D4D696E757465733A5365ED
:1011F000636F6E64732E2020207D4F535443322042
:1012000077696C6C206E6F7420202020207D636FC6
:101210006D70757465204465636F2C204E6F466C4D
:10122000797D74696D6520616E64204465736174B5
:101230002E2D2020207D74696D6520617420616CE5
:101240006C21202020202020207D4465636F74794C
:1012500070653A5A482D4C3136204343207D466F05
:1012600072202853656D692D29436C6F7365642066
:10127000207D43697263756974207265627265616D
:1012800074686572737D436F6E66696775726520F9
:101290007468652033202020207D536574506F6969
:1012A0006E747320696E20434352202D207D536558
:1012B000747570206D656E752E2035206261696CC5
:1012C0002D7D6F7574732061726520617661696C24
:1012D00061626C652E7D4465636F747970653A2038
:1012E00041706E6F65202020207D4F535443322083
:1012F00077696C6C20646973706C6179207D6561BD
:1013000063682064657363656E74207365706172D1
:101310002D7D6174656C7920696E204D696E3A533C
:1013200065632E20207D57696C6C2074656D706F2D
:1013300072616C6C79207365747D73616D706C651E
:101340007261746520746F2031207365637D4E6F08
:10135000204465636F2063616C63756C6174696FB1
:101360006E7D4465636F747970653A204C31362D1B
:101370004746204F437D4465636F6D70726573739C
:10138000696F6E2063616C2D207D63756C6174697B
:101390006F6E73207769746820746865207D474696
:1013A0002D4D6574686F64202847465F6C6F2F472A
:1013B000467D5F6869292E20436865636B2043463C
:1013C00033322026207D4346333321204F70656E13
:1013D0002043697263756974207D7769746820445D
:1013E0006565702053746F70732E2020207D4465D6
:1013F000636F747970653A204C31362D474620432F
:10140000437D4465636F6D7072657373696F6E20A1
:1014100063616C2D207D63756C6174696F6E7320E0
:101420007769746820746865207D47462D4D657422
:10143000686F64202847465F6C6F2F47467D5F6862
:1014400069292E20436865636B204346333220268A
:10145000207D4346333321436C6F736564204369B9
:1014600072637569747D776974682044656570205E
:1014700053746F70732E2020207D4465636F6D6FF1
:101480006465206368616E6765642120207D4C314E
:10149000362D47462043437D4E6F7420666F756E30
:1014A000647D536574506F696E747D7D4E6F20440A
:1014B00065636F7D4772617068737D7D4469737089
:1014C0006C61797D4E6F206465636F7D53656172D9
:1014D0006368206D6F64756C657D457869747D7D8A
:1014E00052657365742043462C476173202620445F
:1014F00065636F7D44697361626C65206D6F6475AF
:101500006C657D7D53696D756C61746F727D4F5331
:1015100054432053696D756C61746F727D7D537493
:1015200061727420446976657D7D2B20316D7D7DEF
:101530002D20316D7D7D2B31306D7D7D2D31306DD8
:101540007D7D457869747D7D6E6F74207573657DD2
:10155000787D4461746520666F726D61743A7D7D3B
:101560005365747570204D656E7520323A7D4D4D12
:10157000444459597D7D44444D4D59597D7D5959B7
:101580004D4D44447D7D4F535443207D4261696CF1
:101590007D7D416972207D7D41697220207D43619E
:1015A0006C6962726174657D4D6178204465707408
:1015B000687D6E6F747D666F756E64217D7D6D567E
:1015C0003A7D4E6577204346206164646564217DE1
:1015D0004E657720437573746F6D46756E637469DD
:1015E0006F6E737D77657265206164646564212028
:1015F000436865636B7D4346204920616E642043E8
:1016000046204949204D656E757D666F72204465A0
:101610007461696C73217D7D53616C696E69747945
:101620003A7D426F74746F6D2054696D653A7D7DAB
:101630004D61782E2044657074683A7D43616C6317
:10164000756C617465204465636F7D7D53686F7749
:10165000204465636F706C616E7D4C6561642054DD
:1016600069737D7D4C656164205469737D7D53741D
:101670006F7077617463687D5265736574204C6F19
:1016800067626F6F6B7D5265626F6F74204F53544A
:10169000437D5265736574204465636F6461746152
:1016A0007D7D2C8B01D81200278D05D8279D120037
:1016B0002C8B01D812000B6F800EA66EF86A020EFA
:1016C000F76EFC0EF66E0BC14CF1000E2CBB010E3A
:1016D0004D6F040E4E6F4F6BEEEC0BF04851F6263B
:1016E0004951F7220900F55027BD02D0E8CF7DF01F
:1016F0000900F55027BD02D0E8CF7CF00900F55075
:101700000108E8CF7EF00900F5CF1BF10D6B0E6BE1
:10171000F66AF86A010EF76E01D02C9B0900F550AD
:101720000D27000E0E230B2FF9D72CBBF6D7F86A26
:10173000B00E0D25F66E070E0E21F76E27AD20EECA
:1017400060F009007D0EF56201D00AD0F550DE6E22
:1017500009007D0EF56201D003D0F550DE6EF1D7A1
:1017600027AD24EC0EF0120032C14CF133C14DF123
:101770003C0E4E6F4F6B4FD848C133F14CC132F124
:101780001200D89046334533472FFBD71200D8902C
:101790004B334A3349334833472FF9D71200495165
:1017A000FF08496F4851D890FF08486F12001F97F3
:1017B0005451525D506F55515359516FD8A8120072
:1017C0001F8750C154F151C155F1526953695451A9
:1017D000525D506F55515359516F12004A6B4B6B0C
:1017E0004C514E03F350486FF450496F4C514F0326
:1017F000F3504927F4504A234D514E03F3504927E3
:10180000F4504A23D8B04B2B4D514F03F3504A2785
:10181000F4504B231200486B496B4E514F11D8B412
:10182000FF0C010E476F4FBF05D0472BD8904E37A6
:101830004F37F9D7D890483749374E514C5F4F5101
:10184000D8A04F294D5FD8B005D04E514C274F51ED
:101850004D2301D048814707D8B41200D8904F33A8
:101860004E33E8D7200E476F4B514D6F4A514C6FA6
:101870004951536F4851526F4B6B4A6B496B486BE0
:10188000556B546BD890523753374C374D375437CC
:1018900055374F51555DD8A450EF0CF04E51545D63
:1018A000D8A05AEF0CF04E51545FD8A055074F51B5
:1018B000555FD880483749374A374B37472F42EF73
:1018C0000CF01200D89075337433762FFBD71200CA
:1018D000D8907A33793378337733762FF9D712006B
:1018E0007851FF08786F7751D890FF08776F120012
:1018F0002A978351815D7F6F84518259806FD8A868
:1019000012002A877FC183F180C184F181698269D5
:101910008351815D7F6F84518259806F1200796B92
:101920007A6B7B517D03F350776FF450786F7B5166
:101930007E03F3507827F45079237C517D03F350D4
:101940007827F4507923D8B07A2B7C517E03F3505A
:101950007927F4507A2312000A6FB8EF0CF00000D8
:101960000000000000000000000000000000000077
:101970000000000000000000000000000000000067
:101980000000000000000000000000000000000057
:101990000000000000000000000000000000000047
:1019A00000000000000000000A2FAFEF0CF0120052
:1019B000096FE4EF0CF000000000000000000000E0
:1019C0000000000000000000000000000000000017
:1019D0000000000000000000000000000000000007
:1019E00000000000000000000000000000000000F7
:1019F00000000000000000000000000000000000E7
:101A00000000630EACEC0CF0092FDBEF0CF01200C1
:101A1000630E3261326F32C134F1356B1F950A0E9D
:101A20003A6F366B67D8010E3A6F366B1F8562D8F6
:101A3000120032C134F1356B1F85F1D732C134F158
:101A4000356B1F95640E3A6F366B54D8E8D7259FD7
:101A5000376F1F8B372B372F1F9B238B372B372F3E
:101A6000239B32C134F133C135F11F95100E3A6F0B
:101A7000270E366F1FAD3ED8E80E3A6F030E366F55
:101A800023BB07D025BF03D01F85372D1F9523B952
:101A90001F851FAD2FD81F9D640E3A6F366B27B977
:101AA00024D023BB09D025BF03D01F85372D1F9518
:101AB00023B91F8523BB1F851DD80A0E3A6F366BCD
:101AC00023BB09D025BF03D01F85372D1F9523B910
:101AD0001F8523BB1F8529B708D00CD8010E3A6F8C
:101AE000366B1F8524A506D824952799386B382B8B
:101AF00023991200396B3651355DD8A00ED004E120
:101B00003A51345DD8A009D03651355F3A51345F2F
:101B1000D8A03507392B1F85EED7382F1200382B68
:101B2000300E39251FB504D01FBF04D0200E01D0C0
:101B3000258FDE6E372F12002E0EDE6E23891200E7
:101B4000A96E31D0A96E2BD02B91010EAA6E690E11
:101B500003D02691AA6A640EAD6E238F040EA96E7F
:101B60009D9A9E9A08EC4BF049D8AECFA8FFFAECAC
:101B70004AF026BF11D017D8FCEC4AF0A8CFADFF31
:101B800037D8A93EF1D70AEC4BF09E9A9D8AAA6AF3
:101B9000269F239FF9EF48F0FF0EAD6EF4D7A69E67
:101BA000A69CA6801200A69EA69CA684F29E550E18
:101BB000A76EAA0EA76EA682F28EA6B2FED7A69434
:101BC0001200948C948E240EAC6E900EAB6E080EA8
:101BD000B86EB06A220EAF6EAE6A9E6A9D8A12001F
:101BE000AC6AAB6A9D9A949C949E829C829E1200E1
:101BF000ABAE12000000ACA2FBD712009E9A269F4B
:101C0000436B446B9EBA120000000000000000000D
:101C10009EBA120000000000000000009EBA1200F0
:101C200000000000000000009EBA1200000000004A
:101C3000000000009EBA1200442FE4D7432FE1D7E2
:101C4000AB98AB88268F1200DE6A7BC0FAF17AC0AF
:101C5000F9F134EC5AF00101FAC17BF0F9C17AF0E4
:101C60001200106F10C17DF0210E2DD9D8901035C3
:101C7000000ED8B0010E2CD9D890103529D91200F9
:101C80000F6F0FC17CF0200E1ED9000E21D90F510D
:101C90001FD91200220E17D984807AC083FF809446
:101CA00080847BC083FF80948084210E0CD9D890DF
:101CB0001035000ED8B0010E0BD9D890103710296E
:101CC00007D9200E00D9000E03D90F5101D9220ED9
:101CD000FAD884807AC083FF809480847BC083FF9D
:101CE000809480841200220EEED884807AC083FF14
:101CF000809480847BC083FF809480841200836AF8
:101D000080968194809A8494809484921200F451F5
:101D100024EC10F0F5C11CF11C51B2DFF75131EC8D
:101D20000EF0E1DF1C2B1C51F663F6D71C51A8DF27
:101D3000F75131EC0EF0D7DFF5C11CF11C51A0DFDB
:101D4000F85131EC0EF0CFDF1C2B1C51F663F6D7A7
:101D50001C5196DFF85131EC0EF0C5DFF7C11CF1D4
:101D60001C517FDFF5518CDF95DF1C2B1C51F86374
:101D7000F7D7F7C11CF11C5174DFF65181DF8ADF00
:101D80001C2B1C51F863F7D731EC1AF01200F451F8
:101D900024EC10F0350E97D8F7C11CF1D8901C3503
:101DA000000ED8B0010E94D8D8901C3591D8360EBC
:101DB0008AD8F8C11CF1D8901C35000ED8B0010E9D
:101DC00087D8D8901C3584D8370E7DD8F5C11CF142
:101DD0001C517ED8F6C11CF11C517AD8200E73D844
:101DE000000E76D8F5C11CF11C5172D8210E6BD8AB
:101DF000F7C11CF1D8901C35000ED8B0010E68D880
:101E0000D8901C3565D8220E5ED8F5C11CF1F6C1FC
:101E10001DF11C511D5F1D2BF7C11CF1F8C11EF1F6
:101E20001C511E5F1E2B84801EC11CF17AC083FFD3
:101E3000809480847BC083FF809480847AC083FFF9
:101E4000809480847BC083FF809480841C2FEED795
:101E50001D2FEAD7000E37D831EC1AF01200350EDC
:101E600032D8000E35D8000E33D8360E2CD8010EDD
:101E70002FD83F0E2DD8370E26D8000E29D8EF0EBA
:101E800027D8200E20D8000E23D8000E21D8210EEE
:101E90001AD8000E1DD8000E1BD8220E14D884802C
:101EA000836A0A0E1E6F1E0E1D6F1C6B8094808449
:101EB000809480841C2FFAD71D2FF7D71E2FF3D7BD
:101EC000000E01D812008490836E809480841200EA
:101ED0008480836E8094808412008096200ED8ECDB
:101EE0000CF081840000809A00008482FA0ED8EC05
:101EF0000CF0848400008492020EACEC0CF084821E
:101F00000A0ED8EC0CF0240EDEDF020EDCDF000E31
:101F1000DFDF000EDDDF030ED6DF000ED9DF300E6F
:101F2000D7DF180ED0DF000ED3DF280ED1DFF80E7A
:101F3000CADF000ECDDF0F0ECBDFF90EC4DF000EBF
:101F4000C7DF0F0EC5DF100EBEDF000EC1DF000EB3
:101F5000BFDF0CD884DF8086200ED8EC0CF0050E95
:101F6000B2DF000EB5DF010EB3DF1200700EABDF83
:101F70001F0EAEDF000EACDF710EA5DF230EA8DF53
:101F8000800EA6DF720E9FDF2A0EA2DF800EA0DF7A
:101F9000730E99DF150E9CDF110E9ADF740E93DF1E
:101FA0001C0E96DF110E94DF750E8DDF1B0E90DF79
:101FB000150E8EDF760E87DF1A0E8ADF150E88DF8C
:101FC000770E81DF1C0E84DF180E82DF780E7BDF38
:101FD000210E7EDF150E7CDF1200700E74DF140EF2
:101FE00077DF000E75DF710E6EDF170E71DF000EEA
:101FF0006FDF720E68DF150E6BDF800E69DF730E08
:1020000062DF150E65DF110E63DF740E5CDF140EE8
:102010005FDF0B0E5DDF750E56DF1B0E59DF150EF1
:1020200057DF760E50DF130E53DF0E0E51DF770EA3
:102030004ADF1C0E4DDF180E4BDF780E44DF150E05
:1020400047DF0E0E45DF12002E6F2EC12FF1030E5B
:102050002F17000E2F4F500E2F4FA00E2F4FF80EA0
:10206000306F2EC12FF11C0E2F172F432F43000E60
:102070002F4F040E2F4F080E2F4F0C0E2F4F100E08
:102080002F4F140E2F4F200E2F4F3F0E316F313335
:10209000303331333033313330332EC12FF12E6BA7
:1020A00031332E3331332E3331332E33E00E2F17AD
:1020B0002F432F432F432F432F43000E2F4F040E48
:1020C0002F4F080E2F4F0C0E2F4F100E2F4F140EA8
:1020D0002F4F200E2F4F3F0E316F31332E333133C0
:1020E0002E3331332E3331332E3331332E332EC151
:1020F0007AF030C17BF01200E46F1F0EE46505D06A
:10210000010EAA6E200EE45F01D0AA6AE451040D0C
:10211000F350820FA96ECFEC0DF0A850AA6A1200FE
:10212000E46F1F0EE46505D0010EAA6E200EE45F79
:1021300001D0AA6AE451040DF350820FA96ECFECCE
:102140000DF0A8CF32F1A92ACFEC0DF0A8CF33F1D2
:10215000AA6A12009A0EE36F2A8D03D0240EE36F51
:102160002A9D1F8F2FEC0FF0010EBA6F2199219736
:102170002099AA6BA56B229D229FC6EC2AF0010E26
:10218000E8CF7FF02AAD04D0BA0E5BEC0BF003D0A1
:102190001B0E5BEC0BF0000EE8CF7FF0010E2AADBA
:1021A000000EAA6EB86B21912193140EE8CF7DF03A
:1021B000230EE8CF7CF020EE60F0AAC132F1000ED1
:1021C0002ABD200E322732C1DCF1386B382B376B39
:1021D00019EC0DF03A0EDE6E200EDE6E24EC0EF0E1
:1021E000E351AA255BEC0BF01F0EDC5DD8B411D0D7
:1021F000260EDC5DD8B40DD0270EDC5DD8B409D036
:10220000280EDC5DD8B405D0290EDC5DD8B401D031
:1022100003D0010EDC6F01D0DC6B140EE8CF7DF033
:10222000410EE8CF7CF020EE60F02B0EDE6E2F0E1C
:10223000DE6E2D0EDE6E3A0EDE6E200EDE6E2B0E84
:1022400022BD2D0EDE6E24EC0EF0140EE8CF7DF0D4
:102250005F0EE8CF7CF020EE60F0310EDE6E2F0EC8
:10226000DE6E310EDE6E300EDE6E3A0EDE6E200E4B
:10227000DE6E310EDE6E300E22BFDE6E200EDE6EA2
:1022800024EC0EF0140EE8CF7DF07D0EE8CF7CF04C
:1022900020EE60F0590E54EC0BF0A551800FA96EA2
:1022A000CFEC0DF0A8CF32F1A551810FA96ECFEC84
:1022B0000DF0A8CF33F1339F386B382B376B375184
:1022C00027EC0DF0280EDE6E310EA8AE380EDC675E
:1022D000310EDE6E350EA8BEDE6E420EDE6E290EAB
:1022E000DE6E200EDE6E200EDE6E200EDE6E24EC24
:1022F0000EF0140EE8CF7DF09B0EE8CF7CF020EEC0
:1023000060F0610E54EC0BF0A551820FA96ECFEC7A
:102310000DF0A8CF32F1A551830FA96ECFEC0DF0CF
:10232000A8CF33F1386B382B376B375127EC0DF0D2
:10233000200EDE6E200EDE6E200EDE6E24EC0EF021
:102340000B0E5BEC0BF0F6EC12F01BEC1DF0D0EC7E
:102350002FF021B30FD021B11AD020B3F9EF48F0FC
:1023600020B10CEC3CF020B10BEC42F0209120B9F4
:102370001CD0EDD7BA2B070EBA6302D0010EBA6F8C
:10238000B86B1BEC1DF0F6EC12F02193E0D7AA6AB3
:10239000010E2ABDAA6EBA4F0FD0BA4F17D0BA4F4E
:1023A00019D0BA4F1BD0BA4F39D0020E2AAD010E48
:1023B000BA6FAA6AA7EF13F0AA2BAABBAA6BAA51FD
:1023C000040DF3CFA5F1010EBA6FE8D6227D020EFF
:1023D000BA6FE4D6227F030EBA6FE0D6A551800F04
:1023E000A96ECFEC0DF0A8CF32F1A551810FA96EE7
:1023F000CFEC0DF0A8CF33F1339FA551820FA96E1A
:1024000032C1A8FFD3EC0DF0A551830FA96E33C1E3
:10241000A8FFD3EC0DF0040EBA6FC0D6A551820F01
:10242000A96ECFEC0DF0A8CF32F1A551830FA96EA4
:10243000CFEC0DF0A8CF33F1A551810FA96ECFECF1
:102440000DF0A8CFA6F1010EDC6305D0326732692A
:10245000322B336B16D022AD0BD0010E22BF0A0EE9
:10246000325F000EA6BF335B7F0E33BF336F09D0E0
:10247000010E22BF0A0E3227000EA6BF332333BF40
:10248000336BA551820FA96E32C1A8FFD3EC0DF0BA
:10249000A551830FA96E33C1A8FFD3EC0DF0050E33
:1024A000BA6F7CD6E46F1F0EE46505D0010EAA6EEC
:1024B000200EE45F01D0AA6AE451040DF350800FAE
:1024C000A96ECFEC0DF0A8CF32F1A92ACFEC0DF018
:1024D000A8CF33F1AA6A1200CF4F14D0CF4F19D032
:1024E0001200CF4F0FD0CF4F14D0CF4F19D0CF4FB6
:1024F0001ED0CF4F23D0CF4F28D0CF4F2FD0CF4F8C
:1025000034D012000B0E3DD8BCEC12F0020ECF6F8F
:1025100012000C0E49D8BCEC12F0030ECF6F120063
:10252000110E2FD8BCEC12F0040ECF6F1200120E59
:102530003BD8BCEC12F0050ECF6F1200130E34D84E
:10254000BCEC12F0060ECF6F1200060ECF6F1D0E00
:102550003ED8BCEC12F0070ECF6F1200200E24D82C
:10256000BCEC12F0080ECF6F1200210E1DD8BCEC8F
:1025700012F0010ECF6F1200326F32671200F6EFC9
:1025800028F0396F90EC10F032C152F133C153F1A1
:10259000395152EC12F032C154F133C155F1D7EC3C
:1025A0000BF01FA7FF0C000C396F90EC10F032C13C
:1025B00054F133C155F1395152EC12F032C152F19C
:1025C00033C153F1D7EC0BF01FA7FF0C000C396F90
:1025D00090EC10F032C154F133C155F1CFC152F13A
:1025E000536BD7EC0BF01FA7FF0C000C280E2BA38E
:1025F000C80EE56F050ED8EC0CF081B008D0E52FC1
:10260000F9D781B006D02B8324872499120081A2A8
:10261000F1D7249724992B9306EC4BF012002B97BB
:10262000010EBA6F1F9F2FEC0FF0B86B209921910C
:102630002193208F2187B5EC1DF01BEC1DF0249712
:1026400024993CEC13F021B124D020AFF9EF48F0ED
:1026500020B10CEC3CF020B10BEC42F020B13EEC90
:102660003BF020B1B8EC46F0209120B9F9EF48F0EA
:1026700020B3F9EF48F0E5D724A908D02183BA2B7D
:10268000060EBA6518D0010EBA6F15D024B7218195
:102690001200BA4F8AEF2CF0BA4F48EF34F0BA4F1D
:1026A0000EEF15F0BA4FA4EF13F0BA4F61EF13F02D
:1026B000BA4FF9EF48F0B86B21B71BEC1DF0249925
:1026C0001200010EBA6F1F9F2FEC0FF0B86B20990C
:1026D00021912193208F218709EC1EF01BEC1DF026
:1026E000249724993CEC13F0050EBA6304D0060E2F
:1026F000BA6F1BEC1DF021B115D020AF90D720B1DF
:102700000CEC3CF020B10BEC42F020B13EEC3BF085
:1027100020B1B8EC46F0209120B981D720B3F9EF71
:1027200048F0E0D7BA4FB1EF16F0BA4F08EF32F0E9
:10273000BA4F2AEF33F0BA4FEDEF49F0BA4FEDEF51
:1027400049F0050EBA6F6ED72B97010EBA6F1F9F17
:102750002FEC0FF0D3EC1DF0B86B20992191219351
:10276000208F2187F1EC13F09DEC14F01BEC1DF091
:10277000249724993CEC13F021B117D020AFF9EF46
:1027800048F020B10CEC3CF020B10BEC42F020B151
:102790003EEC3BF020B1B8EC46F0209120B9F9EFC7
:1027A00048F020B3F9EF48F0E5D7BA4FAEEF10F09C
:1027B000BA4FAAEF10F0BA4FACD0BA4F03D0BA4F0D
:1027C0005CD036D02B87220EA2EC0DF0A82A060E84
:1027D000A86201D0A86AD3EC0DF0040EBA6F249958
:1027E000BBD7220EA2EC0DF0A86604D0650E5BEC00
:1027F0000BF01200A82E04D0660E5BEC0BF012005A
:10280000A82E04D0680E5BEC0BF01200A82E04D0AA
:102810008A0E5BEC0BF01200A82E04D0980E5BEC35
:102820000BF01200A82E1200EC0E5BEC0BF0120065
:102830002BA7F9EF48F02FEC0FF0C6EC2AF0010EB1
:10284000E8CF7FF0EB0E5BEC0BF0000EE8CF7FF0F3
:10285000220EA2EC0DF0070EA802F350C10FBA6FC2
:10286000070E396FBA515BEC0BF0BA2B392FFAD740
:102870001E0E96EC49F0F9EF48F0010EBA6F1F9F5B
:102880002FEC0FF0F1EC1DF0B86B20992191219302
:10289000208F2187FFEC14F0D9EC14F01BEC1DF015
:1028A000249724993CEC13F0040EBA6304D0060E6E
:1028B000BA6F1BEC1DF021B117D020AFF9EF48F033
:1028C00020B10CEC3CF020B10BEC42F020B13EEC1E
:1028D0003BF020B1B8EC46F0209120B9A4EF13F002
:1028E00020B3F9EF48F0DED7BA4F54D0BA4F74D0C6
:1028F000BA4F07D0BA4F28D7BA4F26D7050EBA6FAE
:1029000026D776EC49F091EC49F0030EBA6F249982
:10291000B6D71A0EA2EC0DF0A82A630EA8640AD04E
:10292000690EA86007D01A0EA0EC0DF0030EBA6F66
:10293000249912D7640EA86EF6D71A0EA2EC0DF0E9
:10294000630EA86421D8690EA8601ED85F0EE8CF78
:102950007CF0530EE8CF7DF0000EE8CF7EF020EE45
:1029600060F0A8CF32F1336B1F8F030E27EC0DF010
:102970001F9F6B0EDE6E670EDE6E2F0EDE6E6C0E10
:10298000DE6E24EC0EF01200640EA86E1A0EA0EC9F
:102990000DF012005B0EA2EC0DF0A82A020EA86446
:1029A00001D0A86A5B0EA0EC0DF0010EBA6F24995D
:1029B0006BD75B0EA2EC0DF0A86604D0030E58ECAA
:1029C0000BF01200A82E04D0040E58EC0BF01200ED
:1029D000050E58EC0BF01200270EA2EC0DF0A82A01
:1029E000010EA86401D0A86A270EA0EC0DF02A857C
:1029F000010EA8622A95020EBA6F249945D7270EB8
:102A0000A2EC0DF0A86603D0830E5BEC0BF0A806D9
:102A1000A866F6D6820E5BEC0BF01200010EBA6FC0
:102A20002FEC0FF024EC1EF0B86B2099219121932C
:102A3000208F218724EC1EF01BEC1DF02497249995
:102A40003CEC13F021B116D020AFE9D520B10CEC4D
:102A50003CF020B10BEC42F020B13EEC3BF020B159
:102A6000B8EC46F0209120B90FEF13F020B3F9EF46
:102A700048F0E6D7BA4F08D0BA4F3AD0BA4F16D07E
:102A8000BA4F05D0BA4F20D0030EBA6FCBD548EC61
:102A900021F0BA6FBA6701D0F7D77FEC0EF0000EC5
:102AA0009B6E7E0ED36EFF0000EF00F048EC21F02D
:102AB000BA6FBA6701D0E8D72FEC0FF0190E5BECB4
:102AC0000BF08AEC16F0E0D748EC21F0BA6FBA6749
:102AD00001D0DAD72FEC0FF0190E5BEC0BF08DC1A3
:102AE00000F58EC101F520EC80F00101F9EF48F00E
:102AF00048EC21F0BA6FBA6701D0C6D72FEC0FF0BF
:102B0000190E5BEC0BF08DC100F58EC101F520ECC8
:102B100080F00101AA6A030EA96E336B150EE2D88C
:102B2000150EE0D8150EDED8150EDCD8150EDAD845
:102B3000150ED8D8010EA86E210EA0EC0DF0A86AD3
:102B4000220EA0EC0DF0A86A230EA0EC0DF0000EF2
:102B5000A86A270EA0EC0DF0A86A5A0EA0EC0DF0A2
:102B6000A86A5B0EA0EC0DF0640E1A0EA0EC0DF03E
:102B70001F0EA86E1B0EA0EC0DF0A86A1C0EA0EC98
:102B80000DF0A86A1D0EA0EC0DF0A86A1E0EA0ECB8
:102B90000DF0A86A1F0EA0EC0DF0A86A200EA0ECA4
:102BA0000DF0640EA86E240EA0EC0DF0250EA0EC26
:102BB0000DF0260EA0EC0DF0010ECC6FCD6B7F0E4C
:102BC000A96E336B640E8ED81E0E8CD8F00E8AD888
:102BD000780E88D8050E86D8070E84D8040E336F79
:102BE000338F880E7FD8040E336F338F4C0E7AD814
:102BF000140E78D8140E76D81E0E74D86E0E72D8B5
:102C00005A0E70D83C0E6ED8640E6CD8640E6AD81A
:102C10000A0E68D8130E66D8A00E64D8960E62D835
:102C20000A0E60D8060E5ED8060E5CD8000E5AD882
:102C3000000E58D80C0E56D8000E54D8140E52D888
:102C4000336B338F000E4ED8030E4CD80A0E4AD881
:102C5000000E48D8010EAA6E7F0EA96E336B1E0EB1
:102C600041D85A0E3FD8DF0E3DD8FF0E3BD8E00EBC
:102C700039D8000E37D8000E35D8000E33D8000EE4
:102C800031D8000E2FD8000E2DD8000E2BD8000EF4
:102C900029D8000E27D8000E25D8000E23D8000E04
:102CA00021D8000E1FD8000E1DD8000E1BD8000E14
:102CB00019D8000E17D8000E15D8000E13D8000E24
:102CC00011D8000E0FD8000E0DD8000E0BD8000E34
:102CD00009D8000E07D8000E05D8000E03D8AA6A3E
:102CE000F9EF48F0326FA92A32C1A8FFD3EC0DF0FA
:102CF000A92A33C1A8FFD3EC0DF0A92A32C1A8FF3D
:102D0000D3EC0DF0A92A339F33C1A8FFD3EC0DF00B
:102D1000336B1200BD6BBE6B020E366F376B400E0D
:102D20003A6F23933B693B5188EC2BF03A2FFAD74B
:102D3000C5843EEC2CF0070ED8EC0CF0372FEFD703
:102D4000362FECD72393BD6BBE6BFD0E7CEC2BF0C6
:102D5000FD0E7CEC2BF0FE0E7CEC2BF0BD6BBE6B05
:102D600012002FEC0FF0219521992197B86B21913A
:102D700021932099229122932295BB6BC6EC2AF0D5
:102D8000010EE8CF7FF01D0E5BEC0BF0000EE8CFDC
:102D90007FF0160E5BEC0BF0170E5BEC0BF0EBEC20
:102DA00016F0180E5BEC0BF02497249924B7B0ECC6
:102DB00017F024B97CEC17F021B942D020B10CEC0B
:102DC0003CF020B10BEC42F0209120B991D020B31F
:102DD000F9EF48F0EBD7460EE8CF7DF0410EE8CF93
:102DE0007CF020EE60F005C132F1386B382B376B88
:102DF00019EC0DF03A0EDE6E04C132F1386B382B4F
:102E0000376B19EC0DF0200EDE6E200EDE6E24EC1A
:102E10000EF0460EE8CF7DF05F0EE8CF7CF020EE9E
:102E200060F007C1F1F106C1F2F108C1F3F1C4ECA1
:102E300023F0200EDE6E200EDE6E24EC0EF012006B
:102E400007C132F1324F1F0E324F1C0E324F1F0E90
:102E5000324F1E0E324F1F0E324F1E0E324F1F0EBC
:102E6000324F1F0E324F1E0E324F1F0E324F1E0EAC
:102E7000324F1F0E066502D0010E066F200EE8CFFE
:102E80007DF09B0EE8CF7CF0080E396F95EC1CF0BE
:102E9000050E0A6F036B209120A1FED7209109EC4B
:102EA00017F0460EE8CF7DF0410EE8CF7CF020EE23
:102EB00060F005C132F1386B382B376B19EC0DF02F
:102EC0003A0EDE6E04C132F1386B382B376B19ECD9
:102ED0000DF03A0EDE6E03C132F1386B382B376BD2
:102EE00019EC0DF0200EDE6E24EC0EF00A2FD4D774
:102EF000010EBA6F63EF13F022B12189BB2BBBC166
:102F0000BCF1BC4F2185BC4F2285BC4F2283BC4FF6
:102F10002281200EE8CF7DF09B0EE8CF7CF020EEE2
:102F200060F05E0E54EC0BF0BBC1BCF1BC2F04D0C2
:102F30005A0E54EC0BF00FD0BC2F04D05B0E54ECA7
:102F40000BF009D0BC2F04D05C0E54EC0BF003D076
:102F50005D0E54EC0BF024EC0EF0F6EC12F01200C7
:102F60002499036B22B120D022B310D022B515D002
:102F700021B506D0052B170E05651CD0056B1AD0A0
:102F8000042B3B0E046516D0046B14D0062B1F0EC9
:102F9000066510D0010E066F0DD0072B0C0E0765CD
:102FA00009D0010E076F06D0082B140E086502D059
:102FB000080E086FEBEC16F0F6EC12F012007C6BCA
:102FC000080E7B6F6CC17DF16DC17EF18FEC0CF052
:102FD000100E7727270E782372C181F173C182F119
:102FE00077C183F178C184F178EC0CF07FC185F171
:102FF00080C186F12AB71ED0239585C17BF186C199
:103000007CF185C17DF186C17EF18FEC0CF0110E53
:10301000766F68EC0CF085C181F186C182F177C1D1
:1030200083F178C184F178EC0CF07FC187F180C125
:1030300088F117D0238585C17BF186C17CF185C1DC
:103040007DF186C17EF18FEC0CF00F0E766F68EC8F
:103050000CF0855177278651782377C187F178C1A5
:1030600088F16AC181F16BC182F1FA0E836F846BC2
:1030700078EC0CF07FC17BF180C17CF185C17DF1E2
:1030800086C17EF18FEC0CF077C174F178C175F1D7
:103090000C0E766F62EC0CF074C177F175C178F1AB
:1030A0002AA70DD06451772765517823100E772712
:1030B000270E782377C189F178C18AF10FD064C1D6
:1030C00081F165C182F177C183F178C184F178EC37
:1030D0000CF07FC177F180C178F1E8D766C168F163
:1030E00067C169F1C80E6827000E692368C17BF1CA
:1030F00069C17CF185C17DF186C17EF18FEC0CF058
:1031000077C174F178C175F10D0E766F62EC0CF039
:1031100074C18BF175C18CF162C174F163C175F139
:10312000010E766F62EC0CF074518B2775518C2375
:10313000B80E8B270B0E8C2370C181F171C182F107
:1031400089C183F18AC184F178EC0CF07FC17BF1F5
:1031500080C17CF18BC17DF18CC17EF18FEC0CF0D4
:103160000C0E766F68EC0CF02AB770EC0CF0E80EE1
:103170007727030E782377C18DF178C18EF125ADC5
:1031800004D0C6C18DF1C7C18EF16EC168F16FC1A7
:1031900069F1640E6827000E692368C17BF169C17B
:1031A0007CF187C17DF188C17EF18FEC0CF00B0EB4
:1031B000766F68EC0CF0249D23B509D0C80E7727F4
:1031C000000E782377C197F178C198F11200C80EEC
:1031D000816F826B77C183F178C184F178EC0CF058
:1031E0002AB7248D7FC197F180C198F11200C7D80A
:1031F000A00E3D6F0C0E586FFBD81200D6D857C1E9
:1032000071F156C170F11200BAD8900EF2D7CDD834
:1032100057C173F156C172F11200B1D80D0E586F3B
:10322000540E3D6FE5D8C1D857C15BF156C15AF174
:103230000D0E586F580E3D6FDBD8B7D857C15DF1F2
:1032400056C15CF10D0E586F640E3D6FD1D8ADD8EC
:1032500057C15FF156C15EF10D0E586F680E3D6F9C
:10326000C7D8A3D857C161F156C160F15BC163F102
:10327000D8906333D8906333D89063335AC162F1E6
:10328000D8805BA1D8906233D8805BA3D89062339A
:10329000D8805BA5D89062335CC164F1D8805DA111
:1032A000D8906433D8805DA3D8906433D8805DA56E
:1032B000D8906433D8805DA7D8906433D8805DA956
:1032C000D8906433D8805DABD89064335DC165F12C
:1032D000D8805AA1D8906533D8805AA3D890653346
:1032E000D8805AA5D8906533D8906533D890653387
:1032F000D89065335FC166F1D8805EAFD8906637ED
:10330000D8805EADD8906637676B5FBF67835FBD5F
:10331000678161C16AF1D88060AFD8906A376B6B02
:1033200061BF6B815EC16CF16C9D5CB16C8D6C9FFB
:103330005CB36C8F6D6B5CB56D815CB76D835CB994
:103340006D855CBB6D876F6B60C16EF16E9F239F57
:10335000120080820000808E00000000000000004B
:1033600000000000809E120080920000808E00000D
:1033700000000000000000000000809E1200E9DF55
:10338000F3DFE7DFF1DFE5DFEFDFE3DFEDDFE1DFF5
:10339000EBDFDFDFE9DFDDDFE7DFDBDFE5DFE4DF1A
:1033A000E3DFE2DFE1DFE0DF1200080E586F10D844
:1033B0003DC157F1080E586F0BD83DC156F1808EB4
:1033C000000000000000000000000000809E1200CD
:1033D000808E000000000000000000000000809EC1
:1033E00080A8D89080B8D8803D37582FF1D71200E8
:1033F000809E8082030E585F808E000000000000D7
:10340000000000000000809E00000000000000009E
:1034100000000000808E000000000000000000009E
:103420000000809E0000000000000000000000007E
:10343000808E000000000000000000000000809E60
:103440003DAF80923DBF8082D8903D37808E000096
:1034500000000000000000000000809E582FF0D700
:103460001200230E7CEC10F024EC10F01200240E5D
:103470007CEC10F024EC10F01200DB6FD9C1DAF113
:10348000D8C1D9F1D7C1D8F1D6C1D7F1D5C1D6F1BC
:10349000DBC1D5F12AA51200C80EE8CF7CF0640E7E
:1034A000E8CF7DF0000EE8CF7EF0000EE8CF7FF091
:1034B00031EC1AF020EE60F0D551DE6ED651DE6EA2
:1034C000D751DE6ED851DE6ED951DE6EDA51DE6E26
:1034D000200EDE6E24EC0EF01200FEEC4AF00EEC34
:1034E0004BF06DEC0FF02FEC0FF031EC1AF0850E75
:1034F0005BEC0BF0860E5BEC0BF0870E5BEC0BF0DD
:10350000880E5BEC0BF0640EE8CF7CF00A0EE8CF7F
:103510007DF0000EE8CF7EF0000EE8CF7FF031ECBA
:103520001AF020EE60F0D551DE6ED651DE6ED75126
:10353000DE6ED851DE6ED951DE6EDA51DE6E2E0EA1
:10354000DE6E200EDE6E1FC132F1386B382B376B0A
:103550001EEC0DF0200EDE6E20C132F1386B382BE0
:10356000376B1EEC0DF024EC0EF07D0EE8CF7CF0F6
:103570000A0EE8CF7DF0000EE8CF7EF0000EE8CF17
:103580007FF031EC1AF020EE60F021C132F1386B9F
:10359000382B376B1EEC0DF0200EDE6E22C132F19F
:1035A000386B382B376B1EEC0DF0200EDE6E23C10E
:1035B00032F1386B382B376B1EEC0DF0200EDE6EBF
:1035C00024C132F1386B382B376B1EEC0DF0200E16
:1035D000DE6E25C132F1386B382B376B1EEC0DF0E7
:1035E00024EC0EF0960EE8CF7CF00A0EE8CF7DF0CA
:1035F000000EE8CF7EF0000EE8CF7FF031EC1AF03D
:1036000020EE60F026C132F1386B382B376B1EECA0
:103610000DF0200EDE6E27C132F1386B382B376B80
:103620001EEC0DF0200EDE6E28C132F1386B382B07
:10363000376B1EEC0DF0200EDE6E29C132F1386BB7
:10364000382B376B1EEC0DF0200EDE6E2AC132F1E6
:10365000386B382B376B1EEC0DF024EC0EF024A7E2
:10366000FED7FCEC4AF0120037EC1AF00B0E58ECC7
:103670000BF0560E5BEC0BF0570E5BEC0BF031ECE5
:103680001AF01200000EE8CFF4F13C0EE8CFF5F18D
:10369000EF0EE8CFF6F15A0EE8CFF7F19F0EE8CF24
:1036A000F8F1C7EC0EF08EEC1EF0F8EC1EF01200F4
:1036B000E9DF37EC1AF0540E5BEC0BF031EC1AF04A
:1036C000080E396F910EE8CF7CF0000EE8CF7DF048
:1036D00095EC1CF012002BB512007A0E3DEC1AF09E
:1036E000B90EE8CF7CF0770EE8CF7DF0010EE8CF81
:1036F0007EF0000EE8CF7FF031EC1AF020EE60F0A3
:1037000022C532F1386B382B376B1EEC0DF0270ECB
:10371000DE6E24EC0EF0000EE8CF7EF01200B2DF79
:1037200037EC1AF0550E5BEC0BF031EC1AF012008E
:103730002BB5120020BF31D0790E3DEC1AF037ECDA
:103740001AF0520E5BEC0BF031EC1AF0760EE8CF6B
:103750007CF05E0EE8CF7DF0010EE8CF7EF0000E2B
:10376000E8CF7FF031EC1AF020EE60F02BC532F19B
:10377000386B382B376B08EC0DF06D0EDE6E24C500
:1037800032F1386B382B376B08EC0DF0270EDE6EFC
:1037900024EC0EF0000EE8CF7EF02BB51200780E70
:1037A0003DEC1AF0B90EE8CF7CF0770EE8CF7DF053
:1037B000010EE8CF7EF0000EE8CF7FF031EC1AF07A
:1037C00020EE60F031C532F1C70E3261326F1F9FBB
:1037D000386B382B376B1EEC0DF0270EDE6E24ECA9
:1037E0000EF032C532F1080E7CEC10F0326101D0DF
:1037F00067D7770E3DEC1AF0910EE8CF7CF0000E03
:10380000E8CF7DF0000EE8CF7EF031EC1AF020EE2C
:1038100060F0470EDE6E460EDE6E3A0EDE6E32C58C
:1038200032F1386B382B376B1EEC0DF0250EDE6E47
:10383000200EDE6E24EC0EF01200410EE8CF7CF07C
:10384000690EE8CF7DF0000EE8CF7EF031EC1AF083
:1038500020EE60F0EBC132F11F8F386B382B376BE5
:103860001EEC0DF01F9F6D0EDE6E690EDE6E6E0E8D
:10387000DE6E200EDE6E24EC0EF05F0EE8CF7CF0E4
:10388000640EE8CF7DF0000EE8CF7EF031EC1AF048
:1038900020EE60F0ECC132F11F8F386B382B376BA4
:1038A0001EEC0DF01F9F6D0EDE6E200EDE6E24EC02
:1038B0000EF012002BB51200760E3DEC1AF05A0EE7
:1038C000E8CF7CF0000EE8CF7DF0000EE8CF7EF070
:1038D00031EC1AF020EE60F02D0E1FB72B0EDE6ECD
:1038E00045C132F1386B382B376B08EC0DF0530EB5
:1038F00054EC0BF024EC0EF02B891200080E396FFB
:103900005A0EE8CF7CF0000EE8CF7DF02B990DD059
:10391000060E396F020EE8CF7CF0730EE8CF7DF013
:1039200004D0010EE8CF7EF003D0000EE8CF7EF089
:1039300020EE60F0200EDE6E392FFCD724EC0EF066
:10394000000EE8CF7EF01200630E3DEC1AF0320E4E
:10395000E8CF7CF0000EE8CF7DF0000EE8CF7EF0DF
:10396000000EE8CF7FF031EC1AF020EE60F019C1C4
:1039700032F1326705D01AC132F1326701D039D045
:103980002DAF34D0B72F01D034D02D8F060EB761B4
:1039900025D819C132F11AC133F1B4EC0BF033510F
:1039A00032C133F1326F490EDE6E6E0EDE6E740E72
:1039B000DE6E3A0EDE6E386B382B376B19EC0DF07D
:1039C0003A0EDE6E33C132F1386B382B376B19EC9F
:1039D0000DF0200EDE6E24EC0EF012002D9F050E71
:1039E000B76F12002D8F050EB76F1200B72F01D0E1
:1039F000CCD72D9F060EB761F5DF05C132F1386BCC
:103A0000382B376B19EC0DF03A0EDE6E04C132F133
:103A1000386B382B376B19EC0DF03A0EDE6E03C1A4
:103A200032F1386B382B376B19EC0DF0200EDE6E4F
:103A300024EC0EF01200230EE8CF7CF0000EE8CF4D
:103A40007DF0000EE8CF7EF0000EE8CF7FF031EC85
:103A50001AF020EE60F0B80EDE6E24EC0EF0410E8F
:103A6000E8CF7CF0000EE8CF7DF0000EE8CF7EF0CE
:103A7000000EE8CF7FF031EC1AF020EE60F0B80EC7
:103A8000DE6E24EC0EF05F0EE8CF7CF0000EE8CF87
:103A90007DF0000EE8CF7EF0000EE8CF7FF031EC35
:103AA0001AF020EE60F0B80EDE6E24EC0EF07D0E03
:103AB000E8CF7CF0000EE8CF7DF0000EE8CF7EF07E
:103AC000000EE8CF7FF031EC1AF020EE60F0B80E77
:103AD000DE6E24EC0EF09B0EE8CF7CF0000EE8CFFB
:103AE0007DF0000EE8CF7EF0000EE8CF7FF031ECE5
:103AF0001AF020EE60F0B80EDE6E24EC0EF0B90E77
:103B0000E8CF7CF0000EE8CF7DF0000EE8CF7EF02D
:103B1000000EE8CF7FF031EC1AF020EE60F0B80E26
:103B2000DE6E24EC0EF0BAC139F1394F230E394F55
:103B3000410E394F5F0E394F7D0E394F9B0E394F75
:103B4000B90EE8CF7CF0000EE8CF7DF0000EE8CF94
:103B50007EF0000EE8CF7FF031EC1AF020EE60F03E
:103B6000B70EDE6E24EC0EF01200C6EC2AF0010E49
:103B7000E8CF7FF0050E5BEC0BF0000EE8CF7FF096
:103B8000060E5BEC0BF0070E5BEC0BF0090E5BEC2A
:103B90000BF00A0E5BEC0BF08E0E5BEC0BF00B0ED9
:103BA0005BEC0BF01200C6EC2AF0010EE8CF7FF0C0
:103BB000620E5BEC0BF0000EE8CF7FF0630E5BEC67
:103BC0000BF0990E5BEC0BF0140E58EC0BF0640E3E
:103BD0005BEC0BF08E0E5BEC0BF00B0E5BEC0BF06A
:103BE0001200C6EC2AF0010EE8CF7FF0020E58EC6E
:103BF0000BF0000EE8CF7FF0010E58EC0BF0810EB9
:103C00005BEC0BF0BB0E5BEC0BF00B0E5BEC0BF00C
:103C10001200C6EC2AF0010EE8CF7FF0900E5BECAC
:103C20000BF0000EE8CF7FF0080E5BEC0BF06E0E91
:103C30005BEC0BF0710E5BEC0BF0F70E5BEC0BF03A
:103C40000B0E5BEC0BF01200C6EC2AF0010EE8CF75
:103C50007FF01C0E5BEC0BF0000EE8CF7FF0150E32
:103C60005BEC0BF0F50E5BEC0BF01C0E58EC0BF064
:103C70001D0E58EC0BF01E0E58EC0BF00B0E5BEC0F
:103C80000BF01200C6EC2AF0010EE8CF7FF0F80E20
:103C90005BEC0BF0000EE8CF7FF0F90E5BEC0BF065
:103CA000150E58EC0BF0160E58EC0BF0170E58ECE6
:103CB0000BF0180E58EC0BF00B0E5BEC0BF0120037
:103CC000650E3DEC1AF097C199F198C19AF1640E16
:103CD000E8CF7CF0000EE8CF7DF0000EE8CF7EF05C
:103CE000000EE8CF7FF031EC1AF020EE60F02D0EE0
:103CF00024BDDE6E97C132F198C133F1030E386FE7
:103D00001F8F020E27EC0DF01F9FB00EDE6E430ECC
:103D1000DE6E200EDE6E24EC0EF012002BB51200CB
:103D2000750E3DEC1AF097C199F198C19AF1D80E31
:103D3000E8CF7CF0410EE8CF7DF0000EE8CF7EF0BA
:103D4000000EE8CF7FF031EC1AF020EE60F02D0E7F
:103D500024BDDE6E97C132F198C133F1030E386F86
:103D60001F8F020E27EC0DF01F9FB00EDE6E200E8F
:103D7000DE6E24EC0EF01200740E3DEC1AF0780E9C
:103D8000E8CF7CF0000EE8CF7DF0000EE8CF7EF0AB
:103D900031EC1AF020EE60F0700EDE6E700EDE6E0A
:103DA0004F0EDE6E320EDE6E3A0EDE6E48C132F11E
:103DB00049C133F12987010E27EC0DF02997200E18
:103DC000DE6E24EC0EF012000A0E396F780EE8CF8A
:103DD0007CF0000EE8CF7DF095EC1CF01200C00ED8
:103DE000E8CF7CF0410EE8CF7DF0050E396F9DD510
:103DF0002ABB12002BB51200730E3DEC1AF0C00E58
:103E0000E8CF7CF0410EE8CF7DF0000EE8CF7EF0E9
:103E1000000EE8CF7FF031EC1AF0640E10C532F1DD
:103E2000D880325511C532F1D8803257090E7CEC5A
:103E300010F011C533F1326501D005D0336703D0DE
:103E4000050E396F72D5150E32630ED033670CD064
:103E500020EE60F0080E51EC0BF0200E2CBD2A0E67
:103E6000DE6E24EC0EF0120020EE60F01F8F386B37
:103E7000382B376B1EEC0DF02F0EDE6E11C532F1B4
:103E8000386B382B376B1EEC0DF0200E2CBD2A0E34
:103E9000DE6E1F9F24EC0EF01200550EE8CF7DF071
:103EA000000EE8CF7EF0000EE8CF7FF0AA6A220E67
:103EB000A2EC0DF0A86620D07D0EE8CF7CF031ECAE
:103EC0001AF020EE60F04F0EDE6E24EC0EF0550E70
:103ED000E8CF7DF0000EE8CF7EF0000EE8CF7FF057
:103EE000960EE8CF7CF031EC1AF020EE60F0430E35
:103EF000DE6E24EC0EF01200A806A86601D01200B7
:103F0000A806A86629D07D0EE8CF7CF031EC1AF027
:103F100020EE60F0430EDE6E550EE8CF7DF0000E11
:103F2000E8CF7EF0000EE8CF7FF024EC0EF0960E86
:103F3000E8CF7CF031EC1AF020EE60F0430EDE6E3C
:103F4000550EE8CF7DF0000EE8CF7EF0000EE8CFF2
:103F50007FF024EC0EF01200A806A86601D0120033
:103F6000A806A86629D07D0EE8CF7CF020EE60F090
:103F7000470EDE6E550EE8CF7DF0000EE8CF7EF0E6
:103F8000000EE8CF7FF031EC1AF024EC0EF0960E24
:103F9000E8CF7CF020EE60F0460EDE6E550EE8CFE6
:103FA0007DF0000EE8CF7EF0000EE8CF7FF031EC20
:103FB0001AF024EC0EF012007D0EE8CF7CF020EE1B
:103FC00060F0470EDE6E550EE8CF7DF0000EE8CFB4
:103FD0007EF0000EE8CF7FF031EC1AF024EC0EF00A
:103FE000960EE8CF7CF020EE60F0460EDE6E550EA9
:103FF000E8CF7DF0000EE8CF7EF0000EE8CF7FF036
:1040000031EC1AF024EC0EF01200000EE8CFF4F1BF
:10401000190EE8CFF5F1780EE8CFF6F1520EE8CFA1
:10402000F7F19F0EE8CFF8F1C7EC0EF029B164D09C
:104030006D0E3DEC1AF05A0EE8CF7DF0000EE8CF81
:104040007EF01F8F020E0A6F000E096F336B332B49
:10405000040E0A2720EE60F0470EDE6E33C132F107
:10406000386B382B376B1EEC0DF03A0EDE6E200EDF
:10407000DE6E0AC1A9FFCFEC0DF0A8CF32F1386B8C
:10408000382B376B1EEC0DF02F0EDE6EA92ACFEC0D
:104090000DF0A8CF32F1386B382B376B1EEC0DF0DA
:1040A0001B0EA2EC0DF033C132F1A832322FFDD736
:1040B000D8B004D0490E24EC10F005D0230E7CECCF
:1040C00010F024EC10F0210EA2EC0DF0A850336398
:1040D00001D009D0190E09275A0EE8CF7DF009C189
:1040E0007CF024EC0EF0230E7CEC10F024EC10F0AD
:1040F000050E3363ACD712005A0EE8CF7DF0000EE8
:10410000E8CF7EF01F8F230E0A6F000E096FE66B5B
:104110000A2BE62B190E09275A0EE8CF7DF009C1AC
:104120007CF020EE60F0530EDE6E500EDE6EE6C1C7
:1041300032F1386B382B376B1EEC0DF03A0EDE6E19
:10414000200EDE6E0AC1A9FFCFEC0DF0A8CF32F130
:10415000336B030E27EC0DF024EC0EF0030EE66338
:10416000D7D71F9F1200710E3DEC1AF02ABB120028
:1041700028BF120029A123D0870EE8CF7CF05A0E69
:10418000E8CF7DF0000EE8CF7EF0000EE8CF7FF0A4
:1041900031EC1AF020EE60F0240EA2EC0DF0A8CF66
:1041A00032F1336B030E27EC0DF0420EDE6E610E22
:1041B000DE6E720EDE6E1F9F24EC0EF057D0820E64
:1041C000E8CF7CF0640EE8CF7DF0010EE8CF7EF002
:1041D000000EE8CF7FF031EC1AF0210EA2EC0DF0CA
:1041E000A8CFD1F1D105040DF350070FA96ECFEC84
:1041F0000DF0A8CF11F5D105040DF350060FA96EEF
:10420000CFEC0DF0A8CFD0F111C50AF1D880640E23
:104210000A55D880A856A8CF10F5640E10C532F103
:10422000D880325511C532F1D880325711C533F1DB
:10423000150E326306D0336704D0090E58EC0BF02C
:1042400015D020EE60F01F8F386B382B376B1EECCB
:104250000DF02F0EDE6E11C532F1386B382B376B37
:104260001EEC0DF01F9F24EC0EF000D0000EE8CFE6
:10427000F4F17A0EE8CFF5F1AF0EE8CFF6F1520E79
:10428000E8CFF7F19F0EE8CFF8F187EC0EF01200BF
:10429000000EE8CFF4F1440EE8CFF5F1920EE8CF2E
:1042A000F6F1220EE8CFF7F1650EE8CFF8F1C7EC92
:1042B0000EF0230E7CEC10F0E8CFF4F1460EE8CFC0
:1042C000F5F1900EE8CFF6F1230EE8CFF7F1640E8A
:1042D000E8CFF8F187EC0EF08F0E5BEC0BF0910E4F
:1042E0005BEC0BF0920E5BEC0BF0010EBA6F000E64
:1042F000E8CFF4F1600EE8CFF5F18F0EE8CFF6F1DC
:10430000270EE8CFF7F1330EE8CFF8F1C7EC0EF047
:10431000BAC139F1600E394F600E394F780EE8CFCF
:104320007CF0270EE8CF7DF0000EE8CF7EF0000E87
:10433000E8CF7FF031EC1AF020EE60F0B70EDE6EC1
:1043400024EC0EF020992191219324992497B86BA5
:10435000640ED8EC0CF0D0EC2FF021B315D021B1C5
:104360000ED020B10CEC3CF020B10BEC42F02091CF
:1043700020B903D020B301D0EED7000C010CBA4F06
:10438000FCD7BA4FFBD7F9D7BA2B030EBA6302D0CA
:10439000010EBA6FACD7720E3DEC1AF090C133F13A
:1043A0008FC132F144EC2BF0270E33616FD02BBB61
:1043B0006CEC22F02B9B20EE60F0030E536FE80EA6
:1043C000526F33C155F132C154F1542B000E5523B5
:1043D000D7EC0BF01FA77DD8180EE8CF7CF0000EAD
:1043E000E8CF7DF0020EE8CF7EF0000EE8CF7FF040
:1043F00031EC1AF0000E536F630E526F33C155F15A
:1044000032C154F1D7EC0BF01FA70AD01F8F2987B8
:10441000386B382B376B375127EC0DF01F9F02D0CC
:10442000300EDE6E24EC0EF02997010EE8CF7EF000
:10443000320EE8CF7CF0280EE8CF7DF031EC1AF098
:1044400090C133F18FC132F144EC2BF020EE60F0DB
:104450002E0EDE6E000E536F090E526F33C155F1F2
:1044600032C154F1D7EC0BF01FA707D0040E386F00
:104470002485000E27EC0DF002D0300EDE6E24EC09
:104480000EF02495000EE8CF7EF012002BAB6CEC02
:1044900022F020EE60F0180EE8CF7CF0000EE8CF9E
:1044A0007DF0020EE8CF7EF0000EE8CF7FF031EC19
:1044B0001AF029871F8F386B382B376B375127EC51
:1044C0000DF01F9F24EC0EF02997000EE8CF7EF030
:1044D0001200200EDE6E1200000EE8CFF4F1180E6E
:1044E000E8CFF5F15A0EE8CFF6F1000EE8CFF7F17C
:1044F0005A0EE8CFF8F1C7EC0EF02B8B1200680EC5
:104500003DEC1AF0960EE8CF7CF0000EE8CF7DF07F
:10451000000EE8CF7EF0000EE8CF7FF031EC1AF00D
:1045200020EE60F00E0E54EC0BF0200EDE6E20C577
:1045300032F121C533F1B4EC0BF01F8F325133C18E
:1045400032F1336F386B382B376B1EEC0DF03A0EAF
:10455000DE6E33C132F1386B382B376B19EC0DF04E
:104560001F9F24EC0EF01200670E3DEC1AF07D0E3A
:10457000E8CF7CF0000EE8CF7DF0000EE8CF7EF0B3
:10458000000EE8CF7FF031EC1AF020EE60F0230E41
:1045900054EC0BF0200EDE6ECCC132F1CDC133F104
:1045A000B4EC0BF01F8F325133C132F1336F386BE3
:1045B000382B376B1EEC0DF03A0EDE6E33C132F144
:1045C000320732BF326B386B382B376B19EC0DF07A
:1045D0001F9F24EC0EF0120020BD1200620E3DEC75
:1045E0001AF0190EE8CF7CF0000EE8CF7DF0000E37
:1045F000E8CF7EF0000EE8CF7FF031EC1AF020EE2D
:1046000060F08DC132F18EC133F11F8F386B382BC2
:10461000376B375127EC0DF01F9F6D0EDE6E620E6B
:10462000DE6E610EDE6E720EDE6E200EDE6E24EC2D
:104630000EF01200660E3DEC1AF01F0E7CEC10F02E
:10464000326F010E326323D0AF0EE8CF7CF0000E44
:10465000E8CF7DF0000EE8CF7EF0000EE8CF7FF0CF
:1046600031EC1AF020EE60F0C2C132F1C3C133F177
:10467000010E386F24851F8F020E27EC0DF01F9F4F
:10468000560EDE6E200EDE6E24EC0EF01200230EAF
:104690007CEC10F0E8CFF4F1AE0EE8CFF5F1C20EED
:1046A000E8CFF6F1000EE8CFF7F11F0EE8CFF8F1F2
:1046B00087EC0EF0100E526F0E0E536FC2C154F104
:1046C000C3C155F1D7EC0BF01FB748D0B80E546FEB
:1046D0000B0E556FC2C152F1C3C153F1D7EC0BF0B1
:1046E0001FB739D050C14CF151C14DF1140E4E6F6E
:1046F0004F6B0BEC0CF048C10AF1020E0A650A6F11
:10470000230E7CEC10F0E8CFF4F1B50EE8CFF5F114
:10471000BB0EE8CFF6F11F0EE8CFF7F1210EE8CF80
:10472000F8F187EC0EF0220E7CEC10F0E8CFF4F1FB
:10473000AF0EE8CFF5F1C10EE8CFF6F1010EE8CFEC
:10474000F7F10AC1F8F1C7EC0EF0230E7CEC10F083
:1047500024EC10F01200010E0A6FD2D71E0E0A6F61
:10476000230E7CEC10F0E8CFF4F1B50EE8CFF5F1B4
:10477000BB0EE8CFF6F11F0EE8CFF7F1210EE8CF20
:10478000F8F1C7EC0EF0CFD75B0EA2EC0DF0A866E7
:104790000ED0F1C132F11F8F386B382B376B19EC0B
:1047A0000DF01F9F2F0EDE6EF2C132F112D05B0EA4
:1047B000A2EC0DF0A82E1FD0F2C132F11F8F386B82
:1047C000382B376B19EC0DF01F9F2F0EDE6EF1C1E9
:1047D00032F11F8F386B382B376B19EC0DF01F9FA0
:1047E0002F0EDE6EF3C132F11F8F386B382B376B13
:1047F00019EC0DF01200F3C132F11F8F386B382B1A
:10480000376B19EC0DF01F9F2F0EDE6EF1C132F1E8
:104810001F8F386B382B376B19EC0DF01F9F2F0E45
:10482000DE6EF2C132F11F8F386B382B376B19EC0B
:104830000DF012005B0EA2EC0DF0A86615D0F1C1D0
:1048400032F11F8F386B382B376B19EC0DF01F9F2F
:104850002F0EDE6EF2C132F11F8F386B382B376BA3
:1048600019EC0DF01F9F12005B0EA2EC0DF0A82EAC
:10487000E6D7F2C132F11F8F386B382B376B19EC4A
:104880000DF01F9F2F0EDE6EF1C132F11F8F386BBE
:10489000382B376B19EC0DF01F9F1200640E3DECA6
:1048A0001AF04B0EE8CF7CF0000EE8CF7DF0000E42
:1048B000E8CF7EF0000EE8CF7FF031EC1AF020EE6A
:1048C00060F007C1F1F106C1F2F108C1F3F1C4ECE7
:1048D00023F024EC0EF01200000EE8CFF4F1000EED
:1048E000E8CFF5F11A0EE8CFF6F1410EE8CFF7F177
:1048F000640EE8CFF8F1C7EC0EF012002BB51200F1
:10490000700E3DEC1AF0B80EE8CF7CF0000EE8CF48
:104910007DF0010EE8CF7EF0000EE8CF7FF031ECA5
:104920001AF020EE60F091C132F192C133F144EC03
:104930002BF01F8F2485030E27EC0DF01F9F1F9D6A
:1049400024EC0EF0000EE8CF7EF0120020BF120023
:10495000410E3DEC1AF028BF92D02ABB90D0260E13
:104960007CEC10F0326F010E326301D088D0A5C10B
:1049700032F1A6C133F11F9F20EE60F0386B382B67
:10498000376B1F8D375127EC0DF0140EE8CF7CF0FC
:10499000780EE8CF7DF0010EE8CF7EF031EC1AF012
:1049A00024EC0EF0000EE8CF7EF0120020BF1200C3
:1049B00037EC1AF08C0E5BEC0BF031EC1AF0550E64
:1049C000E8CF7CF05A0EE8CF7DF0010EE8CF7EF004
:1049D00031EC1AF0E1C132F11F9F20EE60F0386B2C
:1049E000382B376B1EEC0DF03A0EDE6EE2C132F161
:1049F000386B382B376B19EC0DF024EC0EF0000EF1
:104A0000E8CF7EF01200000EE8CFF4F13C0EE8CFC4
:104A1000F5F1770EE8CFF6F15A0EE8CFF7F19F0ED9
:104A2000E8CFF8F1C7EC0EF0120037EC1AF08B0E5D
:104A30005BEC0BF031EC1AF0910EE8CF7CF05A0EE3
:104A4000E8CF7DF0010EE8CF7EF031EC1AF0DCC14A
:104A500032F120EE60F0386B382B376B1EEC0DF026
:104A60003A0EDE6EDDC132F1386B382B376B19EC44
:104A70000DF024EC0EF0000EE8CF7EF01200A5C180
:104A800032F1A6C133F11F9F1F8D20EE60F0386B0D
:104A9000382B376B1F8D375127EC0DF03A0EDE6E39
:104AA000A7C132F1386B382B376B19EC0DF0140EAF
:104AB000E8CF7CF05A0EE8CF7DF0010EE8CF7EF013
:104AC00031EC1AF024EC0EF01F9D000EE8CF7EF0C2
:104AD0001200000EE8CFF4F1360EE8CFF5F1660EC5
:104AE000E8CFF6F13E0EE8CFF7F19F0EE8CFF8F1F0
:104AF000C7EC0EF0120020BF1200560E3DEC1AF06B
:104B000037EC1AF01B0E58EC0BF031EC1AF0500E8B
:104B1000E8CF7CF06E0EE8CF7DF0000EE8CF7EF09F
:104B200031EC1AF020EE60F017C132F118C133F108
:104B3000020E325F000E335BB4EC0BF032C10AF1AF
:104B400033C132F1336B000E1F9F1F8D386B382B32
:104B5000376B1F8D375127EC0DF03A0EDE6E0AC110
:104B600032F1386B382B376B19EC0DF01F9F24ECAA
:104B70000EF0550E3DEC1AF0500EE8CF7CF03E0ED4
:104B8000E8CF7DF0000EE8CF7EF031EC1AF020EE99
:104B900060F093C132F194C133F144EC2BF01F8FDC
:104BA0002485030E27EC0DF01F9F6D0EDE6E200E88
:104BB000DE6E24EC0EF01200610E3DEC1AF0000ED9
:104BC000E8CF7CF0000EE8CF7DF0000EE8CF7EF05D
:104BD000000EE8CF7FF031EC1AF020EE60F0060E08
:104BE00051EC0BF0AA6AA96ACFEC0DF0A8CF32F114
:104BF000A92ACFEC0DF0A8CF33F11F8F386B382BDB
:104C0000376B375127EC0DF0200EDE6E560EDE6E40
:104C1000010E326F1F8F386B382B376B1EEC0DF087
:104C20002E0EDE6E360E326F1F8F386B382B376BC1
:104C300019EC0DF01F9F24EC0EF012006F0E3DECEE
:104C40001AF06CEC24F01F0E5BEC0BF029B107D0CE
:104C5000200E5BEC0BF07A0E5BEC0BF006D0EE0E48
:104C60005BEC0BF0890E5BEC0BF0210E5BEC0BF0B8
:104C7000220E5BEC0BF012006F0E3DEC1AF0F00E02
:104C80005BEC0BF0F10E5BEC0BF0190E58EC0BF03B
:104C9000930E5BEC0BF0F40E5BEC0BF01200640E69
:104CA000E8CF7DF0000EE8CF7CF0000EE8CF7EF07C
:104CB00031EC1AF020EE60F0530EDE6E650EDE6E03
:104CC0006C0EDE6E180EA2EC0DF0A8CF32F11F9F15
:104CD000386B382B376B08EC0DF02F0EDE6E190E8B
:104CE000A2EC0DF0A8CF32F1386B382B376B08EC03
:104CF0000DF024EC0EF07B0E5BEC0BF07C0E5BEC0D
:104D00000BF07D0E5BEC0BF07E0E5BEC0BF01200FB
:104D1000FE0E5BEC0BF0FA0E5BEC0BF0FB0E5BECAB
:104D20000BF0FC0E5BEC0BF0FD0E5BEC0BF01200DD
:104D3000230E7CEC10F0E8CFF4F17CC0F5F17CC0E0
:104D4000F6F1140EF6277A0EE8CFF7F13227320784
:104D50008A0E3261326F32C1F8F1C7EC0EF0000EEC
:104D6000E8CFF4F17CC0F5F17CC0F6F1140EF62723
:104D700032C1F7F1F72B8B0EE8CFF8F1C7EC0EF04C
:104D80001200000EE8CFF4F133C1F5F17D0EE8CF4B
:104D9000F6F1640EE8CFF7F19F0EE8CFF8F1C7EC1B
:104DA0000EF012006E0E3DEC1AF02BC532F1326798
:104DB00006D052EC28F0EF0E5BEC0BF012001F8FC8
:104DC000640EE8CF7DF0000EE8CF7CF0336F40EC4E
:104DD0000EF020EE60F02BC532F13251D8B4C1EFA5
:104DE00026F0386B382B376B1EEC0DF06D0EDE6E37
:104DF00024EC0EF08C0EE8CF7DF0000EE8CF7CF0B6
:104E000020EE60F024C532F1386B382B376B19EC8B
:104E10000DF0270EDE6E24EC0EF098EC26F0640EFA
:104E2000E8CF7DF0190EE8CF7CF0336F40EC0EF048
:104E300020EE60F02CC532F13251D8B4C1EF26F02B
:104E4000386B382B376B1EEC0DF06D0EDE6E24ECDC
:104E50000EF08C0EE8CF7DF0190EE8CF7CF020EE3E
:104E600060F025C532F1386B382B376B19EC0DF03B
:104E7000270EDE6E24EC0EF098EC26F0640EE8CFE0
:104E80007DF0320EE8CF7CF0336F40EC0EF020EE78
:104E900060F02DC532F13251D8B4C1EF26F0386B35
:104EA000382B376B1EEC0DF06D0EDE6E24EC0EF021
:104EB0008C0EE8CF7DF0320EE8CF7CF020EE60F073
:104EC00026C532F1386B382B376B19EC0DF0270EF5
:104ED000DE6E24EC0EF098EC26F0640EE8CF7DF048
:104EE0004B0EE8CF7CF0336F40EC0EF020EE60F01C
:104EF0002EC532F13251D8B4C1EF26F0386B382BC1
:104F0000376B1EEC0DF06D0EDE6E24EC0EF08C0E89
:104F1000E8CF7DF04B0EE8CF7CF020EE60F027C5A7
:104F200032F1386B382B376B19EC0DF0270EDE6E33
:104F300024EC0EF098EC26F0640EE8CF7DF0640EC1
:104F4000E8CF7CF0336F40EC0EF020EE60F02FC520
:104F500032F13251D8B4C1EF26F0386B382B376BB1
:104F60001EEC0DF06D0EDE6E24EC0EF08C0EE8CF14
:104F70007DF0640EE8CF7CF020EE60F028C532F1C1
:104F8000386B382B376B19EC0DF0270EDE6E24ECE6
:104F90000EF098EC26F012006D0E3DEC1AF0640E47
:104FA000E8CF7DF0000EE8CF7EF01F8F020E0A6F73
:104FB000E70E096F336B332B040E0A27190E0927EE
:104FC000640EE8CF7DF009C17CF020EE60F0470E62
:104FD000DE6E33C132F1386B382B376B1EEC0DF0BF
:104FE0003A0EDE6E0AC1A9FFCFEC0DF0A8CF32F168
:104FF000386B382B376B1EEC0DF02F0EDE6EA92AA6
:10500000CFEC0DF0A8CF32F1386B382B376B1EEC9C
:105010000DF01B0EA2EC0DF033C132F1A832322F8D
:10502000FDD70F0ED8A00A0E1B6F24EC0EF00F0E4A
:105030001B6F050E3363BFD71200640EE8CF7DF0FF
:10504000000EE8CF7EF01F8F230E0A6FE70E096F68
:10505000E66B0A2BE62B190E092709C17CF0640EBA
:10506000E8CF7DF020EE60F0530EDE6E500EDE6E67
:10507000E6C132F1386B382B376B1EEC0DF03A0E6F
:10508000DE6E0AC1A9FFCFEC0DF0A8CF32F1336B71
:10509000030E27EC0DF024EC0EF0030EE663D9D7D7
:1050A0001F9F1200000EE8CFF4F1000EE8CFF5F1DB
:1050B0007D0EE8CFF6F1520EE8CFF7F19F0EE8CF64
:1050C000F8F1C7EC0EF012006C0E3DEC1AF0000E79
:1050D000E8CF7CF0550EE8CF7DF0000EE8CF7EF0F3
:1050E000000EE8CF7FF031EC1AF020EE60F0B80E41
:1050F000DE6E24EC0EF0190EE8CF7CF0550EE8CFF2
:105100007DF0000EE8CF7EF0000EE8CF7FF031ECAE
:105110001AF020EE60F0B80EDE6E24EC0EF0320EC7
:10512000E8CF7CF0550EE8CF7DF0000EE8CF7EF0A2
:10513000000EE8CF7FF031EC1AF020EE60F0B80EF0
:10514000DE6E24EC0EF04B0EE8CF7CF0550EE8CF6F
:105150007DF0000EE8CF7EF0000EE8CF7FF031EC5E
:105160001AF020EE60F0B80EDE6E24EC0EF0640E45
:10517000E8CF7CF0550EE8CF7DF0000EE8CF7EF052
:10518000000EE8CF7FF031EC1AF020EE60F0B80EA0
:10519000DE6E24EC0EF0BAC139F1000E394F000E6C
:1051A000394F190E394F320E394F4B0E394F640EAD
:1051B000E8CF7CF0550EE8CF7DF0000EE8CF7EF012
:1051C000000EE8CF7FF031EC1AF020EE60F0B70E61
:1051D000DE6E24EC0EF012007F0E5BEC0BF0800E06
:1051E0005BEC0BF0840E5BEC0BF01200000EE8CFD2
:1051F000F4F1380EE8CFF5F1580EE8CFF6F1450E90
:10520000E8CFF7F1730EE8CFF8F1C7EC0EF0230EFC
:105210007CEC10F0E8CFF4F13A0EE8CFF5F1560E41
:10522000E8CFF6F1460EE8CFF7F1720EE8CFF8F1CD
:1052300087EC0EF03C0EE8CF7CF0470EE8CF7DF017
:10524000000EE8CF7EF0010EE8CF7FF037EC1AF0C9
:1052500020EE60F0430EDE6E460EDE6E39C132F196
:10526000386B382B376B1EEC0DF0210EDE6E24EC04
:105270000EF0000EE8CF7FF031EC1AF01200680E4D
:105280003DEC1AF0690E3DEC1AF0000EE8CFF4F197
:10529000190EE8CFF5F1780EE8CFF6F1520EE8CF0F
:1052A000F7F19F0EE8CFF8F1C7EC0EF0230E7CEC7F
:1052B00010F0E8CFF4F1190EE8CFF5F1780EE8CF51
:1052C000F6F1520EE8CFF7F19F0EE8CFF8F187EC38
:1052D0000EF025EE33F0100E0A6F096B230E7CECF6
:1052E00010F0E8CFF4F11C0E0925E8CFF5F11C0E03
:1052F0000925E8CFF6F1092B092B640EE8CFF7F169
:10530000DECFF8F1D890F833D890F833640EF82750
:105310009D0EF861F86FC7EC0EF00A2FDFD725EE6F
:1053200043F0100E0A6F096B230E7CEC10F0E8CFEF
:10533000F4F1560E0925E8CFF5F1560E0925E8CF10
:10534000F6F1092B092B640EE8CFF7F1DECFF8F167
:10535000D890F833D890F833640EF8279D0EF86192
:10536000F86FC7EC0EF00A2FDFD7540EE8CF7DF0B0
:10537000200EE8CF7CF031EC1AF020EE60F04E0EFB
:10538000DE6E320EDE6E24EC0EF0540EE8CF7DF0B1
:105390005A0EE8CF7CF031EC1AF020EE60F0480EA7
:1053A000DE6E650EDE6E24EC0EF01200C6EC2AF006
:1053B000010EE8CF7FF0030E5BEC0BF0000EE8CFA0
:1053C0007FF0440E5BEC0BF0450E5BEC0BF0460EF1
:1053D0005BEC0BF0470E5BEC0BF0480E5BEC0BF05C
:1053E000490E5BEC0BF04A0E5BEC0BF01200C6ECC6
:1053F0002AF0010EE8CF7FF0030E5BEC0BF0000EFD
:10540000E8CF7FF04B0E5BEC0BF04C0E5BEC0BF03F
:105410004D0E5BEC0BF04E0E5BEC0BF04F0E5BECAD
:105420000BF0500E5BEC0BF0510E5BEC0BF012002E
:10543000C6EC2AF0010EE8CF7FF00F0E58EC0BF00F
:10544000000EE8CF7FF0100E58EC0BF0110E58EC68
:105450000BF0120E58EC0BF0130E58EC0BF0120080
:105460002BB512006A0E3DEC1AF0A80EE8CF7CF0C6
:10547000410EE8CF7DF0000EE8CF7EF0000EE8CFC1
:105480007FF031EC1AF020EE60F018C532F132678F
:1054900006D0070E51EC0BF024EC0EF012008DC17B
:1054A0004CF18EC14DF10A0E4E6F4F6B0BEC0CF0B0
:1054B0004967486959C1E8FF486103D048C118F5F8
:1054C00002D059C118F518C532F1336B1F8F030E86
:1054D00027EC0DF01F9F24EC0EF0120030EC80F052
:1054E00001011A0E58EC0BF020EE60F0230EDE6E78
:1054F00063C532F163C50AF11F8F386B382B376BE8
:105500001EEC0DF0200EDE6E280EDE6E100E0A610F
:1055100005D04E0EDE6E320EDE6E04D0480EDE6E0C
:10552000650EDE6E290EDE6E200EDE6E640EE8CF96
:105530007DF0190EE8CF7CF0000EE8CF7EF031EC64
:105540001AF024EC0EF020EE60F015EE33F00A2B8A
:10555000E6CF32F10A2FFCD7386B382B376B1EECB5
:105560000DF0250EDE6E200EDE6E640EE8CF7DF0AF
:10557000320EE8CF7CF0000EE8CF7EF031EC1AF06E
:1055800024EC0EF01F9F1200000E03D0230E7CECC3
:1055900010F0E8CFF4F1000EE8CFF5F11A0EE8CFE5
:1055A000F6F1000EE8CFF7F19F0EE8CFF8F1C7EC67
:1055B0000EF012002BB5120028BF12002ABB1200F9
:1055C0002BB912006B0E3DEC1AF05A0EE8CF7CF0AE
:1055D000000EE8CF7DF0000EE8CF7EF031EC1AF03F
:1055E00020EE60F0430EDE6E4E0EDE6E530EDE6E6B
:1055F0003A0EDE6E65C532F11F8F386B382B376B74
:105600001EEC0DF01F9F250EDE6E24EC0EF0120036
:10561000400EA2EC0DF0010EA86229D0C80EE8CF12
:105620007CF0000EE8CF7DF0000EE8CF7EF0000E9B
:10563000E8CF7FF037EC1AF020EE60F0400E326FCA
:10564000180E336F322B32EC2BF07D0EA86201D096
:1056500004D0A8CFDEFF332FF5D724EC0EF031ECC9
:105660001AF0120032C1A9FFCFEC0DF01200180E93
:10567000396FC80EE8CF7CF0000EE8CF7DF095ECD6
:105680001CF012001200120025BD12001A0EA2EC2E
:105690000DF0A8CF0AF1690E0A611200630E0A65C7
:1056A000120032C14CF133C14DF1640E4E6F4F6B9D
:1056B000EEEC0BF00AC14EF14F6B32EC0CF048C12E
:1056C00032F149C133F112003B6F010EBD27000ECC
:1056D000BE23BEAF02D0BD6BBE6B3B2FF6D7120010
:1056E0003B6F010EBD5F000EBE5BBEAF02D07F0EF2
:1056F000BE6F3B2FF6D712009CD8010EBD27000EBF
:10570000BE232391BEAF1200BD6BBE6B238112007E
:1057100023B31CD823A30BD82383000EBD2BBE2399
:105720002391BEAF1200BD6BBE6B238112003B6F95
:10573000C580A4D8A60EC96EA1D894D8BEC1C9FF91
:105740009DD890D8BDC1C9FF99D88CD83BC1C9FF9D
:1057500095D888D812003B6B3C6B229F229DC58454
:105760008DD8C5808BD8A60EC96E88D8C5BCF7D792
:105770003CC1C9FF83D876D83BC1C9FF7FD872D856
:10578000C5827CD8A70EC96E79D86CD8C58676D864
:1057900022BD05D0228DFD0EC962229D11D022BFEF
:1057A00005D0228FFD0EC96209D00AD0FE0EC96253
:1057B00005D03BC1BDF13CC1BEF10DD0229F229D61
:1057C000010E3B27000E3C233CBF03D0C58856D8B2
:1057D000DDD7BD6BBE6BC58451D8229F229D1200C0
:1057E000C5844CD8C5804AD8A60EC96E47D8C5BC5A
:1057F000F7D7BEC1C9FF42D835D8BDC1C9FF3ED811
:1058000031D8C5823BD8A70EC96E38D82BD8C586EB
:1058100035D8C950C58432D81200E2DF010EBD2749
:10582000000EBE232391BEAF1200BD6BBE6B238161
:1058300012003B6FC58022D8A60EC96E1FD812D8A1
:10584000BEC1C9FF1BD80ED8BDC1C9FF17D80AD821
:105850003BC1C9FF13D806D8C58410D8060ED8ECB2
:105860000CF01200C5BC01D812004D0E3DEC1AF030
:10587000FAEC4AF00BD89E96C46B1200C42F01D0EC
:10588000F4D79EA6FBD7C46B9E961200C66A4E0E36
:105890003DEC1AF0C56AC76A949694888296090E00
:1058A000C46F8286000082B804D082968296C42F8C
:1058B000F8D79486C66A0A0ED8EC0CF0000EC76EB4
:1058C000280EC66E000EC56E080EC86EFCEC4AF0BF
:1058D0004F0E3DEC1AF01200C56FC580CFDF900E61
:1058E000C96ECCDFBFDFC5C1C9FFC8DFBBDFC58460
:1058F000C5DF12009E96C580C1DF910EC96EBEDF66
:10590000B1DFC586BBDFC9CFC5F1C588B7DFC584A8
:10591000B5DF1200259529952FEC0FF025932597DB
:105920002599BC6BBB6BC16B010EE8CF7FF00C0EF1
:105930005BEC0BF0000EE8CF7FF0A56BA66B46EC9E
:105940002CF0ABEC2BF0396B3A6B050EBA6F010EF5
:10595000E8CF7FF00C0E5BEC0BF0000EE8CF7FF091
:10596000229D229F010EA527000EA623A6BF27D0A9
:10597000010E70EC2BF0F0EC2BF022BD05D0228D47
:10598000FA0EC962229D10D022BF05D0228FFA0ED6
:10599000C96207D809D0BDC1BFF1BEC1C0F1C12BDA
:1059A00013D0229F229D1200010E3927000E3A23A8
:1059B0003ABF01D0D7D725A90FEF13F02CD0C15192
:1059C000D8B4F9D7258327D0030E64EC2BF025A794
:1059D00004D0A751C163DED264D025B31CD0F5DA60
:1059E000050EBA6316D0C1C1ACF1BFC1AAF1C0C1E6
:1059F000ABF1A5C191F1A6C192F139C1F0F13AC163
:105A0000A8F1030EAA27000EAB23030E915F000E30
:105A1000925BBA2FBFD225A97DD7C6EC2AF0010E22
:105A2000E8CF7FF01A0E5BEC0BF0000EE8CF7FF0B2
:105A30000B0E5BEC0BF02099219121932197249977
:105A40002497B86B010E25B5AD51BA6F25952599F0
:105A50001BEC1DF0D0EC2FF021B3A7D221B10ED05A
:105A600020B10CEC3CF020B10BEC42F0209120B9BD
:105A70000FEF13F020B3F9EF48F0ECD72191060EA9
:105A8000BA6302D00FEF13F0BAC1ADF12585BB5157
:105A9000050DF350BA25A76F2FEC0FF02587C16BCA
:105AA00043D7259788EC1CF0000EE8CF7CF0000E61
:105AB000E8CF7DF020EE60F0230EDE6E1C0E90EC41
:105AC00010F0326703D0336701D016D0010E3227B1
:105AD000000E332332C152F133C153F1A7C154F147
:105AE000556BD7EC0BF050C132F151C133F11F8F20
:105AF0000A0E27EC0DF007D0A7C132F1386B382B16
:105B0000376B19EC0DF0200EDE6E0DEC2CF0C9CFCA
:105B100032F10DEC2CF0C9CF32F1BDC1AFF1BEC1F5
:105B2000AEF1200E64EC2BF0F0EC2BF0C9CFA9F114
:105B3000AFC1BDF1AEC1BEF132C1F1F10DEC2CF03F
:105B4000C9CFF2F10DEC2CF0C9CFF3F1C4EC23F086
:105B5000200EDE6E0DEC2CF0C9CF32F1386B382BF5
:105B6000376B19EC0DF03A0EDE6E0DEC2CF0C9CF50
:105B700032F1386B382B376B19EC0DF024EC0EF04A
:105B8000190EE8CF7CF0050EE8CF7DF020EE60F036
:105B90000DEC2CF0C9CF32F10DEC2CF0C9CF33F164
:105BA00032C14CF133C14DF1A40E4E6F4F6B0BEC73
:105BB0000CF048C1C6F149C1C7F1C62B000EC7237E
:105BC0001F8F030E27EC0DF06D0EDE6E200EDE6EC5
:105BD0000DEC2CF0C9CF32F10DEC2CF0C9CF33F124
:105BE00032C14CF133C14DF13C0E4E6F4F6BEEECB8
:105BF0000BF01F8F386B382B376B375127EC0DF0BC
:105C0000270EDE6E0DEC2CF0C9CF32F13251482751
:105C1000000E492348C14CF149C14DF19F0E4E6F12
:105C20004F6B0BEC0CF048C14CF149C14DF1A9513F
:105C30004E6F4F6B0BEC0CF048C1C8F149C1C9F174
:105C4000C82B000EC9231F8F386B382B376B19EC0C
:105C50000DF0220EDE6E200EDE6E0DEC2CF0C9CFA4
:105C600032F10DEC2CF0C9CF33F1030E386F1F8FDA
:105C7000020E27EC0DF0B00EDE6E430EDE6E24EC4D
:105C80000EF0320EE8CF7CF0050EE8CF7DF020EE6E
:105C900060F00DEC2CF0C9CF32F10DEC2CF0C9CF37
:105CA00033F11F8F386B382B376B375127EC0DF0E2
:105CB0006D0EDE6E620EDE6E610EDE6E720EDE6EDA
:105CC000200EDE6E440EDE6E650EDE6E730EDE6E30
:105CD000610EDE6E740EDE6E200EDE6E0DEC2CF0AC
:105CE000C9CF32F10DEC2CF0C9CF33F1B4EC0BF08D
:105CF0001F8F325133C132F1336F386B382B376B12
:105D00001EEC0DF03A0EDE6E33C132F1386B382BDB
:105D1000376B19EC0DF01F9F24EC0EF00DEC2CF0FE
:105D20000DEC2CF00DEC2CF00DEC2CF00DEC2CF01F
:105D30000DEC2CF00DEC2CF00DEC2CF00DEC2CF00F
:105D40000DEC2CF00DEC2CF00DEC2CF00DEC2CF0FF
:105D50000DEC2CF00DEC2CF00DEC2CF00DEC2CF0EF
:105D60000DEC2CF00DEC2CF0C9CFB1F1B199B19B39
:105D7000B19DB19FB12BB1C1EBF10DEC2CF0C9CFAE
:105D8000B2F1B299B29BB29DB29FB2C1ECF10DECEF
:105D90002CF0C9CFB3F10DEC2CF0C9CFB4F10DEC60
:105DA0002CF0C9CFB5F10DEC2CF0C9CFB6F10DEC4C
:105DB0002CF00DEC2CF0010EE8CFF4F14B0EE8CFF7
:105DC000F5F1EF0EE8CFF6F1000EE8CFF7F19F0EF8
:105DD000E8CFF8F1C7EC0EF00DEC2CF0B86B0DEC41
:105DE0002CF09E0E386F229F050EB96F4B0EDC6FA4
:105DF000B92931EC0EF0C8C1CAF1C9C1CBF1CB2B26
:105E000061D822BF23D0C6C14EF1C7C14FF132C104
:105E10004CF133C14DF10BEC0CF04B0E48273FEC2D
:105E20002FF048C1DCF1485140EC0EF0B92BB951CC
:105E300031EC0EF031EC1AF04AEC0EF0CA4F02D001
:105E400041D8FCD7CB2FFAD7382FD5D7209921911D
:105E5000219324992497B86BD0EC2FF021B177D0FF
:105E600021B31CD120B10CEC3CF020B10BEC42F082
:105E7000209120B96CD020B3F9EF48F0EDD748510C
:105E8000DC6301D012004851DC650ED0DCC149F161
:105E90004907495140EC0EF031EC1AF073EC0EF06A
:105EA00048514963F5D7120048C149F149074951A2
:105EB00040EC0EF031EC1AF073EC0EF0DC5149635B
:105EC000F5D712000DEC2CF0C9CF32F10DEC2CF00F
:105ED000C9CF33F10DEC2CF0C9CFB8F1289BB8BF76
:105EE000288BB89FFD0E326305D0FD0E336302D0C0
:105EF000228F1200B22F23D0ECC1B2F128AB11D007
:105F00000DEC2CF0B807000EC9B8020FC9BA010F8A
:105F1000EF6FEF6701D005D00DEC2CF0B807EF2F35
:105F2000FBD7040EB86306D00DEC2CF0B8070DECCF
:105F30002CF0B8070DEC2CF0B82FFCD71200B86786
:105F400001D012000DEC2CF0B82FFCD712002099D4
:105F5000B86BAAC1BDF1ABC1BEF191C1A5F192C1AF
:105F6000A6F1ACC1C1F1F0C139F1A8C13AF1C10744
:105F70002593BB07BC6B050EBA6FBB2B2FEC0FF044
:105F8000E6D425B38BEF2CF0BC6B050EBA6FBB2BA0
:105F90002FEC0FF0BFC1BDF1C0C1BEF1A7EF2CF0D7
:105FA00024B9218324B721811200BA2B070EBA63CA
:105FB00001D0E7D7BC29BA6302D0060EBA6FB86B1E
:105FC0001BEC1DF02499219345D52589BC2B29B5BF
:105FD0000CD0C6EC2AF0010EE8CF7FF01A0E5BEC75
:105FE0000BF0000EE8CF7FF02985140EE8CF7DF08E
:105FF000BB51050DF350C15D1E0DF350050FE8CFE9
:106000007CF020EE60F0C1C132F1386B382B376B79
:1060100019EC0DF0200EDE6E0DEC2CF0C9CF32F134
:106020000D0E326504D00DEC2CF0C9CF32F132C127
:10603000F1F10DEC2CF0C9CFF2F10DEC2CF0C9CF41
:10604000F3F11AEC24F00DEC2CF00DEC2CF0200EFA
:10605000DE6E0DEC2CF0C9CF32F10DEC2CF0C9CF77
:1060600033F11F8F2485030E27EC0DF06D0EDE6ECD
:10607000200EDE6E0DEC2CF0C9CF32F10DEC2CF0C1
:10608000C9CF33F11F8F386B382B376B375127EC63
:106090000DF0270EDE6E24EC0EF01200010EBA6F2A
:1060A00052EC28F0ECEC28F064EC28F020992191D7
:1060B000219324992497B86BD0EC2FF021B315D0FD
:1060C00021B10DD020B10CEC3CF020B10BEC42F032
:1060D000209120B93CD720B3F9EF48F0EDD7BA4F63
:1060E00036D7BA4F18D0BA4F07D0BA2B040EBA63BE
:1060F00002D0010EBA6FD8D748EC21F0BA6FBA6758
:1061000001D025D72FEC0FF00C0E5BEC0BF08AECD6
:1061100016F00FEF13F048EC21F0BA6FBA6701D018
:1061200016D72FEC0FF00C0E5BEC0BF0010E70ECA1
:106130002BF0BDC1A5F1BEC1A6F1010EBF27000E17
:10614000C023C0BFBF6BC0BFC06BA5C1BDF1A6C19E
:10615000BEF1F0EC2BF0C86FFE0EC86331D0BFC1AA
:10616000BDF1C0C1BEF1FE0E19EC2CF0010EBF272F
:10617000000EC023C0BFBF6BC0BFC06BBFC1BDF1AD
:10618000C0C1BEF1010EA527000EA623A6AF02D006
:10619000A56BA66BFF0E19EC2CF0010E64EC2BF036
:1061A000A5C152F1A6C153F1BDC154F1BEC155F113
:1061B000D7EC0BF05067EED75167ECD78AEF2CF095
:1061C000ABEC2BF0020E64EC2BF0BDC1C8F1BEC1EC
:1061D000C9F1020E70EC2BF0BDC1A5F1BEC1A6F154
:1061E000A5C1BDF1A6C1BEF1F0EC2BF0BFC1BDF160
:1061F000C0C1BEF119EC2CF0A5C1BDF1A6C1BEF124
:10620000FF0E19EC2CF0010EA527000EA623A6BF49
:10621000A56BA6BFA66B010EBF27000EC023C0BF93
:10622000BF6BC0BFC06BA5C152F1A6C153F1C8C1BD
:1062300054F1C9C155F1D7EC0BF05067D1D7516774
:10624000CFD78AEF2CF02D939D9A08EC4BF05DECA4
:106250004AF06B0EAD6EF8EC0DF00AEC4BF09D8A37
:1062600083EF3AF028959D9A08EC4BF020EC80F0F3
:10627000010130EC80F0010118EC80F00101010E09
:10628000CC6FCD6B680EAD6EF8EC0DF020850AEC8E
:106290004BF09D8A83EF3AF028939D9A08EC4BF0DF
:1062A000AA6AAAD80AEC4BF09D8A83EF3AF02A9F9B
:1062B0009D9A08EC4BF0010EAA6E9ED8AA6A0AECD1
:1062C0004BF09D8A83EF3AF0279F9D9A08EC4BF0A4
:1062D000F8EC0DF0010EAD6EF8EC0DF0360EAD6E73
:1062E00029EE4AF0100E396FF8EC0DF0DECFADFF5D
:1062F000392FFAD70AEC4BF09D8A83EF3AF0259BB1
:106300009D9A08EC4BF02FEC0FF0C6EC2AF0010E32
:10631000E8CF7FF00F0E5BEC0BF0000EE8CF7FF0C4
:10632000050E436FAA0EAD6EF8EC0DF0432FFAD7B1
:10633000550EAD6E100E5BEC0BF0ABEC2BF0010EBE
:10634000BD27000EBE23110E5BEC0BF055D8F8EC08
:106350000DF0C2C1ADFFF8EC0DF0C3C1ADFFF8EC1C
:106360000DF0010EAD6EF8EC0DF0360EAD6E120EA6
:106370005BEC0BF0436B446BC5803EEC2CF0A60E3F
:10638000C96E3EEC2CF0C5BCF7D7BEC1C9FF3EECD0
:106390002CF032EC2CF0BDC1C9FF3EEC2CF032ECFD
:1063A0002CF0C5823EEC2CF0A70EC96E3EEC2CF012
:1063B00032EC2CF0130E5BEC0BF0F8EC0DF0C58614
:1063C0003EEC2CF0C9CFADFF010E4327000E442355
:1063D00044BF04D0C5883EEC2CF0EFD7C5843EEC1A
:1063E0002CF0140E5BEC0BF0FA0ED8EC0CF00AEC6F
:1063F0004BF09D8A0EEF3AF0436BA96ACFEC0DF09B
:10640000A8CFADFFA92AF8EC0DF0432FF7D7120063
:10641000010EBA6F219921972099AA6B229D229F84
:106420002FEC0FF0C6EC2AF0010EE8CF7FF06F0ED4
:106430005BEC0BF0000EE8CF7FF0B86B219121935D
:10644000140EE8CF7DF0230EE8CF7CF020EE60F054
:10645000700E54EC0BF0AAC132F1322B1F8F386B47
:10646000382B376B08EC0DF0200EDE6E280EDE6E3A
:10647000C00E54EC0BF0200EDE6E210EA2EC0DF0DF
:10648000A8CFD1F1D105040DF350060FA96ECFECC2
:106490000DF0A8CF32F11F8F386B382B376B08EC1B
:1064A0000DF02F0EDE6ED105040DF350070FA96E0F
:1064B000CFEC0DF0A8CF32F11F8F386B382B376B34
:1064C00008EC0DF0290EDE6E24EC0EF0140EE8CF71
:1064D0007DF0410EE8CF7CF020EE60F0610E54ECD0
:1064E0000BF0AA51240FA96ECFEC0DF0A8CF32F11A
:1064F000336B1F8F030E27EC0DF01F9F420EDE6ED5
:10650000610EDE6E720EDE6E200EDE6E24EC0EF07C
:10651000140EE8CF7DF05F0EE8CF7CF020EE60F047
:10652000BE0E54EC0BF024EC0EF0140EE8CF7DF010
:106530007D0EE8CF7CF020EE60F0BF0E54EC0BF047
:1065400024EC0EF0140EE8CF7DF09B0EE8CF7CF02B
:1065500020EE60F0590E54EC0BF0310EDE6E2E0E74
:10656000DE6E300EDE6E300EDE6E24EC0EF00B0EA4
:106570005BEC0BF0F6EC12F01BEC1DF0D0EC2FF006
:1065800021B30FD021B11ED020B3F9EF48F020B1D4
:106590000CEC3CF020B10BEC42F0209120B91CD067
:1065A000EDD7BA2B020EBA6301D0BA2B070EBA632D
:1065B00002D0010EBA6FB86B1BEC1DF0F6EC12F0B6
:1065C0002193DCD7BA4F3ED0BA4F0AD0BA4F08D089
:1065D000BA4F1AD0BA4F2CD0020EBA6F63EF13F035
:1065E000AA51240FA96ECFEC0DF0A8CF32F1322BB7
:1065F000FB0E326302D0FA0E326F32C1A8FFD3EC29
:106600000DF0030EBA6F19D7AA51240FA96ECFEC63
:106610000DF0A8CF32F13207FF0E326302D0000E28
:10662000326F32C1A8FFD3EC0DF0040EBA6F05D75C
:10663000AA51240FA96E640EA86ED3EC0DF0050EBE
:10664000BA6FFBD6AA2B030EAA6301D0AA6B010E68
:10665000BA6FF3D62FEC0FF0C6EC2AF0010EE8CF9C
:106660007FF0720E5BEC0BF0000EE8CF7FF0230E94
:10667000E8CF7CF0000EE8CF7DF0000EE8CF7EF092
:1066800020EE60F0730E54EC0BF0320EA2EC0DF025
:10669000A8CF32F1330EA2EC0DF0A8CF33F11F8F4B
:1066A000386B382B376B375127EC0DF0200EDE6E30
:1066B000280EDE6E340EA2EC0DF0A8CF32F1350EAE
:1066C000A2EC0DF0A8CF33F11F8F386B382B376B4E
:1066D000375127EC0DF0290EDE6E24EC0EF0410E42
:1066E000E8CF7CF020EE60F0750E54EC0BF02F0E2E
:1066F000A2EC0DF0A8CFF1F1300EA2EC0DF0A8CF76
:10670000F2F1310EA2EC0DF0A8CFF3F1C4EC23F0BE
:1067100024EC0EF05F0EE8CF7CF020EE60F0760EF9
:1067200054EC0BF0280EA2EC0DF0A8CF32F1290E9C
:10673000A2EC0DF0A8CF33F1010E386F1F8F020EBF
:1067400027EC0DF01F9F560EDE6E24EC0EF07D0E32
:10675000E8CF7CF020EE60F0770E54EC0BF02A0EC0
:10676000A2EC0DF0A8CFF1F12B0EA2EC0DF0A8CF0A
:10677000F2F12C0EA2EC0DF0A8CFF3F1C4EC23F053
:1067800024EC0EF09B0EE8CF7CF020EE60F0780E4B
:1067900054EC0BF0360EA2EC0DF0A8CF32F1370E10
:1067A000A2EC0DF0A8CF33F1030E386F1F8F020E4D
:1067B00027EC0DF01F9FB00EDE6E200EDE6E280E51
:1067C000DE6E380EA2EC0DF0A8CFF1F1390EA2EC7E
:1067D0000DF0A8CFF2F13A0EA2EC0DF0A8CFF3F134
:1067E000C4EC23F0290EDE6E200EDE6E24EC0EF0DB
:1067F000B90EE8CF7CF020EE60F0790E54EC0BF08F
:106800003B0EA2EC0DF0A8CF32F13C0EA2EC0DF045
:10681000A8CF33F1030E386F1F8F020E27EC0DF057
:106820001F9FB00EDE6E200EDE6E280EDE6E3D0E59
:10683000A2EC0DF0A8CFF1F13E0EA2EC0DF0A8CF26
:10684000F2F13F0EA2EC0DF0A8CFF3F1C4EC23F06F
:10685000290EDE6E200EDE6E24EC0EF081A0FED737
:10686000249724992191D0EC2FF021B10DD020B3A1
:10687000F9EF48F020B10CEC3CF020B10BEC42F009
:10688000209120B901D0EFD7030EBA6F63EF13F058
:10689000010EBA6F2FEC0FF0B86B20992191219364
:1068A000C6EC2AF0010EE8CF7FF06A0E5BEC0BF02D
:1068B000000EE8CF7FF0AA6BA56B050E096F020EE4
:1068C0000A6F140EE8CF7DF0040E0A271E0E09276A
:1068D0000951E8CF7CF020EE60F0470EDE6EAAC1D1
:1068E00032F1322B1F8F386B382B376B08EC0DF0E1
:1068F0003A0EDE6E94EC38F024EC0EF0280EE8CF61
:106900007DF00951E8CF7CF020EE60F0210EA96EF9
:10691000CFEC0DF0A804AA6302D02A0EDE6E94EC30
:1069200038F024EC0EF0300EE8CF7DF00951E8CFBE
:106930007CF020EE60F00AC1A9FFA92ACFEC0DF08F
:10694000A8CF32F13253000E32651AD08DEC38F0F8
:106950000AC1A9FFCFEC0DF0A8CF32F1386B382B6C
:10696000376B1EEC0DF02F0EDE6EA92ACFEC0DF06A
:10697000A8CF32F1386B382B376B1EEC0DF03FD0BF
:106980000AC1A9FFCFEC0DF0A8CF32F13253150E9A
:10699000326517D0640E326108D086EC38F0386B5F
:1069A000382B376B1EEC0DF02AD04F0EDE6E320EF8
:1069B000DE6E200EDE6E386B382B376B1EEC0DF062
:1069C0001ED03263F2EC34F0410EDE6E490EDE6E04
:1069D000520EDE6E200EDE6E386B382B376B1EECDF
:1069E0000DF00DD0450EDE6E520EDE6E520EDE6ED6
:1069F000200EDE6E386B382B376B1EEC0DF094ECEE
:106A000038F024EC0EF0690EE8CF7DF00951E8CFA4
:106A10007CF020EE60F0200EDE6E690EDE6E6E0EF3
:106A2000DE6E200EDE6EAA511C0FA96ECFEC0DF0AB
:106A3000A8CF32F1386B382B376B1EEC0DF06D0E92
:106A4000DE6E94EC38F024EC0EF031EC1AF0AA2B48
:106A5000050EAA6361EF34F00B0E5BEC0BF0F6EC65
:106A600012F01BEC1DF0D0EC2FF021B30FD021B1B0
:106A70001ED020B3F9EF48F020B10CEC3CF020B16F
:106A80000BEC42F0209120B90ED0EDD7BA2B070EB7
:106A9000BA6302D0010EBA6FB86B1BEC1DF0F6ECB6
:106AA00012F02193E0D7020EBA6F12EF13F0BA4F33
:106AB00009D0BA4F0CD0BA4F0FD0BA4F12D0BA4F3C
:106AC00015D0F1D7000EAA6F000EA56F14D0010EDD
:106AD000AA6F040EA56F0FD0020EAA6F080EA56F45
:106AE0000AD0030EAA6F0C0EA56F05D0040EAA6F74
:106AF000100EA56F00D0010EBA6F2993219921972E
:106B00002099229D2FEC0FF01E0E5BEC0BF00B0E6C
:106B10005BEC0BF0B86B219121934ADA410EE8CF80
:106B20007CF0140EE8CF7DF020EE60F04F0EDE6EAC
:106B3000320EDE6E3A0EDE6E200EDE6EA551060FB0
:106B4000A96ECFEC0DF0A8CF32F1386B382B376B34
:106B50001EEC0DF0250EDE6E200EDE6E280EDE6EB3
:106B60004D0EDE6E4F0EDE6E440EDE6E3A0EDE6EA3
:106B7000120E7CEC10F00A0DF3CF4CF1F4CF4DF176
:106B8000A551060FA96ECFEC0DF0A8CF4EF14F6BBB
:106B90000BEC0CF00A0E485F48C132F1000E495B65
:106BA00049C133F1386B382B376B375127EC0DF077
:106BB0006D0EDE6E290EDE6E200EDE6E200EDE6E97
:106BC00024EC0EF05F0EE8CF7CF020EE60F0480E73
:106BD000DE6E650EDE6E3A0EDE6E200EDE6EA551A6
:106BE000070FA96ECFEC0DF0A8CF32F1386B382B20
:106BF000376B1EEC0DF0250EDE6E200EDE6E200EC5
:106C0000DE6E24EC0EF07D0EE8CF7CF020EE60F01E
:106C10002B0EDE6E2F0EDE6E2D0EDE6E3A0EDE6E4B
:106C2000200EDE6E2B0E22BD2D0EDE6E24EC0EF03D
:106C30009B0EE8CF7CF020EE60F0590E54EC0BF088
:106C4000A551040FA96ECFEC0DF0A8CF32F1386B2F
:106C5000382B376B1EEC0DF02F0EDE6EA551050F95
:106C6000A96ECFEC0DF0A8CF32F1386B382B376B13
:106C70001EEC0DF0200EDE6E200EDE6E24EC0EF00B
:106C8000F6EC12F01BEC1DF0D0EC2FF021B30FD07E
:106C900021B11AD020B3F9EF48F020B10CEC3CF050
:106CA00020B10BEC42F0209120B918D0EDD7BA2BCF
:106CB000070EBA6302D0010EBA6FB86B1BEC1DF061
:106CC000F6EC12F02193E0D7BA4F90D0BA4F11D022
:106CD000BA4F43D0BA4F06D0BA4F69D0AAC1BAF161
:106CE000BA2BD8D5227D040EBA6F14D7010EBA6F15
:106CF00009D7A551060FA96ECFEC0DF0A8CF32F140
:106D000022BD07D0322B650E326310D0040E326FD5
:106D10000DD03207030E326309D0A551070FA96EBB
:106D2000CFEC0DF0640E326FA850325FA551070F03
:106D3000A96ECFEC0DF0A8503225336F650E33638A
:106D400002D0040E326FA551060FA96E32C1A8FF02
:106D5000D3EC0DF0020EBA6FDDD6A551070FA96E68
:106D6000CFEC0DF0A8CF32F122BD06D0322B5C0E55
:106D7000326307D0326B05D03207FF0E326301D089
:106D8000326BA551060FA96ECFEC0DF0A85032253D
:106D9000336F650E336301D03207A551070FA96E1B
:106DA00032C1A8FFD3EC0DF0030EBA6FB3D6A551D4
:106DB000040FA96ECFEC0DF0A8CF32F1A551050F4D
:106DC000A96ECFEC0DF0A8CF33F1A551060FA96E37
:106DD00032C1A8FFD3EC0DF0A551070FA96E33C146
:106DE000A8FFD3EC0DF0050EBA6F94D62FEC0FF080
:106DF000010EBA6F6D0E5BEC0BF00B0E5BEC0BF043
:106E0000B86B21912193D4D8A4D9410EE8CF7CF05E
:106E1000140EE8CF7DF020EE60F0690E54EC0BF01C
:106E20001B0EA2EC0DF0AAC132F1322BA832322F88
:106E3000FDD7D8A004D0600E54EC0BF006D0200E85
:106E4000DE6E200EDE6E200EDE6E24EC0EF05F0E87
:106E5000E8CF7CF0140EE8CF7DF020EE60F0580E05
:106E600054EC0BF0200EDE6E210EA96ECFEC0DF06F
:106E7000A804AA6304D0600E54EC0BF006D0200ED8
:106E8000DE6E200EDE6E200EDE6E24EC0EF07D0E29
:106E9000E8CF7CF0140EE8CF7DF020EE60F06B0EB2
:106EA00054EC0BF024EC0EF09B0EE8CF7CF0140EAB
:106EB000E8CF7DF020EE60F06C0E54EC0BF024EC8B
:106EC0000EF0F6EC12F01BEC1DF0D0EC2FF021B31D
:106ED0000FD021B11AD020B3F9EF48F020B10CEC5B
:106EE0003CF020B10BEC42F0209120B9F7D6EDD761
:106EF000BA2B070EBA6302D0010EBA6FB86B1BEC47
:106F00001DF0F6EC12F02193E0D7BA4FEFD6BA4F4E
:106F100011D0BA4F05D0BA4F23D0BA4F35D0DED6F4
:106F2000AAC1A8FFA82A210EA96ED3EC0DF0030E6A
:106F3000BA6F66D71B0EA2EC0DF0AAC132F1322B4C
:106F4000324FA870324FA872324FA874324FA876D1
:106F5000324FA8781B0EA0EC0DF0020EBA6F50D77E
:106F6000AA511C0FA96ECFEC0DF0A8CF32F1322B35
:106F7000640E326302D0630E326F32C1A8FFD3ECCD
:106F80000DF0040EBA6F3CD7AA511C0FA96ECFECBE
:106F90000DF0A8CF32F13207FF0E326302D0000E9F
:106FA000326F32C1A8FFD3EC0DF0050EBA6F28D7AF
:106FB000C6EC2AF0010EE8CF7FF0020EE8CF7CF09D
:106FC000000EE8CF7DF020EE60F05F0E54EC0BF089
:106FD000AAC132F1322B1F8F386B382B376B08EC7C
:106FE0000DF03A0EDE6E200EDE6E24EC0EF0020E78
:106FF000E8CF7CF0320EE8CF7DF020EE60F0A551B6
:10700000070FA96ECFEC0DF0A8CF32F13253000E6E
:1070100032651DD08DEC38F0A551060FA96ECFEC6E
:107020000DF0A8CF32F1386B382B376B1EEC0DF01A
:107030002F0EDE6EA551070FA96ECFEC0DF0A8CF75
:1070400032F1386B382B376B1EEC0DF041D0A55167
:10705000060FA96ECFEC0DF0A8CF32F13253150E0A
:107060003263326517D0640E326108D086EC38F096
:10707000386B382B376B1EEC0DF02AD04F0EDE6EBE
:10708000320EDE6E200EDE6E386B382B376B1EEC48
:107090000DF01ED032630ED0410EDE6E490EDE6E54
:1070A000520EDE6E200EDE6E386B382B376B1EEC08
:1070B0000DF00ED0450EDE6E520EDE6E520EDE6EFE
:1070C000200EDE6E386B382B376B1EEC0DF000D0C7
:1070D000200EDE6E690EDE6E6E0EDE6E200EDE6E31
:1070E000AA511C0FA96ECFEC0DF0A8CF32F1386B6E
:1070F000382B376B1EEC0DF06D0EDE6E200EDE6E43
:1071000024EC0EF0000EE8CF7FF012004E0EDE6E83
:10711000580EDE6E200EDE6E1200540EDE6E580E1D
:10712000DE6E200EDE6E12001B0EA2EC0DF0AAC168
:1071300032F1322BA832322FFDD7D8A006D0230E41
:107140007CEC10F024EC10F01200490E24EC10F04E
:107150001200A551060FA96ECFEC0DF0A8CF33F1A8
:10716000AA511C0FA96ECFEC0DF0A8CF32F10A0E78
:10717000322733513203F3CF4CF1F4CF4DF10A0EE5
:107180004E6F4F6B0BEC0CF048C132F149C133F13B
:10719000370EE8CF7DF0230EE8CF7CF020EE60F0D4
:1071A000280EDE6E700EDE6E700EDE6E4F0EDE6E20
:1071B000320EDE6E3A0EDE6E030E27EC0DF0420E3E
:1071C000DE6E610EDE6E720EDE6E290EDE6E200E3B
:1071D000DE6E24EC0EF0120025BD1FD0AECF43F1C1
:1071E000600E435F434F258B434F248B434F258DC8
:1071F000434F2681434F278F434F2881434F288396
:10720000434F2885434F2B81434F2A8F434F2D8374
:10721000AE509E9AAB98AB8812002CB7F9D708EC09
:107220004BF0AE6601D0AE2AAE50640DF3CFC6F17E
:10723000F4CFC7F1EDD7F292D5BE09D02487D58E11
:107240001200F090D5BE03D02489D58E1200F2949E
:10725000D56AD76AD66AD58E1200F294D59ED76ABF
:10726000D66A1200F19C2A91000ED56ED58E1200BE
:10727000F18C1200F19A2A93000ED56ED58E120071
:10728000F18A1200A192B19ECA9412009E9000EC65
:107290004BF0080ECF60412B080ECF5E412B0F0E36
:1072A000416502D0B4EC39F020A901D0120023BF0F
:1072B0001200422B010E42630AD0239D3F6B406BAC
:1072C0009B6B9C6B07EC19F0F7EC18F01200020EA8
:1072D00042630FD0FEEC18F004EC19F0DFEC17F06D
:1072E0008D513F278E51402397519B2798519C23C6
:1072F0001200030E426301D0E5D7040E426301D0B1
:10730000E9D7050E426301D0DDD7060E426301D0F6
:10731000E1D7070E426301D0D5D7DCDF426B020E06
:107320003E6FD89040333F33D8909C339B333E2FF1
:10733000F8D740C18EF13FC18DF19CC198F19BC13E
:1073400097F1238D25AD04D0E80E9F6F030EA06F3B
:107350001F979F518D5D8F6FA0518E59906FD8A848
:1073600012008F6B906B1200416B2081D89420A388
:107370001CD0A82BA905A86502D0A86B2287172BC3
:10738000D8B4182B22A911D0A72B3B0EA76505D086
:10739000A76B2087A52BD8B4A62B2AAB06D0DD2B54
:1073A0003B0EDD6502D0DD6BDC2B032B3B0E036552
:1073B0001200036B2085042B3B0E04651200046B46
:1073C000052B170E05651200056B062B2A0E036FA1
:1073D00007C176F1764F1F0E764F1C0E764F1F0EAB
:1073E000764F1E0E764F1F0E764F1E0E764F1F0ED7
:1073F000764F1F0E764F1E0E764F1F0E764F1E0EC7
:10740000764F1F0E06651200010E066F072B0C0E3D
:1074100007651200010E076F082B120043EC49F0BC
:10742000326B32C118F5B6EC0FF046EC2CF0E1EC03
:107430000DF06DEC0FF0DCEC25F0A4EC1CF04EEC44
:1074400024F0A3C100F5A4C101F5A3C102F5A4C1B4
:1074500003F528BF10D02ABB0ED07FEC22F0B4EC8D
:1074600022F02DA542EC29F02DB505EC20F0B3EC6F
:1074700020F04DEC1FF028AF03D0670E5BEC0BF053
:107480002AAB03D0740E5BEC0BF0B86BB96B209D8C
:10749000209F239D956B966B996B9A6B050EB76F2A
:1074A0000AEC4BF0FCEC4AF0259D2C97000EE8CF3F
:1074B0007CF0000EE8CF7DF0000EE8CF7EF0000EED
:1074C000E8CF7FF031EC1AF024972499B3EC20F048
:1074D00008EC2BF0010ECF6F470E3DEC1AF00C0EAE
:1074E0007CEC10F00A6F0AC113F50B0E7CEC10F067
:1074F0000A6F0AC112F530EC80F00101480E3DEC34
:107500001AF0F6EC12F020A119D029A101D000D078
:10751000A4EC1CF03EEC3BF00CEC3CF0B8EC46F07C
:107520001AEC23F0C8EC3BF011EC3BF071EC12F0DC
:107530004DEC1FF02CB18AEF46F02091E5EC3BF0CA
:1075400023BDECEC22F023BD60EC1EF023BD0BEC60
:1075500042F0239D20B5D5EC3AF020BF0FEF13F099
:1075600020B318EF3CF020B9CDEF45F025BB7FEFFD
:1075700031F024BB34EF48F026B1A9EF0DF02BB168
:10758000A4EF0DF027BF64EF31F028B18AEF48F087
:1075900028B34CEF31F028B532EF31F02ABF57EF66
:1075A00031F02DB323EF31F0AED74EEC24F015ECD3
:1075B0003BF0DDEC47F008EC2BF001EC3BF028BF92
:1075C0000ED02ABB0CD0B4EC22F07FEC22F020BD10
:1075D00006D02DA542EC29F02DB505EC20F0F3ECFA
:1075E0003AF0209512002781010ECC5F000ECD5B92
:1075F000CC671200CD67120027910EEC4BF0CC2B1C
:10760000120020C532F121C533F1326705D033674E
:1076100003D0196B1A6B1200010E1927000E1A23E2
:10762000120027B110EC4BF0120004EC4BF0490EA5
:107630003DEC1AF09FC102F5A0C103F50A6B0AC127
:1076400011F54F0E0A6F0AC110F58DC100F58EC1FC
:1076500001F50B0E7CEC10F00A6F0AC112F50C0E4E
:107660007CEC10F00A6F0AC113F540EC80F00101C8
:107670004A0E3DEC1AF006EC4BF012009492828216
:10768000249182A42481829294820A0EACEC0CF0A4
:10769000249382A424839492829224B174D024B33C
:1076A00064D0948229A944D0299F2999320EA2EC52
:1076B0000DF0A8CF39F1330EA2EC0DF0A8CF3AF1BE
:1076C000D890010E3927000E3A2339C1A8FF320E97
:1076D000A0EC0DF03AC1A8FF330EA0EC0DF0340E73
:1076E000A2EC0DF0A8CF39F1350EA2EC0DF0A8CF29
:1076F0003AF1D890010E3927000E3A2339C1A8FF7C
:10770000340EA0EC0DF03AC1A8FF350EA0EC0DF040
:1077100007C1A8FF2F0EA0EC0DF006C1A8FF300E88
:10772000A0EC0DF008C1A8FF310EA0EC0DF0120086
:1077300029AF1200299F320EA2EC0DF0A8CF39F12B
:10774000330EA2EC0DF0A8CF3AF1D890010E3927F4
:10775000000E3A2339C1A8FF320EA0EC0DF03AC159
:10776000A8FF330EA0EC0DF01200FEEC4AF0640E00
:10777000D8EC0CF000EC4BF0640ED8EC0CF0FEEC06
:107780004AF029891200FEEC4AF0298F299912004B
:1077900020AD1200B92B040E7CEC10F0B96512007C
:1077A000209DC4EC2AF028BF08D02ABB06D02DA506
:1077B00042EC29F02DB505EC20F0ECEC22F0DCECED
:1077C00025F0B96B24972499120024B718D024B956
:1077D00007D0D59EF294D76AD66AF292F090120042
:1077E0002499C6EC2AF0010EE8CF7FF0040E5BEC82
:1077F0000BF0000EE8CF7FF0208DB86B12002497BD
:1078000020AD02D0208F12002D752DA542EC29F05D
:107810002DB505EC20F01200B82B030E7CEC10F017
:10782000050FD8B0FF0EE806B865120020891200D7
:1078300056EC42F0520E3DEC1AF02FEC0FF034EC07
:107840001BF0F8EC1EF08EEC1EF02ABB208728BF40
:1078500004D02ABB02D058EC1BF020A142D028BF94
:1078600009D02ABB17D029B118D02CEC3FF0F4EC8A
:107870003CF01BD020ADA6EC24F099EC41F02CB3E9
:107880007BEC25F024BF04D0248F31EC42F00DD0E6
:10789000249F0BD0A1EC3CF008D030EC2AF0F4ECA3
:1078A0003CF02CB52EEC3FF000D099EC41F023B722
:1078B0001AEC23F020BD97EC3CF020BF81EC45F0A2
:1078C000D1EC3CF02CB18AEF46F02CB37BEC25F0E8
:1078D0002091260E7CEC10F0326F010E326301D045
:1078E000268326A30BD020BD08D0A6EC24F029B116
:1078F00030EC2AF027B52CEC3FF0269320AF12ECA9
:1079000043F020BF57EC43F020A3ADD323BDBEEC22
:1079100041F0239D20B5DDEC41F022B711EC3EF0A3
:1079200020BF04D025BD02D00300000096D7B92B9C
:10793000040E7CEC10F0B9651200209D6CEC24F074
:10794000120015EC25F022B90DD0D6EC24F0E22B74
:107950003C0EE26302D0E26BE12B269722B91200C3
:107960002687120026A712000BD803EC25F0E06B47
:10797000E26BE16BDD6BDC6B916B926B2697120017
:10798000DEC152F1DFC153F191C154F192C155F101
:10799000D7EC0BF01FA7120091C1DEF192C1DFF10D
:1079A0001200FCEC4AF032C532F10E0E7CEC10F005
:1079B0003261EEEC3CF027BBFAEC4AF01FC532F125
:1079C000322D120066C532F10E0E7CEC10F03261E1
:1079D000EEEC3CF027BBFAEC4AF01200FAEC4AF06D
:1079E000020EB06F288B120024BFCFD0248F31EC51
:1079F00042F0F7EC3EF08DC14CF18EC14DF10A0E14
:107A00004E6F000E4F6B0BEC0CF048C14CF149C1AE
:107A10004DF1D0C14EF14F6BEEEC0BF048C14CF183
:107A200049C14DF1640E4E6F000E4F6B0BEC0CF024
:107A300048C107F529B118C507F528EC80F0010108
:107A400065C532F11B0E7CEC10F0325DD8B0DAEC7B
:107A50002AF087EC3FF025A18DD08FC14CF190C169
:107A60004DF1640E4E6F4F6B0BEC0CF0326B1B0E36
:107A7000A2EC0DF0A8A00AD01C0EA2EC0DF048510B
:107A8000A86004D0A8CF32F1010E336F1B0EA2EC18
:107A90000DF0A8A210D01D0EA2EC0DF04851A86068
:107AA0000AD01D0EA2EC0DF03251A86404D0A8CF6C
:107AB00032F1020E336F1B0EA2EC0DF0A8A410D011
:107AC0001E0EA2EC0DF04851A8600AD01E0EA2ECCA
:107AD0000DF03251A86404D0A8CF32F1030E336FF9
:107AE0001B0EA2EC0DF0A8A610D01F0EA2EC0DF0FC
:107AF0004851A8600AD01F0EA2EC0DF03251A864C4
:107B000004D0A8CF32F1040E336F1B0EA2EC0DF09F
:107B1000A8A810D0200EA2EC0DF04851A8600AD001
:107B2000200EA2EC0DF03251A86404D0A8CF32F19F
:107B3000050E336F450E3DEC1AF0330732C11BF5CD
:107B40003351040DF350070FA96ECFEC0DF0A8CF01
:107B50001DF53351040DF350060FA96ECFEC0DF057
:107B60001DC50AF1D880640E0A55D880A856A8CF42
:107B70001CF50AD0460E3DEC1AF0326B32C11BF5F3
:107B800032C11CF532C11DF51200249F28BF12001E
:107B90002ABB1200420E3DEC1AF0E7EC3DF000EC7F
:107BA00080F00101430E3DEC1AF023C5CEF1CE6703
:107BB00012002BC50AF10A6729D025B158EC1BF039
:107BC0002591AA6B22C5ABF16BEC1BF012008DC1A5
:107BD00000F58EC101F50B0E7CEC10F00A6F0AC1A6
:107BE00012F50C0E7CEC10F00A6F0AC113F5100EA2
:107BF0007CEC10F00A6F0AC117F51D0E7CEC10F03A
:107C00000A6F0AC11EF543EC49F0120025A18FEC62
:107C10001BF025812BC5AAF124C5ABF198EC1BF014
:107C200012002297268306EC4BF022BB08D0228B51
:107C3000BDC1BFF1BEC1C0F12F0E64EC2BF08F515E
:107C40007CEC2BF090517CEC2BF0AE6BB12D02D084
:107C5000020EAE27B22D02D0020EAE27B32D02D0F7
:107C6000020EAE27B42D02D0030EAE27B52D02D0E2
:107C7000090EAE27B62D02D0000EAE2728AB11D0CC
:107C8000010EAE27AF6BB051AF27B06B28A703D062
:107C9000020EAE27AF8928A903D0010EAE27AF8B05
:107CA000AE8FAE517CEC2BF028AB16D0AF517CECF4
:107CB0002BF028A70CD0180EA2EC0DF0A8507CECED
:107CC0002BF0190EA2EC0DF0A8507CEC2BF028A99B
:107CD00003D0D1517CEC2BF0289B28972899B12F09
:107CE00001D07AD8B22F01D06CD8B32F01D05ED892
:107CF000B42F01D04DD8B52F01D018D8B62F01D050
:107D000010D8B1BFB16BB2BFB26BB3BFB36BB4BF6E
:107D1000B46BB5BFB56BB6BFB66B440E3DEC1AF095
:107D200012001A0E7CEC10F0B66F120031C9B5F1DA
:107D3000B5517CEC2BF030C9B5F1B5517CEC2BF092
:107D400033C9B5F1B5517CEC2BF032C9B5F1B55161
:107D50007CEC2BF035C9B5F1B5517CEC2BF034C976
:107D6000B5F1B5517CEC2BF037C9B5F1B5517CECD0
:107D70002BF036C9B5F1B5517CEC2BF038C9B5F113
:107D8000B5517CEC2BF0190E7CEC10F0B56F1200A5
:107D9000000E7CEC2BF0000E7CEC2BF0000E7CEC4B
:107DA0002BF0180E7CEC10F0B46F1200000E7CEC7F
:107DB0002BF0000E7CEC2BF0170E7CEC10F0B36F68
:107DC0001200AA517CEC2BF0AB517CEC2BF0160E80
:107DD0007CEC10F0B26F120097517CEC2BF09851B4
:107DE0007CEC2BF0150E7CEC10F0B16F120020A390
:107DF0002DD08DC152F18EC153F195C154F196C170
:107E000055F18DC195F18EC196F1D7EC0BF050C1B3
:107E10004CF151C14DF1270E4E6F4F6BEEEC0BF054
:107E200048C145F149C146F1070E476FC1EC0BF05F
:107E3000630E456501D0456F050E7CEC10F0455D85
:107E4000D8A004D0218B5AEC1CF0120021AB1200F8
:107E5000219B7EEC1CF0120029B112008DC14CF167
:107E60008EC14DF10A0E4E6F4F6B0BEC0CF048C1FA
:107E70004CF149C14DF1D0C14EF14F6BEEEC0BF01E
:107E800048C154F149C155F1130E7CEC10F0640D5A
:107E9000F3CF52F1F4CF53F1D7EC0BF027951FB786
:107EA0002785279B48C154F149C155F1120E7CEC3E
:107EB00010F0640DF3CF52F1F4CF53F1D7EC0BF087
:107EC0001FA704D0278B050EB06F288B48C154F133
:107ED00049C155F1110E7CEC10F0640DF3CF52F155
:107EE000F4CF53F1D7EC0BF01FB705D0278B2785C4
:107EF000040EB06F288B27B506D027A307D0E4EC7B
:107F00001EF0279303D0BCEC1EF0278312002C9D9B
:107F10008FC14CF190C14DF1640E4E6F4F6B0BEC65
:107F20000CF01B0EA2EC0DF0A8A011D0010ED16335
:107F300001D00DD01C0EA2EC0DF0030EA86407D0EA
:107F40004851A86404D0030EA85C48612C8D1B0E18
:107F5000A2EC0DF0A8A211D0020ED16301D00DD079
:107F60001D0EA2EC0DF0030EA86407D04851A864C2
:107F700004D0030EA85C48612C8D1B0EA2EC0DF002
:107F8000A8A411D0030ED16301D00DD01E0EA2EC17
:107F90000DF0030EA86407D04851A86404D0030E66
:107FA000A85C48612C8D1B0EA2EC0DF0A8A610D089
:107FB000040ED16301D00CD01F0EA2EC0DF0A8640A
:107FC00007D04851A86404D0030EA85C48612C8DEA
:107FD0001B0EA2EC0DF0A8A810D0050ED16301D0A5
:107FE0000CD0200EA2EC0DF0A86407D04851A86474
:107FF00004D0030EA85C48612C8DF8EC1EF0120032
:1080000020C54CF121C54DF14C6707D04D6705D017
:10801000010ECC6FCD6B279112004CC104F54DC100
:1080200005F50D0E7CEC10F04E6F4EC106F54B0EB3
:108030003DEC1AF01CEC80F001014C0E3DEC1AF006
:1080400004C54CF105C54DF14C6707D04D6705D00F
:10805000010ECC6FCD6B279112004CC1CCF14DC1FC
:10806000CDF12781120020A78FEF41F02ABB88DCD9
:10807000A3C100F5A4C101F50C0E7CEC10F00A6F51
:108080000AC113F5470E3DEC1AF030EC80F0010107
:10809000B7DF480E3DEC1AF0FD0E7CEC2BF0FD0E28
:1080A0007CEC2BF0FE0E7CEC2BF0BFC1BDF1C0C10F
:1080B000BEF1FA0E7CEC2BF0FA0E7CEC2BF0200ECD
:1080C0007CEC2BF007517CEC2BF006517CEC2BF078
:1080D00008517CEC2BF005517CEC2BF004517CEC2E
:1080E0002BF02AAB11D0DEC132F1DFC133F144EC09
:1080F0002BF032C1DEF133C1DFF1DE517CEC2BF02D
:10810000DF517CEC2BF010D091C132F192C133F1F0
:1081100044EC2BF032C191F133C192F191517CECDE
:108120002BF092517CEC2BF0A5517CEC2BF0A6515E
:108130007CEC2BF0A7517CEC2BF0AC517CEC2BF0C1
:10814000AD517CEC2BF0A3517CEC2BF0A4517CECDA
:108150002BF020C532F121C533F132517CEC2BF0EC
:1081600033517CEC2BF0060EA2EC0DF0A8507CEC09
:108170002BF0070EA2EC0DF0A8507CEC2BF00A0EB1
:10818000A2EC0DF0A8507CEC2BF00B0EA2EC0DF045
:10819000A8507CEC2BF00E0EA2EC0DF0A8507CEC5D
:1081A0002BF00F0EA2EC0DF0A8507CEC2BF0120E71
:1081B000A2EC0DF0A8507CEC2BF0130EA2EC0DF00D
:1081C000A8507CEC2BF0160EA2EC0DF0A8507CEC25
:1081D0002BF0170EA2EC0DF0A8507CEC2BF0180E33
:1081E000A2EC0DF0A8507CEC2BF0190EA2EC0DF0D7
:1081F000A8507CEC2BF0210EA2EC0DF0A8507CECEA
:108200002BF0010E7CEC2BF0360E7CEC2BF0C251E7
:108210007CEC2BF0C3517CEC2BF0140E7CEC10F0BA
:108220002ABB010E7CEC2BF0020E396F393B150E88
:108230007CEC10F039257CEC2BF0020E396F393BC9
:10824000160E7CEC10F039257CEC2BF0020E396F09
:10825000393B170E7CEC10F039257CEC2BF0030E2B
:10826000396F393B180E7CEC10F039257CEC2BF083
:10827000090E396F393B190E7CEC10F039257CEC76
:108280002BF0000E396F393B1A0E7CEC10F03925BB
:108290007CEC2BF01A0EA2EC0DF0A8507CEC2BF02D
:1082A000000E7CEC2BF0FB0E7CEC2BF0FB0E7CEC40
:1082B0002BF0020EA2EC0DF0A8CF39F1030EA2ECC8
:1082C0000DF0A8CF3AF1D890010E3927000E3A23CD
:1082D00039C1A8FF020EA0EC0DF03AC1A8FF030EB1
:1082E000A0EC0DF01C0E90EC10F0326703D0336759
:1082F00001D012D0010E3227000E3323700E820FF0
:10830000A96E32C1A8FFD3EC0DF0700E830FA96ED9
:1083100033C1A8FFD3EC0DF0259D0AEC4BF02DB135
:1083200068EC4AF060EC80F00101196B1A6B0EEFFB
:108330003AF020A712002ABB0ED025BD19D02093F9
:10834000B72B020E7CEC10F0020FD8B0FF0EE8063F
:10835000B76520831200B72B3C0EB7631200B76BD2
:108360002093E02B1E0E7CEC10F0E06320831200C3
:108370002093B72B050EB765208312000BEC42F05B
:1083800020B3E7EC41F020B3FAEC41F0219D975186
:108390009963218D98519A63218D21BD8EEC1EF039
:1083A000219F8D519563218F8E519663218F25BD1D
:1083B000218F21BFCBEC21F01200B8EC46F021EC6C
:1083C00042F07EEC24F0DDEC47F02095120091C1E4
:1083D00052F192C153F18FC154F190C155F1D7ECD4
:1083E0000BF01FA712008FC191F190C192F17EECAA
:1083F00024F01200ACC152F1ADC153F197C154F158
:1084000098C155F1D7EC0BF01FB7120097C1ACF132
:1084100098C1ADF112002299000E7CEC10F0526F61
:10842000536B8FC154F190C155F1D7EC0BF01FA7DE
:1084300005D020B7B76B20832289120020A7209394
:10844000120023B709D00C0EC36501D01200070E2D
:10845000B06F288B238712000D0EC365F8D72397C2
:1084600012008FC115F190C116F115511127165147
:108470001223000E13231423155111271651122312
:10848000000E1323142317C14EF118C14FF111C16F
:1084900048F112C149F113C14AF114C14BF132EC58
:1084A0000CF048C193F149C194F11200510E3DEC1A
:1084B0001AF0916B926B936B946BEDEC0FF05A0E7C
:1084C000A2EC0DF0000EA864B6EC0FF0116B126B6D
:1084D000136B146B010E176F186B010EDE6FDF6BE1
:1084E000E16BE26BDC6BDD6BA56BA66BA76BA86B1E
:1084F000E06BB76BB86BB06B289B2B9BD269E86BBA
:1085000025912C952C9DABEC2BF0A4C103F5A3C1B8
:1085100002F597C1ACF198C1ADF10A6B0AC14EF2F8
:108520000AC14FF202EE50F0200E0A6FEE6A0A2FD7
:10853000FDD702EE70F0200E0A6F010EEE6E0A2FCC
:10854000FCD702EE90F0EE6AEE6A200E7CEC10F0A2
:10855000A8CF15F5210E7CEC10F0A8CF14F52C83D4
:10856000290E7CEC10F0326F010E32632C93140E46
:108570007CEC10F0A96F150E7CEC10F0B16F160EAC
:108580007CEC10F0B26F170E7CEC10F0B36F180E8D
:108590007CEC10F0B46F190E7CEC10F0B56F1A0E75
:1085A0007CEC10F0B66F2AAB02D0010EA96F240E3E
:1085B000A2EC0DF029B1A8CF18F5A8CF59F10EEC17
:1085C0004BF02397229B209D2097268325ADF0EC2E
:1085D0000DF0210EA2EC0DF0A8CFD1F1D105040DC4
:1085E000F350070FA96ECFEC0DF0A8CF11F5D10510
:1085F000040DF350060FA96ECFEC0DF0A8CFD0F10B
:1086000011C50AF1D880640E0A55D880A856A8CFA3
:1086100010F5326B32C11BF532C11CF532C11DF5AC
:108620002B95120024B718D024A91200249724995E
:108630002A99208D209FB96B2ABB0AD0010EE8CF62
:108640007FF0040E5BEC0BF0000EE8CF7FF0120021
:108650008D0E5BEC0BF012002497249920AD14D002
:108660002AAB03D02093209D1200208F209D52EC36
:1086700028F01EEC26F02C992B9F010EBA6F64ECAB
:1086800028F02499249712002CB7ABD004EC4BF0BF
:10869000060EB06F288B2CA31200116B126B136B9C
:1086A000146B020E176F186B31EC42F0120024B7F6
:1086B00015D024A912002DB9FFD026B91CD126BD92
:1086C000F3D02499B96BBA2B060E2BBD040EBA63F6
:1086D00002D0010EBA6F64EC28F01200249724999E
:1086E000208F209DB96B2DB9E7D026BBB0D126B91C
:1086F00002D126BDD9D026B500D12CB900EF44F067
:108700002BBF0BD0BA4FDAD0BA4F8AD1BA4F53D061
:10871000BA4F45D0BA4F0BD21200BA4FBCD0BA4FA5
:1087200017D0BA4FC3D0BA4F03D0BA4F00D21200FD
:108730002C732CA30AD0116B126B136B146B020EEB
:10874000176F186B31EC42F0F2D169EC25F0EFD1E4
:108750005A0EA2EC0DF0A86608D0EDEC0FF0010E59
:10876000A86E5A0EA0EC0DF007D0B6EC0FF0000E7C
:10877000A86E5A0EA0EC0DF0F8EC1EF08EEC1EF078
:10878000CBEC21F07EEC24F02ABBD1D128BFCFD195
:1087900025B18FEC1BF025A158EC1BF0C8D152EC91
:1087A00028F03CEC26F0010EBA6F2B8F64EC28F019
:1087B00024992497120029B126D1268552EC28F05D
:1087C000D0C1A8FF180EA0EC0DF011C5A8FF190E1E
:1087D000A0EC0DF04FEC26F0010EBA6F64EC28F01F
:1087E0001200208F209D249924972C8952EC28F088
:1087F00088EC26F02B9F010EBA6F64EC28F0120073
:10880000BA4F95D1BA4F39D0BA4F3ED0BA4F2ED0C9
:10881000BA4F25D08CD188EC26F0980E526F3A0EC4
:10882000536FC6C154F1C7C155F1D7EC0BF01FA768
:1088300005D0980EC66F3A0EC76F1200E80E526F41
:10884000030E536FC6C154F1C7C155F1D7EC0BF0FD
:108850001FB71200E80EC66F030EC76F1200E80EB6
:10886000C65F030EC75B050EBA6FD5D7E80EC627E5
:10887000030EC723040EBA6FCED7640EC627000EB0
:10888000C723020EBA6FC7D7640EC65F000EC75B60
:10889000030EBA6FC0D7268D52EC28F030EC80F072
:1088A00001013FEC29F01200269D41D12D8952ECA7
:1088B00028F06EEC2AF012002D9939D12689220E6B
:1088C000A2EC0DF0030EA8640DD00CD02B852FEC7C
:1088D0000FF042EC2BF023C5CEF1CE67120043EC33
:1088E0002BF0120052EC28F023C5CEF1CE67120017
:1088F000D2EC26F0120026991AD1BA4F6FD0BA4F97
:108900004ED0BA4F38D0BA4F17D0BA4F01D012005C
:10891000190EA2EC0DF0A8CF32F13207FF0E326330
:1089200001D0322B32C1A8FF190EA0EC0DF04FEC94
:1089300026F0050EBA6F1200190EA2EC0DF0A8CFAA
:1089400032F1322B650E326302D0040E326F180EF4
:10895000A2EC0DF0A8503225336F650E336301D0C1
:10896000320732C1A8FF190EA0EC0DF04FEC26F033
:10897000040EBA6F1200180EA2EC0DF0A8CF32F15F
:108980003207030E326301D0322B32C1A8FF180E1A
:10899000A0EC0DF04FEC26F0030EBA6F1200180E8B
:1089A000A2EC0DF0A8CF32F1322B650E326302D06B
:1089B000050E326F190EA2EC0DF0A8503225336F60
:1089C000650E336301D0320732C1A8FF180EA0EC48
:1089D0000DF04FEC26F0020EBA6F1200190EA2EC49
:1089E0000DF0A8CF11F5180EA2EC0DF0A8CFD0F124
:1089F00011C50AF1D880640E0A55A856A8CF10F503
:108A00002887288B94D0268B52EC28F029912A892C
:108A1000CCEC27F02981010EBA6F64EC28F012002B
:108A200029B10AD0268B52EC28F0CCEC27F0010EAD
:108A3000BA6F64EC28F012002B8D268B52EC28F0D4
:108A40001DEC28F0010EBA6F64EC28F012002AB970
:108A500034D029A132D02C95E4EC1EF0230EBA2597
:108A6000A96ECFEC0DF0A8CF18F5A8CF59F12B9D2A
:108A7000210EA2EC0DF0A8CFD1F1D105040DF350D9
:108A8000070FA96ECFEC0DF0A8CF11F5D105040D9D
:108A9000F350060FA96ECFEC0DF0A8CFD0F111C5A1
:108AA0000AF1D880640E0A55D880A856A8CF10F5D0
:108AB000EFEC1EF02889288B3AD02C85326B32C11E
:108AC00018F5269BBAC1D1F1BA05040DF350070F72
:108AD000A96ECFEC0DF0A8CF11F5BA05040DF35037
:108AE000060FA96ECFEC0DF0A8CFD0F111C50AF199
:108AF000D880640E0A55A856A8CF10F52889288B6F
:108B000016D020AF12002DB945D02CB93ED026A9E1
:108B100008D02BB531D023C5CEF1CE6702D0D2EC30
:108B200026F0B92B0A0E7CEC10F0B96512002BA5CB
:108B30000DD02B952FEC0FF08EEC1EF07EEC24F078
:108B400025B18FEC1BF025A158EC1BF02B95209F35
:108B5000209DF8EC1EF052EC28F034EC1BF0A6EC53
:108B600024F0B96B26992D99269B269D26952B9D41
:108B70002C9924972499120042EC2BF023C5CEF1B6
:108B8000CE67CFD743EC2BF0CCD788EC26F064EC43
:108B900028F0C7D76EEC2AF0C4D729EE4AF0100EA1
:108BA000396FDE660DD0392FFCD72FEC0FF0010E98
:108BB0005BEC0BF0020E5BEC0BF070EC80F0010153
:108BC0007FEC0EF0F0EC0DF0A56BA66B939C939EE2
:108BD000819C819E20B509D820B14FD820A9F9EFFA
:108BE00048F0000003000000F5D7B8EC46F02CB1C7
:108BF0008AEF46F001EC3BF0F3EC3AF0A62B0E0EB8
:108C0000A66526D072D8DDEC47F01AEC80F00101A1
:108C1000A1C1A3F1A2C1A4F18DC1A1F18EC1A2F1A4
:108C2000A66B070E90EC10F032C152F133C153F134
:108C3000A1C154F1A2C155F1D7EC0BF01FB701D07F
:108C400007D0070E90EC10F032C1A1F133C1A2F1B0
:108C50008DC100F58EC101F50B0E7CEC10F00A6F92
:108C60000AC112F50C0E7CEC10F00A6F0AC113F564
:108C700040EC80F00101209512003EEC3BF027A172
:108C800005D00CEC4BF00000030000000EEC4BF0A4
:108C9000A52B050EA56512D028D8060E90EC10F075
:108CA00032C152F133C153F18DC154F18EC155F12E
:108CB000D7EC0BF020891FB72099A56B209124B722
:108CC0000AD024B908D0F292F0902A932A912499DC
:108CD0002497D59E1200F292F0902A932A9124991B
:108CE0002497D59E20992787120004EC19F00300E1
:108CF000000003000000030007EC19F0F7EC18F087
:108D000003000000030000000300FEEC18F0DFEC9D
:108D100017F01200F26AF16AF06AC290F0EC0DF0FE
:108D2000100E926E806A936A816A1D0E946E826A3A
:108D3000956A836A966A846AD56ACD6ACA6A9B6AAA
:108D4000020ED36ED180EAC137F10F0E396F0300E6
:108D50000000392FFCD7FAEC4AF00400050EACEC09
:108D60000CF0FCEC4AF003000000372FF4D7EBD7EF
:108D7000C2800000C282C2B2FED7C4CF4DF1C3CFC1
:108D80004CF1C60E4E6F030E4F6FEEEC0BF0640EFF
:108D90004E6F4F6B32EC0CF048C1C2F149C1C3F1C8
:108DA000C290C2C154F1C3C155F1280E526F0A0ED0
:108DB000536FD7EC0BF02C911FB703D0020EEA6F64
:108DC0002C818DC154F18EC155F1990E526F3A0E1E
:108DD000536FD7EC0BF02C911FA703D0030EEA6F53
:108DE0002C81299B299D280EA2EC0DF0A8CF54F1CF
:108DF000290EA2EC0DF0A8CF55F1D00E526F070E40
:108E0000536FD7EC0BF01FA7298B940E526F110EE6
:108E1000536FD7EC0BF01FA7298D29AB73D029AD69
:108E200071D0680EA86E280EA0EC0DF0100EA86E82
:108E3000290EA0EC0DF007C1A8FF2A0EA0EC0DF042
:108E400006C1A8FF2B0EA0EC0DF008C1A8FF2C0E48
:108E5000A0EC0DF097C1A8FF2D0EA0EC0DF098C16D
:108E6000A8FF2E0EA0EC0DF0A86A2F0EA0EC0DF0BE
:108E7000A86A300EA0EC0DF0A86A310EA0EC0DF03F
:108E8000A86A320EA0EC0DF0A86A330EA0EC0DF02B
:108E9000A86A340EA0EC0DF0A86A350EA0EC0DF017
:108EA00097C1A8FF360EA0EC0DF098C1A8FF370EB1
:108EB000A0EC0DF007C1A8FF380EA0EC0DF006C124
:108EC000A8FF390EA0EC0DF008C1A8FF3A0EA0ECE7
:108ED0000DF097C1A8FF3B0EA0EC0DF098C1A8FFC4
:108EE0003C0EA0EC0DF007C1A8FF3D0EA0EC0DF06C
:108EF00006C1A8FF3E0EA0EC0DF008C1A8FF3F0E72
:108F0000A0EC0DF0280EA2EC0DF0A8CF54F1290E24
:108F1000A2EC0DF0A8CF55F1C2C152F1C3C153F17B
:108F2000D7EC0BF01FA71200C2C1A8FF280EA0ECBF
:108F30000DF0C3C1A8FF290EA0EC0DF007C1A8FFDA
:108F40002A0EA0EC0DF006C1A8FF2B0EA0EC0DF030
:108F500008C1A8FF2C0EA0EC0DF097C1A8FF2D0EA4
:108F6000A0EC0DF098C1A8FF2E0EA0EC0DF01200A1
:108F7000800ECF6ECE6A3C0E036111D03C0E0461B0
:108F80000ED0180E05610BD0200E066108D00C0E15
:108F9000076105D0640E086102D09D801200000EAA
:108FA000036F000E046F0C0E056F010E066F030EAB
:108FB000076F0A0E086F9D801200360EA2EC0DF0AE
:108FC000A8CF54F1370EA2EC0DF0A8CF55F197C100
:108FD00052F198C153F1D7EC0BF01FA719D097C1EC
:108FE000A8FF360EA0EC0DF098C1A8FF370EA0EC3C
:108FF0000DF007C1A8FF380EA0EC0DF006C1A8FFC8
:10900000390EA0EC0DF008C1A8FF3A0EA0EC0DF04F
:109010003B0EA2EC0DF0A8CF54F13C0EA2EC0DF0EB
:10902000A8CF55F197C152F198C153F1D7EC0BF08D
:109030001FB7120097C1A8FF3B0EA0EC0DF098C11E
:10904000A8FF3C0EA0EC0DF007C1A8FF3D0EA0EC60
:109050000DF006C1A8FF3E0EA0EC0DF008C1A8FF60
:109060003F0EA0EC0DF01200249B9D9A08EC4BF0F3
:109070009E9A620EAD6EF8EC0DF0FEEC0DF0AECFE8
:1090800005F1180E0561056BFEEC0DF0AECF04F195
:109090003C0E0461046BFEEC0DF0AECF03F13C0E10
:1090A0000361036BFEEC0DF0AECF07F10C0E07650C
:1090B00001D0076FFEEC0DF0AECF06F107C132F123
:1090C000324F1F0E324F1C0E324F1F0E324F1E0EEC
:1090D000324F1F0E324F1E0E324F1F0E324F1F0ED9
:1090E000324F1E0E324F1F0E324F1E0E324F1F0ECA
:1090F000066502D0010E066FFEEC0DF0AECF08F152
:10910000640E0861086B0AEC4BF09E9A20859D8ADC
:1091100083EF3AF028919D9A9D8A83EF3AF00101FE
:10912000AAEC49F020B36DEC1AF0FC6A01EE09F0EC
:10913000EE6A0A0EEA62FCD7F0EC0DF0B8EC47F0EC
:109140000DEC19F0239D23ADFED78F6B906B196B3F
:109150001A6B208975EC46F020998DC19FF18EC164
:10916000A0F18DC1A1F18EC1A2F18DC1A3F18EC17B
:10917000A4F1CC2B0A6B0AC111F54F0E0A6F0AC17C
:1091800010F58DC100F58EC101F520EC80F00101D4
:1091900030EC80F0010118EC80F0010115EC3BF09F
:1091A000010140EC80F00101010EA96E010EAA6ED2
:1091B000CFEC0DF0A8CF39F1A92ACFEC0DF0A8CF54
:1091C0003AF1AA6A010E396304D0360E3A6301D02F
:1091D00010D0010EA96E010EAA6E010EA86ED3EC7E
:1091E0000DF0A92A360EA86ED3EC0DF0AA6A2AEF6C
:1091F00016F000EC4BF00EEC4BF01F6B206B216B6C
:10920000226B236B246B256B266B276B286B296BDA
:109210002A6B2B6B2C6B2D6B6DEC0FF0000EE8CFD7
:109220007CF0000EE8CF7DF0000EE8CF7EF0000E5F
:10923000E8CF7FF0FF0E2E6F2EC17AF0FF0E2E6F5B
:109240002EC17BF046EC2CF0A3C19FF1A4C1A0F18C
:10925000AA6A5C0EA2EC0DF0290EA86201D006D01D
:109260000ED8290EA86E5C0EA0EC0DF0270EA2EC15
:109270000DF02A85010EA8622A950EEF3AF018EC3F
:109280002AF0140E53D0289F29912A9BAA6A220EF5
:10929000A2EC0DF0010EA86206D0288F000E0A6F16
:1092A0000AC11FF51200020EA86206D02981000E25
:1092B0000A6F0AC11FF51200030EA86206D02A8B9E
:1092C000000E0A6F0AC11FF51200040EA86205D035
:1092D000010E0A6F0AC11FF51200050EA8621200E6
:1092E0002981010E0A6F0AC11FF512002FEC0FF041
:1092F000D6EC29F00A0E396FC80ED8EC0CF0249782
:10930000249920B10BEC42F020B139072091396744
:1093100001D0120020B3120024B7120024B91200A9
:10932000F0D72FEC0FF0F7EC29F0E4D7396FC80E27
:10933000D8EC0CF02497249920B10BEC42F020B12A
:1093400039072091396701D0120024B7120024B9DF
:109350001200F2D76C0ED36E110E926E806A030E5D
:10936000936E816ADD0E946E826A000E966E846A38
:10937000000E956E836A400E9B6E1F0ED56E070E13
:10938000CD6ED00EF26E050EF16E080EF06E210E4F
:109390009D6E000EA06ED06A000EC26E0E0EC16EE3
:1093A0008A0EC06EC66A000EC76E280EC66E000E0C
:1093B000C56E080EC86EBD6ABA6A070EB46E200E7E
:1093C0006F6E240EAC6E900EAB6E080EB86EB06A67
:1093D000220EAF6EAE6A9E6A1200010EEB6F0F0E88
:1093E000EC6F010EBA6FB86B208F21872FEC0FF056
:1093F00042EC1EF024972499219121931DEC1CF03E
:109400001BEC1DF03CEC13F020A109D00CEC3CF05F
:109410000BEC42F03EEC3BF0B8EC46F0209121B171
:109420001CEF4AF020AF0FEF13F020B961EF13F0FB
:1094300020B3F9EF48F0E6D7BA4F1CD0BA4F0AD0A4
:10944000BA4F10D0BA4F79D0BA4F58D0040EBA6F75
:1094500063EF13F0020EEB27C70EEB61EB6F020E0A
:10946000BA6FC8D7030EEC27630EEC61EC6F030EE6
:10947000BA6FC0D7258D2C87ECC14CF14D6B640EB3
:109480004E6F4F6BEEEC0BF0E80E4827030E4923AE
:1094900048C1C6F149C1C7F1C6C18DF1C7C18EF13E
:1094A00021912193209F249724995DEC4AF02083F9
:1094B000500E3DEC1AF018EF3CF02D81530E3DECB0
:1094C0001AF062EC80F00101540E3DEC1AF012002B
:1094D0002D91530E3DEC1AF064EC80F00101540E16
:1094E0003DEC1AF0470E3DEC1AF030EC80F0010133
:1094F00000EC40F0480E3DEC1AF012002FEC0FF09B
:109500005EEC44F02497249920A109D00CEC3CF0A7
:109510000BEC42F03EEC3BF0B8EC46F0209124B767
:1095200009D024B907D020B961EF13F020B3F9EFC7
:1095300048F0EAD7050EBA6F56D756EC42F0258DA3
:109540002C87ECC14CF14D6B640E4E6F4F6BEEEC03
:109550000BF0E80E4827030E492348C1C6F149C164
:10956000C7F1C6C18DF1C7C18EF15DEC4AF0010EA5
:10957000E8CF7FF00C0E5BEC0BF0000EE8CF7FF035
:109580001E0EED6F1DEC1CF002EC4BF02BEC3DF0D1
:10959000E7EC3DF000EC80F00101430E3DEC1AF0E9
:1095A000ED2FF2D7EB2FECD723C5CEF1CE6716D037
:1095B000FEEC4AF068EC4AF0259D2C97FA0ED8ECA8
:1095C0000CF0FA0ED8EC0CF0FA0ED8EC0CF000EC23
:1095D0004BF0010EEB6F050EBA6F05D72BEC3DF08B
:1095E000E7EC3DF000EC80F0010123C5CEF1CE6741
:1095F000F5D7DED781881200819812008188120089
:1096000081981200817812008188120081981200DE
:1096100081861200819612008186120081961200C6
:1096200081761200FFFFFFFFFFFFFFFFFFFFFFFF3D
:10963000FFFFFFFFFFFFFFFFFFFFFFFFFFFFFFFF3A
:10964000FFFFFFFFFFFFFFFFFFFFFFFFFFFFFFFF2A
:10965000FFFFFFFFFFFFFFFFFFFFFFFFFFFFFFFF1A
:10966000FFFFFFFFFFFFFFFFFFFFFFFFFFFFFFFF0A
:109A0000AF9BAFAFAFAFD1AFB205B007B008AF09F2
:109A1000AF09AF09AF09B108B2079B049F9F9F9F91
:109A2000AE9FFFFFFFFFFFFFFFFFFFFFFFFFFFFFF7
:109A3000FFFFFFFFFF8F82FFAC04A1149B1A96204B
:109A400092248F288A0E8C10940B8A0C9609870F0B
:109A5000960885129707830785079706850783076A
:109A600096068708820796058A07810696058C0761
:109A7000810594058E088005940490078005930461
:109A80009107800591049208800590049407800551
:109A90008E05950780058C05960880058A06960830
:109AA000820588069707820685079708840683073C
:109AB00097088507800898078707970F8908950DED
:109AC0008B0A8C108E0E912894269922A01CAA1520
:109AD0009707FFFFD7FFB701B403B404B403B4047E
:109AE000B304B304B305B205B206B205B2068136BB
:109AF0008137813781378137FF37FFFFFFFFACFFA9
:109B0000FFFF90FF8903A8008705A5038607A3052B
:109B10008508A007840A9F08840B9F06830D9F0673
:109B2000820E9F06810882049E05830882049E049B
:109B3000840881049D05850881049C0587078104AC
:109B40009C04880781049B04890781049A048A077E
:109B5000810499048B07810498048C07810496057D
:109B60008D07810495058E07810494058F07810474
:109B70009206900782049006910782048E0792074E
:109B800083048B07930883048609940A8404951937
:109B900085049617860498148704991289049B0EED
:109BA0008C049D08B305BA05FFFF8EFFB7008A023B
:109BB000A8018804A5038607A3058608A5058407D0
:109BC000A7058406A8058206AA058205AA058105BF
:109BD00091059504800591059504800591059504EE
:109BE00080059204950480059204950480059204F2
:109BF00095048005920494058005900594068005DF
:109C00009005940680058F05920882058E059208BE
:109C100082058C06900A82068A078E0C84068707C6
:109C200081068C06850781158907870883138918A3
:109C300085118B16870F8D148A0C91128E07AC0E2E
:109C4000FF0AFFB88BFFB205B006AF08AD09AC0B39
:109C5000AA0CA90E8107A7058208A6058407A405FA
:109C60008607A3058707A10589079F058A089E0522
:109C70008C079C058D089B058F0799059008980512
:109C80009207960594079505950793059707920502
:109C9000813581378137813781378137A437B305E3
:109CA000B305B305B305B305B3058F05FFFF8CFFFF
:109CB000A20192009203901085058F1C84078E1DCF
:109CC00083088E1D8308911C8207931B82068E05D4
:109CD000950581068E05970481058E0597048105FB
:109CE0008D05980580058D05990480058D059904DD
:109CF00080058D05990480058D05990480058D05E5
:109D0000990480058D05990480058D0599048005C9
:109D10008D05990480058D05970581058D059705AD
:109D200081058E05950581068E05930682068E05B2
:109D3000910782078F058D0883089005870A830B9A
:109D40009105841C9205851A930586189405A5151E
:109D5000AA11C50CFFFF11F11BA2219A269429908C
:109D60002B8E0D8C05850E850B880588098B088840
:109D70000689088E0786058B07910784058B069355
:109D80000683058C06950582058D05960681048D52
:109D900006970580058D05980580058D059804803A
:109DA000048E0B99048E0B99058E0B98058E0B98DB
:109DB000058E05980480068E05960481058F05960C
:109DC0000581068E05940582078F07900583098E0D
:109DD000088C07840B8D0A8607851B8E05871990D2
:109DE00003891792008B13960FA707ADFFC8FFFFDB
:109DF000059605B305B305B305B305B301AF0581FA
:109E000004AC058107A905810AA605810CA405817A
:109E10000FA10581129E0581139B0583139805866A
:109E2000129605891293058C1290058F118E05925A
:109E3000118B0595108905981086059B0F84059E4A
:109E4000108115A012A310A60DA80BAB09AD06AF8B
:109E500004B2A7FFFFFF03CA0BB10FAB0790118F2E
:109E60000C8D148A0F8A1688118818861486078428
:109E7000088715850683078B068408860681068D6C
:109E8000068307890480069005820C8B0591058165
:109E90000A8D05920481088F05940480069005952B
:109EA000048006900B9505910B9505910B950592F5
:109EB0000B94069105940480079105930580088F03
:109EC000049305810A8E059106810C8C068F06820B
:109ED00006890681058E088308850781068C15840E
:109EE0000883078813860A850A82118716870F89D7
:109EF00014890C8B128C068F10900CAA06AFFFC52C
:109F0000E9FFAC09980F8D0095138A029217880417
:109F1000901986068E1B850788098F0A83068D088F
:109F20009007820590078F078205930690058005AC
:109F300094068F06800596058F05800597058F048A
:109F4000800598048F04800598048E05980B8E0573
:109F5000980B8F04800598048E04810597058E0464
:109F6000810596058D05810695068E048305940569
:109F70008D05830693068D04850690078B0586075D
:109F80008D098A058808880B8706890C8C2D8F2BF4
:109F9000932796249D1FA917D30700FFFFFFFFFFFC
:109FA000000022003500D2000001A8014302AC02EB
:109FB0005403ED035404FF049A0500EE00F00D0E67
:109FC000EE6AEA62FDD71200FFFFFFFFFFFFFFFF0F
:109FD000FFFFFFFFFFFFFFFFFFFFFFFFFFFFFFFF91
:109FE000FFFFFFFFFFFFFFFFFFFFFFFFFFFFFFFF81
:109FF000FFFFFFFFFFFFFFFFFFFFFFFFFFFFFFFF71
:10A0000000000F0016006B008300DC002D016601CC
:10A01000C10116024C02AB0202031B032A034403D4
:10A020006F0375039F9F03BA049A059A0499039BD3
:10A030009F9F9FC0BF9F9F7FBF9F03CD0E96128E95
:10A04000168A0487078B0385038C04800383048BA3
:10A0500004820282048B03840281038B02870281C3
:10A06000038A028802810488038902800387028BA5
:10A0700003810385028C03820482038C03830480A2
:10A08000038C0685048C168713890E8E0395FFCDED
:10A090000084019E029C029B029C039B029B1D9BD1
:10A0A0001D811D81FFFFFCC0850194008403910286
:10A0B0008305900382069003820790028103810248
:10A0C0008F02820481028E02830481028D02840445
:10A0D00081028D02850381028C02860381028A033C
:10A0E000870382028802880482028603890483022D
:10A0F0008A0D84028C0A85028D0887029003E00293
:10A100009AFF8501920283049303820495028203DD
:10A110009602810289028A02810289028A028102F0
:10A1200089028A02810289028A02810288028A03E4
:10A130008202870289048202850387068303810ADB
:10A1400084038404810A870C84068A0A8802FF0734
:10A15000D3849A0299049705960781039402820496
:10A160009302840391028504900287038E0288047F
:10A170008D028A038B028B048A02811C811D811D42
:10A18000941D9C029C029C02C80200FA068D028863
:10A190000F8304870F82038809820281038A028168
:10A1A0000287028C02810287028C02810187028D64
:10A1B00002810187028E02800187038D028002875F
:10A1C000028C02810287028C02810387038A02814A
:10A1D0000388048802810588058402820E8902832F
:10A1E0000C8A0894ECE591088B1188158517840575
:10A1F0008602840585038902830386038A0281031C
:10A2000086038C02810287028C02810287028D0202
:10A21000800287028C02810287028C0281028702FF
:10A220008B038102880289038302870284058305E8
:10A230008703850E8A00950CE60680FF9C029C022F
:10A240009C029702810294028105910281088F028B
:10A2500082098C0285098902880987028B08840299
:10A260008D0982029008930B950998069A04FC01C7
:10A2700005F4038A088807870A8509850483058110
:10A280000B8303810485028206850388028105878A
:10A29000028902810388028A02810388028A02817C
:10A2A0000289028A02810388028A02810488028963
:10A2B00003810686028803820383038102860B835F
:10A2C0000581048208840B84058709860597E7E5E4
:10A2D00098048B098600890C8402880E8203880307
:10A2E000880382028A02870381028C02870281022C
:10A2F0008C02870280038C02870281028C02870213
:10A3000081028C02870281028A0387028203890309
:10A3100086028303870485028504810781038708F9
:10A320008A168F12E90C9F9F03AB038A048B048962
:10A33000048B0589048A0489028C038B9F9F9FC02C
:10A34000C89F9401940A940A96089F05B99FA9FF93
:10A350009B009403940A95099806FF0302830A94CC
:10A360000A9407940497BAFF15C815891589028BBA
:10A37000019B019C019D029D049C159A148A138BDC
:10A38000028A029B019C019D029D159C1589148ADD
:10A39000118DFFA0FFFFFFFF00FF00000E001B005C
:10A3A00048007D00B400E700F0000D012A014B01D8
:10A3B0006401700185018E01A301D601E20115023D
:10A3C000460267029C02CB02EA02210352036003A9
:10A3D00071039C03CD03F8031B045C047D04B804E3
:10A3E000E5040E05410564059705AC05CD05EA05B4
:10A3F0000F0624063D0656067F06A406D50600076E
:10A40000390752076B0784079D07C607DF0718083F
:10A4100037084C086B087C089508A108D408F9088F
:10A42000200945097A099B09E409F909140A330A44
:10A43000540A710A8A0A9F0AC80AED0A120B270BEE
:10A440005A0B770B8C0BA50BBE0BE30B040C390CD2
:10A450005C0C630C860C9F0CAD0CD60C050D2A0D04
:10A46000610D6C0DAB0DB80D050E3C0E5D0E700E42
:10A47000730EBA0ECB0EE40E150F3C0F610F6B0F6F
:10A48000860F8A0FDB0FE20F03F8018A0C85028228
:10A490000A85028394FF00CD0591039101C70591C0
:10A4A00003919DDA83018F0183018F018301880667
:10A4B000870D81078F0183018F0183018F01820145
:10A4C0008607890D83058F0183018F018301A20017
:10A4D00002B40186048A0186018802810185008810
:10A4E000018300860287028201851285018502842C
:10A4F000018400870185018301880284018201892A
:10A50000058403929A9F9203880585018301850142
:10A51000860283018400890282058B0382039202F2
:10A5200082028C02830289048402820186018503EF
:10A53000830186008701820191019D0403A4069195
:10A5400004880281028208860185008602840185D2
:10A5500000860384018401860582018306860282C7
:10A560000180038803850294069201900082FF9D7A
:10A570000194069002918BFF07E70C8C03890387F7
:10A580000286028B0184028E018201910181029177
:10A5900000800093B0B093008100910181018F028F
:10A5A00082028D0284028B028602870389038D0B4F
:10A5B000E707009F019601950282009002810491B5
:10A5C000078D078F04940092028101900183018F0F
:10A5D0000095A0A6950195019501950191018B0A21
:10A5E000900B9501950195019501A40188FF8201C9
:10A5F0008F0190069404FC0001B801950195019526
:10A60000019501950195019501950195FFBC018783
:10A610000295029494FF01C1039304900490049066
:10A6200003900391039103910193A0C490028B0ABC
:10A6300085028903860187058601830186018600DC
:10A6400084018601840085028601820186028601DA
:10A6500080028701880184048B03900AA30201CA47
:10A66000019501941095108694FF00B3018B01872A
:10A670000389018604890186028801800086018899
:10A68000018200860187018301860185018402869B
:10A69000018301850687018604880187BFB488018C
:10A6A0008B0087018C01860185008501860185006C
:10A6B0008501860185008501860183018502860169
:10A6C000810280018301880182049205B70300A4FE
:10A6D0000294049202910180028F0182028E018312
:10A6E000028C0185108B1086029001940096B7A110
:10A6F0008501880083088702820285018701840022
:10A700008700860184008700860184008700860117
:10A710008400860186018400850187018500870801
:10A720008600B60608B50C8C028901820283018777
:10A7300001830186018601830186008600840187EA
:10A7400000860184018601860283018401870884D2
:10A75000058FB1B7960096008D0086018A008604A9
:10A760008700880585008B0482008D059006930381
:10A77000C30104BB04890682028702800180018331
:10A780000187028301850086018501850086018598
:10A790000185018602830185028601810180018392
:10A7A0000588068102890484B3B68605880084077B
:10A7B0008701840284018601860184008601870066
:10A7C000830186018700840086018501830187015A
:10A7D0008402820188028B0DB80901FE0186028C79
:10A7E0000285028B028594FF01FF018601820286A9
:10A7F0000685028704850094A0FC950193029303CB
:10A80000810091018101900183018F0184018D01FB
:10A8100085018D0186018B0187018B0188018901EA
:10A8200089019E01009E00840090008400900084B5
:10A8300000900084009000840090008400900084C8
:10A8400000900084009000840090008400900084B8
:10A85000009000849AA189018A0188018A018701F8
:10A860008C0186018C0185018E0184018E0183019A
:10A870009001810192018100920194039402A4014C
:10A8800001B101950194019501940188028201842E
:10A890000486028101850284018402860282068F79
:10A8A00004919DBF8D0781048A04870288028B0171
:10A8B0008701840183038700840082058601830069
:10A8C0008201820186018300840082008601820168
:10A8D0008400820086018102830082018701820A4E
:10A8E0008A00A10802A70491048F068F048D0182BB
:10A8F000038B0185048C0183048F018005910494EE
:10A9000004950294999C8610861085008501860125
:10A910008500860086018500860086018500860008
:10A9200086018500850186018301850286018301F8
:10A9300084028702800581028902820393059F02B7
:10A94000069E0A8E038A0385018902890187028B8C
:10A950000086018D0086018D0086018D0186018CA7
:10A960000186018B028802880089008A999E8610E0
:10A9700086108D0086018D0086018D0086018D0078
:10A9800086018C0186018C0186018A02880186037A
:10A990008B028E0AA20510B1108600860185018502
:10A9A0000086018501850086018501850086018577
:10A9B0000185008601850185008601850185008667
:10A9C000018501850086018DB1B486108610850051
:10A9D0008E0185008F0085008F0085008F00850027
:10A9E0008F0085008F0085008F00C400069E0B8DB0
:10A9F000028A02870288018A0187018C0086018D04
:10AA00000086018D0086008701840186008601840E
:10AA10000186008600840288068400890585B19E2F
:10AA200086108D10950195019501950195018E0176
:10AA30008610B41000B1008E0086018D0086018D55
:10AA40000086018D108610860086018D0086018D9E
:10AA50000086018DBFCC9601950186018D0086018F
:10AA60008D0086018C008701870F890D9600960066
:10AA7000AC0010991086028D02930493029102801B
:10AA8000028F0282018D0385018A02880188038A70
:10AA90000086018D0096B19C861095109501950158
:10AAA00095019501950195019501B40110991086C4
:10AAB00003870395039503950293029203920391F2
:10AAC00010921086999C8610861095039502950326
:10AAD0009503950395039502870386109C10089DA6
:10AAE0000C8C028903870187018B0187018C00860A
:10AAF000018D0086018D0186018C0186018B028803
:10AB000002880C89088CB1A08610861086008E0001
:10AB100086008E0086008E0086008E0084018E01E5
:10AB200084018E0182028F029206A702089D0C8C7E
:10AB3000028902880187028B0186018C0086028EC1
:10AB40000084048E0182018C01810182018C0181CB
:10AB50000283028801820C8401830886B1A08610DA
:10AB6000861086008E0086008E0086008E0086008D
:10AB70008D0184018B04840180018903830788038C
:10AB800086058A028A009C0003B302860588018636
:10AB90000187028201860186018301860086018584
:10ABA0000185008601850185008601850185018674
:10ABB0000185028302860284028101880585019352
:10ABC00099A0960096009600960096008610861032
:10ABD0009600960096009600AC000C990E8A02959D
:10ABE00001950196019501950195019402940E87B6
:10ABF0000C8899A0950194049405940594059205F8
:10AC00008F048F048F048F049204AB0105990A927C
:10AC100009920490058E048E05900694069406927F
:10AC20000989068AA9A686008B0186028803880303
:10AC300084038B0381038F0391058F0581038C03AC
:10AC400085028803870387038B0196029C00009985
:10AC500002960395039503950A94098D048B04903D
:10AC6000039002920094A9AC86008C0086028A00B0
:10AC700086048900800286018700810386018500A1
:10AC80008303860184008502860182008603860193
:10AC90008000880386018A0386018B0295019C014E
:10ACA00015DF0181019101810191018101910181F2
:10ACB0000191018101910181019100820091B0B265
:10ACC00095019503950395039503940495049503C5
:10ACD0009503B30100B000910182019101810191BE
:10ACE0000181019101810191018101910181019114
:10ACF0001581CEE19401920292029402960295028D
:10AD00009503D60100AB009600960096009600963B
:10AD1000009600960096009600960096E09A95019F
:10AD2000950395029502FF00A68993018C04830187
:10AD300080018B02830082018A01830184008A00E2
:10AD4000830184008A00830184008A0083018300D8
:10AD50008C00820182008C018C0BB40A12AF11842A
:10AD6000018C0186008C0188018A0188018A018892
:10AD7000018A0188018B0286038B0283088D04906F
:10AD8000B8A08F068D0884028C0286018A02880191
:10AD90008A0188018A0188018A0188018B01860164
:10ADA0008C0185028D01A60004A10890028D028409
:10ADB000018C0286018A0188018A0188018A018842
:10ADC000008B0088018C018611861284A2B4920245
:10ADD0008E0780048C03810182018B018201830133
:10ADE0008A01820183018A01820183018A01820131
:10ADF00083018B01810183018B0182058D01830415
:10AE0000B50001B601950195109003850181018F70
:10AE10000183008F0184018E0184018E00840190E2
:10AE20000295AAAB8902810480018704810B860107
:10AE300083018101830186008500820083008501F2
:10AE400085008200830085018500820083008501E2
:10AE500083018201830086018305830086008405C7
:10AE600081018601890087048B009A0112AF128448
:10AE7000018C019400950195019502950B950A8C22
:10AE8000CDB488018A0188018A0188018501820187
:10AE9000850C8201950C95019501CC0101C40196A8
:10AEA0000185018D0185018D0185018D0185018C53
:10AEB0000181108202810F810182AFDC84128F1226
:10AEC0009402940192038001900282018E02840117
:10AED0008C0286018A03890096019C0000B0018ED5
:10AEE0000184018E0184018E0184018E12841284FA
:10AEF00001950195019500969DB48A0C8B0C9500E7
:10AF0000950195018B0C8B0B9401950195018B0C90
:10AF10009C0B0CB50C8A018C019400950195019550
:10AF200002950B950A8CA1B491048E0782028C03C2
:10AF300086018B0188018A0188018A0188018A01C2
:10AF400088018B0186018C0183038D029008A00487
:10AF500011B5108501870186008C0088018B01885E
:10AF6000018A0188018A0188018B0286028B028492
:10AF7000088D0490A1A090048D0883028C038700A3
:10AF80008A0288018A0188018A0188018B01880070
:10AF90008C0086018C01860FAF110CCD0C8A018CC0
:10AFA0000194009501950195019501960095B8A72A
:10AFB00085008C0183048C0184048A018201830151
:10AFC0008A01820183018A01820183018A0183014E
:10AFD00082018B01830082018B0182018D05830038
:10AFE000B60301B5019501950E920F88018A01887B
:10AFF000018A0188018A0188018A01880194B5B516
:10B000008C0A950B950296019600950095008B0190
:10B010008A0CB40C009D0396049404950494049443
:10B020000393039103910490039000939DA89305CB
:10B03000930893058F038F04920495039405930559
:10B040008C038B09A20601B50188028A0286028C54
:10B050000382028E02800491049202910280028E89
:10B060000383028B0286008A0189ACB486018C02BC
:10B0700085018905880187048A0184048E0191076E
:10B080008F0490048F0490049303A70100A9018A00
:10B090000287018A0386018A0485018A028401806D
:10B0A000018A02820182018A02810183018A02806F
:10B0B0000184048A0185028A0187018A0188019539
:10B0C000A29C960095019301810586028107830861
:10B0D0008A06810291018101920181009201810021
:10B0E0009201C80090FF8115FF15C8909201810060
:10B0F0009201810092018100910182018506810106
:10B10000830381078A0881058F019501BA01009F99
:10B11000019501950194019501960295019501957E
:10B12000019501940195F8A6890185048103850C98
:10B130008302FF0AA19491028E0782038C03860189
:10B140008B0188018A0186008607860E84088701A4
:10B15000810088018A0187018B028601B60100A95E
:10B16000018C0186048902850E8702870682018090
:10B170000187018300860087018401860086018D96
:10B180000186008D0186008D01950195B49C860095
:10B190008E008F0882018F0184018F0084018E014F
:10B1A00084018E018401900082018F018E08860047
:10B1B000B90001B100870081038901840081038BFC
:10B1C00001820081028D018100810A8F0A8C038A2D
:10B1D00001800081038B0182008103890184008149
:10B1E0000189018600810089FFAC099008820981EC
:10B1F000088290FF02B800850486048002830784D9
:10B20000018101840184018201830184018201831F
:10B21000018301840182018401820184008301840D
:10B2200001830182018402840780018504830480F4
:10B23000018EC8BB94019502C50194019502DC0101
:10B2400002890791018E0285018B02820082008BA8
:10B2500005810082018900810183008100890181CB
:10B2600001840080008901810184008001890180BE
:10B2700000840081008A018101820081018A0081AD
:10B280000185018B0186028D02820490BC898F01A9
:10B2900081038A01810181048A0182008101800188
:10B2A0008A018200820080018A018200820080017E
:10B2B0008A018101810081018A0181088B01810756
:10B2C0009501B80101BA03940292018002900182B3
:10B2D000018F018401910394029201800290018206
:10B2E000018F0184D0B6950190018B0C8D0A8F08D7
:10B2F000910693049502BC00FFFF89CF91028E074F
:10B3000085018B0288018B00800081078900800104
:10B310008107890081008200840089008100820009
:10B32000840089008001800182038A0081008102FB
:10B3300081018A0088018B0186018D0182029002C1
:10B34000890400C900960096009600960096009623
:10B350000096CBDC930191058101900183018F015F
:10B3600083018F01830191009205D803009F00871C
:10B37000008D0187008C0187008C0187008C01877C
:10B380000B8701810B870181008C0187008C01876D
:10B39000008C0187008C0187008C0087CA9D860085
:10B3A0008D0084018C0284018C03840180008C0157
:10B3B000830180018C01820181018D0182048E0153
:10B3C0008302D30100D1018E0184018D0186018C9D
:10B3D00000820182018C00820182018C0181018244
:10B3E000058D0180018F0381FFD4019103930193A7
:10B3F00000959DF68511950B960195019501950196
:10B4000094008B02950B9502950195018500FFFF35
:10B4100080CE0195029403920491008604890386EC
:10B4200005870286068504860782048709800F86C1
:10B4300007870780068706800788058008870381BD
:10B4400007880180018106880580058907800488B6
:10B450000A8003860C8002850C8001860B800C8894
:10B46000088B8F8BFFFFFFFF90EC5BF0120000005A
:10B47000849083C083FF80948084120085C000F094
:10B48000016A00C086F084C087F0848086C083FF94
:10B490008094808487C083FF8094808412008EC053
:10B4A00083FF809480848094808412007AC083FF1C
:10B4B000809480847BC083FF80948084120000018C
:10B4C000350E836FD5DF00017D510001846F856BE0
:10B4D0000001D89084378537D1DF0001360E836FA5
:10B4E000C7DF00013F0E846F010E856FC7DF0001CB
:10B4F000370E836FBDDF00017C510001846F856BC7
:10B50000020E00017E5D07E13A0E00018427000E65
:10B510000001852310D000017E0507E1200E000107
:10B520008427000E0001852306D0180E0001842711
:10B53000000E0001852300018407000E855B0001D9
:10B54000EF0ED8808455000E855504E2EF0E000101
:10B55000846F856B7CC000F000C001F0006A005071
:10B560000001841301500001851388DF0001200EC3
:10B57000836F7EDF00017C510001846F856B7EDF6D
:10B580000001210E836F74DF00017D510001846F83
:10B59000856B0001D8908437853770DF1200200E4C
:10B5A0000001825D03E10001B60E826F000182514D
:10B5B0007E0803E2220E0001825F210E0001825DFF
:10B5C00004E300018251A30803E20001820E826FAE
:10B5D000210E0001825DF66EF76AD890F636F736D6
:10B5E0009A0EF626A30EF7220900F5CF88F00A007E
:10B5F000F5CF89F000018229DF0FF66EF76AD89047
:10B60000F636F7369A0EF626A30EF7220900F5CF86
:10B610008AF00A00F5CF8BF01200270E0001825D40
:10B6200003E100013B0E826F220E0001825D03E107
:10B6300000013C0E826F6D0E0001825D03E100018E
:10B640003D0E826F200E0001825D03E100013E0E7F
:10B65000826F2E0E0001825D04E3000182513E08DC
:10B6600003E200013E0E826F2E0E0001825DF66E37
:10B67000F76AD890F636F736000EF626A00EF722B7
:10B680000900F5CF88F00A00F5CF89F00001822982
:10B69000D20FF66EF76AD890F636F736000EF62619
:10B6A000A00EF7220900F5CF8AF00A00F5CF8BF043
:10B6B0001200200E0001825D03E100012F0E826F57
:10B6C0002E0E0001825D04E300018251390803E27D
:10B6D00000012F0E826F2E0E0001825DF66EF76A5A
:10B6E000D890F636F736A00EF6269F0EF722090000
:10B6F000F5CF88F00A00F5CF89F000018229D20F3A
:10B70000F66EF76AD890F636F736A00EF6269F0E3C
:10B71000F7220900F5CF8AF00A00F5CF8BF012006E
:10B7200000017C51006E016A013404E20050E60819
:10B73000000E015403E20001E60E7C6F00017D5112
:10B74000006E016A013404E200509B08000E0154AF
:10B7500003E200019B0E7D6FB2DE0001220E836FBB
:10B7600087DE84800001816B00018151EA6A600FED
:10B77000E96E000EEA22EFCF82F00001825106E16D
:10B7800000013A0E826F0001190E816FF86A000104
:10B79000825101E1DCD01A0E0001815D01E3D7D0B6
:10B7A000020E00017E5D02E184DF06D000017E050D
:10B7B00002E133DF01D0F3DE00018E6B88C08CF034
:10B7C00089C08DF000018A5100018C5D00018B5110
:10B7D00000018D5901E3AFD0020E00017E5D1DE135
:10B7E0008CC0F6FF8DC0F7FF010E0F0B05E0D8905F
:10B7F000F732F632E806FBE1010ED890F636F7365E
:10B80000E806FBE1000EF6269A0EF7220900F5CFB6
:10B8100084F00A00F5CF85F03CD000017E051DE1E3
:10B820008CC0F6FF8DC0F7FF010E0F0B05E0D8901E
:10B83000F732F632E806FBE1010ED890F636F7361D
:10B84000E806FBE1240EF626A00EF7220900F5CF4C
:10B8500084F00A00F5CF85F01CD08CC0F6FF8DC0B7
:10B86000F7FF010E0F0B05E0D890F732F632E8062D
:10B87000FBE1010ED890F636F736E806FBE1880EBC
:10B88000F626A40EF7220900F5CF84F00A00F5CFC2
:10B8900085F000018C51010B05E00001845100018D
:10B8A000806F05D085C000F0016A00C080F0000103
:10B8B0008051006E016A0050800B1DE07F0E000178
:10B8C000805F00017F5109E000018051000804E21F
:10B8D00000018007EBDDF8D70DD08EC083FF00019B
:10B8E0008051000807E200018007809480848094E2
:10B8F0008084F5D71BD00001802B00017F510EE022
:10B900008EC083FF00018051000807E2000180071C
:10B910008094808480948084F5D708D00001805181
:10B92000000804E200018007C1DDF8D700018C2B7C
:10B93000000E8D2347D70001812B00018151EA6A57
:10B94000600FE96E000EEA22EFCF82F020D70001EF
:10B95000836B8EDD1200FFFFFFFFFFFFFFFFFFFF86
:10B96000FFFFFFFFFFFFFFFFFFFFFFFFFFFFFFFFE7
:10B97000FFFFFFFFFFFFFFFFFFFFFFFFFFFFFFFFD7
:10B98000FFFFFFFFFFFFFFFFFFFFFFFFFFFFFFFFC7
:10B99000FFFFFFFFFFFFFFFFFFFFFFFFFFFFFFFFB7
:10C000000901306B316B326B336B3451040B04E03C
:10C01000080E346F356B03D0040E346F356B366BFE
:10C02000376B386934C4B5F935C4B6F936C4B7F9D5
:10C0300037C4B8F938C4B9F939C4BAF93AC4BBF944
:10C040003BC4BCF91FC583F91EC584F90CC485F92E
:10C050000DC486F90EC487F90FC488F997C289F90F
:10C0600098C28AF999C28BF99AC28CF99BC28DF950
:10C070009CC28EF99DC28FF99EC290F9EFC591F9CD
:10C08000F0C592F9F1C593F9F2C594F9F3C595F9A4
:10C09000F4C596F9F5C597F9F6C598F9F7C599F974
:10C0A000F8C59AF9F9C59BF9FAC59CF95FC99DF9DC
:10C0B00060C99EF961C99FF962C9A0F963C9A1F974
:10C0C00064C9A2F965C9A3F966C9A4F96FC9A5F93C
:10C0D00070C9A6F971C9A7F972C9A8F977C9A9F9F0
:10C0E00078C9AAF979C9ABF97AC9ACF97BC9ADF9B4
:10C0F0007CC9AEF97DC9AFF97EC9B0F97FC9B1F984
:10C1000080C9B2F981C9B3F982C9B4F905011F51D7
:10C1100002E0090130812C6A2D6A2E6A2F6AEFC570
:10C1200027F0F0C528F0F1C529F0F2C52AF0C2ECDD
:10C130006EF0010A02E009013083100E0901BE6FA2
:10C14000BF6B200EBFAF02D0D89003D0BE5D000EF3
:10C15000BF592DE2BEC9E9FFBFC9EAFFD890E93651
:10C16000EA36D890E936EA36800EE926040EEA224D
:10C17000EECF00F0EECF01F0EECF02F0EFCF03F004
:10C180002C6A2D6A2E6A2F6A00C027F001C028F0A1
:10C1900002C029F003C02AF0C2EC6EF0010A02E0EE
:10C1A000090130850901BE2B000EBF23CAD72C6AB6
:10C1B0002D6A2E6A2F6AF3C527F0F4C528F0F5C55D
:10C1C00029F0F6C52AF0C2EC6EF0010A02E009017E
:10C1D0003087A40E2C6E700E2D6E7D0E2E6E3F0ECF
:10C1E0002F6E77C927F078C928F079C929F07AC964
:10C1F0002AF0D2EC6EF0010A02E109013089660EE4
:10C200002C6E2D6EA60E2E6E3F0E2F6E77C927F068
:10C2100078C928F079C929F07AC92AF0C9EC6EF0FA
:10C22000010A02E10901308B5C0E2C6E8F0E2D6E1F
:10C23000420E2E6E3E0E2F6E97C227F098C228F047
:10C2400099C229F09AC22AF0D2EC6EF0010A02E1FA
:10C250000901308DAE0E2C6E470E2D6E810E2E6EA6
:10C260003F0E2F6E97C227F098C228F099C229F08E
:10C270009AC22AF0C9EC6EF0010A02E10901308F7E
:10C280009A0E2C6E990E2D6E190E2E6E3F0E2F6E7D
:10C290009BC227F09CC228F09DC229F09EC22AF0C2
:10C2A000D2EC6EF0010A02E109013181AE0E2C6E72
:10C2B000470E2D6E810E2E6E3F0E2F6E9BC227F005
:10C2C0009CC228F09DC229F09EC22AF0C9EC6EF0F3
:10C2D000010A02E10901318338C42CF039C42DF080
:10C2E0003AC42EF03BC42FF034C427F035C428F0F4
:10C2F00036C429F037C42AF0F8EC6CF027C000F0FF
:10C3000028C001F029C002F02AC003F0330E2C6EC1
:10C310002D6E730E2E6E3F0E2F6E00C027F001C0E3
:10C3200028F002C029F003C02AF0C9EC6EF0010A1F
:10C3300002E10901318538C42CF039C42DF03AC42A
:10C340002EF03BC42FF034C427F035C428F036C497
:10C3500029F037C42AF0F8EC6CF027C000F028C0B0
:10C3600001F029C002F02AC003F0CD0E2C6ECC0ED5
:10C370002D6E4C0E2E6E3D0E2F6E00C027F001C0AC
:10C3800028F002C029F003C02AF0D2EC6EF0010AB6
:10C3900002E1090131872C6A2D6A800E2E6E3E0E55
:10C3A0002F6E7FC927F080C928F081C929F082C982
:10C3B0002AF0C9EC6EF0010A02E109013189050198
:10C3C0001E51080802E20901318B2C6A2D6A2E6A7F
:10C3D0002F6AA5C927F0A6C928F0A7C929F0A8C9BE
:10C3E0002AF0C2EC6EF0010A2FE063C92CF064C998
:10C3F0002DF065C92EF066C92FF05FC927F060C91E
:10C4000028F061C929F062C92AF0F8EC6CF027C065
:10C4100000F028C001F029C002F02AC003F0330E5A
:10C420002C6E2D6E730E2E6E3F0E2F6E00C027F0F9
:10C4300001C028F002C029F003C02AF0C9EC6EF058
:10C44000010A02E10901318D2C6A2D6A2E6A2F6AD8
:10C45000A5C927F0A6C928F0A7C929F0A8C92AF0BC
:10C46000C2EC6EF0010A30E063C92CF064C92DF013
:10C4700065C92EF066C92FF05FC927F060C928F0A2
:10C4800061C929F062C92AF0F8EC6CF027C000F00D
:10C4900028C001F029C002F02AC003F0CD0E2C6E96
:10C4A000CC0E2D6E4C0E2E6E3D0E2F6E00C027F062
:10C4B00001C028F002C029F003C02AF0D2EC6EF0CF
:10C4C000010A02E10901318F2C6A2D6A400E2E6E9D
:10C4D0002F6E08C427F009C428F00AC429F00BC441
:10C4E0002AF0C9EC6EF0010A02E10901328108C4A8
:10C4F0002CF009C42DF00AC42EF00BC42FF00CC48C
:10C5000027F00DC428F00EC429F00FC42AF0F7EC70
:10C510006CF027C000F028C001F029C002F02AC04A
:10C5200003F0CD0E2C6ECC0E2D6E4C0E2E6E3E0EEC
:10C530002F6E00C027F001C028F002C029F003C010
:10C540002AF0C9EC6EF0010A02E1090132832C6A7B
:10C550002D6A400E2E6E3F0E2F6E0CC427F00DC4B8
:10C5600028F00EC429F00FC42AF0D2EC6EF0010AB4
:10C5700002E1090132857B0E2C6E140E2D6E8E0E9B
:10C580002E6E3F0E2F6E0CC427F00DC428F00EC483
:10C5900029F00FC42AF0C9EC6EF0010A02E109018A
:10C5A0003287330E2C6E2D6E2E6E3F0E2F6E7BC992
:10C5B00027F07CC928F07DC929F07EC92AF0D2EC89
:10C5C0006EF0010A02E109013289AE0E2C6E470EAF
:10C5D0002D6E810E2E6E3F0E2F6E7BC927F07CC90B
:10C5E00028F07DC929F07EC92AF0C9EC6EF0010A55
:10C5F00002E10901328B9BC22CF09CC22DF09DC23E
:10C600002EF09EC22FF097C227F098C228F099C250
:10C6100029F09AC22AF0C9EC6EF0010A02E1090180
:10C62000328D12000901349536951200FF0E090172
:10C63000385D20E10501B80ED88000550B0E01557C
:10C6400019E222C538F938C900F0016A00BE016854
:10C65000FF0E001801E101500DE138C900F0016A38
:10C6600000BE0168FE0E001801E1015002E0000E5C
:10C6700001D0010E1200D9CFE6FFE1CFD9FF0901A9
:10C68000C06BC16B34C42CF035C42DF036C42EF011
:10C6900037C42FF0B5C927F0B6C928F0B7C929F0BB
:10C6A000B8C92AF0C2EC6EF0010A14E138C42CF0CB
:10C6B00039C42DF03AC42EF03BC42FF0B9C927F08D
:10C6C000BAC928F0BBC929F0BCC92AF0C2EC6EF087
:10C6D000010A02E00901C081EFC52CF0F0C52DF080
:10C6E000F1C52EF0F2C52FF091C927F092C928F0BC
:10C6F00093C929F094C92AF0C2EC6EF0010A02E055
:10C700000901C08377C92CF078C92DF079C92EF0C2
:10C710007AC92FF0A9C927F0AAC928F0ABC929F016
:10C72000ACC92AF0C2EC6EF0010A14E17BC92CF00E
:10C730007CC92DF07DC92EF07EC92FF0ADC927F040
:10C74000AEC928F0AFC929F0B0C92AF0C2EC6EF02A
:10C75000010A02E00901C08905011F510901835D39
:10C7600001E0C08B0CC42CF00DC42DF00EC42EF0D3
:10C770000FC42FF085C927F086C928F087C929F092
:10C7800088C92AF0C2EC6EF0010A02E00901C08DEE
:10C790003AD0100E0901BE6FBF6B200EBFAF02D0A2
:10C7A000D89003D0BE5D000EBF592DE2BEC9E9FF8F
:10C7B000BFC9EAFFD890E936EA36D890E936EA36BA
:10C7C000800EE926040EEA22EECF00F0EECF01F053
:10C7D000EECF02F0EFCF03F02C6A2D6A2E6A2F6A9B
:10C7E00000C027F001C028F002C029F003C02AF0E1
:10C7F000C2EC6EF0010A02E00901C08F0901BE2BF4
:10C80000000EBF23CAD7F7C52CF0F8C52DF0F9C527
:10C810002EF0FAC52FF099C927F09AC928F09BC9C4
:10C8200029F09CC92AF0C2EC6EF0010A02E009016D
:10C83000C1816FC92CF070C92DF071C92EF072C979
:10C840002FF0A5C927F0A6C928F0A7C929F0A8C9C3
:10C850002AF0C2EC6EF0010A28E15FC92CF060C931
:10C860002DF061C92EF062C92FF09DC927F09EC935
:10C8700028F09FC929F0A0C92AF0C2EC6EF0010A85
:10C8800014E163C92CF064C92DF065C92EF066C9A6
:10C890002FF0A1C927F0A2C928F0A3C929F0A4C983
:10C8A0002AF0C2EC6EF0010A02E00901C1837FC9DF
:10C8B0002CF080C92DF081C92EF082C92FF0B1C9AA
:10C8C00027F0B2C928F0B3C929F0B4C92AF0C2ECE4
:10C8D0006EF0010A02E00901C18505011E5109013E
:10C8E000845D01E0C18797C22CF098C22DF099C2F7
:10C8F0002EF09AC22FF089C927F08AC928F08BC977
:10C9000029F08CC92AF0C2EC6EF0010A14E19BC236
:10C910002CF09CC22DF09DC22EF09EC22FF08DC92E
:10C9200027F08EC928F08FC929F090C92AF0C2ECEF
:10C930006EF0010A02E00901C1892C6A2D6A500ECD
:10C940002E6E410E2F6E08C427F009C428F00AC4C9
:10C9500029F00BC42AF0C9EC6EF0010A02E10901CA
:10C96000C18D08C42CF009C42DF00AC42EF00BC4EC
:10C970002FF00CC427F00DC428F00EC429F00FC40A
:10C980002AF0F7EC6CF027C000F028C001F029C0B5
:10C9900002F02AC003F0CD0E2C6ECC0E2D6E4C0E84
:10C9A0002E6E3E0E2F6E00C027F001C028F002C090
:10C9B00029F003C02AF0C9EC6EF0010A02E1090176
:10C9C000C18FFE0EDB5006E00901C0513613C15184
:10C9D000371305D00901C0513413C1513513E55245
:10C9E000E7CFD9FF1200E66A46DEE5521200010EDB
:10C9F000E66E41DEE55212000201706B05011F0573
:10CA000001E0D7D30201925101E04CD1F00E2C6E1F
:10CA1000850E2D6E990E2E6E3E0E2F6EBBC227F028
:10CA2000BCC228F0BDC229F0BEC22AF08EEC6DF067
:10CA300027C014F428C015F429C016F42AC017F42E
:10CA4000A40E2C6E700E2D6E7D0E2E6E3F0E2F6E70
:10CA500014C427F015C428F016C429F017C42AF00E
:10CA6000F8EC6CF093EC6EF028C004F429C005F4E7
:10CA700004011F0ED8800455000E055503E21F0E59
:10CA8000046F056B000E045D000E055902E2046B95
:10CA9000056B04C4C6F2030E0201C603F3CFC5F250
:10CAA000C5C229F0D1EC6CF027C000F028C001F01D
:10CAB00029C002F02AC003F0960E2C6EB20E2D6E25
:10CAC000CC0E2E6E3D0E2F6E00C027F001C028F058
:10CAD00002C029F003C02AF0E1EC6DF027C014F485
:10CAE00028C015F429C016F42AC017F47FC92CF009
:10CAF00080C92DF081C92EF082C92FF014C427F00F
:10CB000015C428F016C429F017C42AF0F8EC6CF00C
:10CB100027C000F028C001F029C002F02AC003F0AD
:10CB20000CC42CF00DC42DF00EC42EF00FC42FF049
:10CB300000C027F001C028F002C029F003C02AF08D
:10CB4000F8EC6CF027C0E8F228C0E9F229C0EAF25C
:10CB50002AC0EBF20201C65105E1A76BA86BA96BD5
:10CB6000AA6B26D0C6C229F0D1EC6CF027C000F029
:10CB700028C001F029C002F02AC003F000C02CF048
:10CB800001C02DF002C02EF003C02FF09FC227F08D
:10CB9000A0C228F0A1C229F0A2C22AF08EEC6DF04A
:10CBA00027C0A7F228C0A8F229C0A9F22AC0AAF279
:10CBB0002C6A2D6A2E6A2F6AA7C227F0A8C228F015
:10CBC000A9C229F0AAC22AF0D2EC6EF0010A05E14E
:10CBD0000201A76BA86BA96BAA6B9FC22CF0A0C225
:10CBE0002DF0A1C22EF0A2C22FF0A7C227F0A8C23A
:10CBF00028F0A9C229F0AAC22AF0C9EC6EF0010AF5
:10CC000008E19FC2A7F2A0C2A8F2A1C2A9F2A2C2E3
:10CC1000AAF22C6A400E2D6E1C0E2E6E460E2F6E42
:10CC2000A7C227F0A8C228F0A9C229F0AAC22AF0F8
:10CC3000E1EC6DF093EC6EF028C042F229C043F2B3
:10CC40002C6A2D6A7A0E2E6E440E2F6EE8C227F0E3
:10CC5000E9C228F0EAC229F0EBC22AF0E1EC6DF05B
:10CC600093EC6EF028C048F229C049F22C6A2D6A74
:10CC70007A0E2E6E440E2F6EAFC227F0B0C228F08F
:10CC8000B1C229F0B2C22AF0E1EC6DF093EC6EF083
:10CC900028C04AF229C04BF2C6C24EF20201010E70
:10CCA000926FC76BC75153E1C6C2C7F2C7C229F022
:10CCB000D1EC6CF027C004F028C005F029C006F0C4
:10CCC0002AC007F0A7C22CF0A8C22DF0A9C22EF0EE
:10CCD000AAC22FF004C027F005C028F006C029F032
:10CCE00007C02AF0E1EC6DF027C000F028C001F089
:10CCF00029C002F02AC003F000C02CF001C02DF0C2
:10CD000002C02EF003C02FF09BC227F09CC228F077
:10CD10009DC229F09EC22AF0F7EC6CF027C0A3F266
:10CD200028C0A4F229C0A5F22AC0A6F20201C75168
:10CD3000EA6A700FE96E020EEA22EF500401046FF6
:10CD4000056B04C408F30301210E096F04D0010E22
:10CD50000401046F056B0401010E041901E1055182
:10CD600001E091D10201C7050401046F056B010EBA
:10CD7000041901E1055101E07FD0C3C228F0C4C20B
:10CD800029F004C42DF005C42EF04EEC6EF026C040
:10CD900004F027C005F004C028F005C029F0E2EC3B
:10CDA0006CF027C000F028C001F029C002F02AC0B2
:10CDB00003F0960E2C6EB20E2D6ECC0E2E6E3D0E26
:10CDC0002F6E00C027F001C028F002C029F003C078
:10CDD0002AF0E1EC6DF027C014F428C015F429C046
:10CDE00016F42AC017F42C6A2D6A400E2E6E2F6E90
:10CDF000A7C227F0A8C228F0A9C229F0AAC22AF027
:10CE00008EEC6DF027C000F028C001F029C002F0C0
:10CE10002AC003F0C3C208F0C4C209F0060ED880CD
:10CE20000856000E095608C028F009C029F0E2ECA7
:10CE30006CF027C004F028C005F029C006F02AC015
:10CE400007F004C02CF005C02DF006C02EF007C07E
:10CE50002FF000C027F001C028F002C029F003C065
:10CE60002AF0E1EC6DF027C0ABF228C0ACF229C08B
:10CE7000ADF22AC0AEF25FD0045105111FE1146B70
:10CE8000156B166B176BA3C22CF0A4C22DF0A5C2B4
:10CE90002EF0A6C22FF09BC227F09CC228F09DC2A4
:10CEA00029F09EC22AF0F7EC6CF027C0ABF228C044
:10CEB000ACF229C0ADF22AC0AEF23DD0030E286E0E
:10CEC000296A04C42DF005C42EF04EEC6EF026C085
:10CED00004F027C005F004C028F005C029F0E2ECFA
:10CEE0006CF027C000F028C001F029C002F02AC071
:10CEF00003F0960E2C6EB20E2D6ECC0E2E6E3D0EE5
:10CF00002F6E00C027F001C028F002C029F003C036
:10CF10002AF0E1EC6DF027C014F428C015F429C004
:10CF200016F42AC017F4A7C2ABF2A8C2ACF2A9C289
:10CF3000ADF2AAC2AEF20CC42CF00DC42DF00EC49A
:10CF40002EF00FC42FF014C427F015C428F016C417
:10CF500029F017C42AF0F8EC6CF027C014F428C0AC
:10CF600015F429C016F42AC017F4ABC22CF0ACC2D9
:10CF70002DF0ADC22EF0AEC22FF0A3C227F0A4C296
:10CF800028F0A5C229F0A6C22AF0F8EC6CF027C060
:10CF900004F028C005F029C006F02AC007F0B3C28B
:10CFA0002CF0B4C22DF0B5C22EF0B6C22FF004C0E2
:10CFB00027F005C028F006C029F007C02AF0E1ECF0
:10CFC0006DF027C000F028C001F029C002F02AC08F
:10CFD00003F0AFC22CF0B0C22DF0B1C22EF0B2C23D
:10CFE0002FF000C027F001C028F002C029F003C0D4
:10CFF0002AF0F8EC6CF027C010F428C011F429C016
:10D0000012F42AC013F414C42CF015C42DF016C465
:10D010002EF017C42FF010C427F011C428F012C44A
:10D0200029F013C42AF0C9EC6EF0010A04E10401EE
:10D03000046B056B27D004C4C7F2ABC22CF0ACC2A2
:10D040002DF0ADC22EF0AEC22FF0A3C227F0A4C2C5
:10D0500028F0A5C229F0A6C22AF0F8EC6CF027C08F
:10D06000A3F228C0A4F229C0A5F22AC0A6F20201A8
:10D07000C751EA6A700FE96E020EEA22EF5004010E
:10D08000046F056B68D60201C751000801E386D022
:10D09000F00E006E850E016E990E026E3E0E036E4E
:10D0A000C7C229F0D1EC6CF027C004F028C005F00D
:10D0B00029C006F02AC007F004C02CF005C02DF0EE
:10D0C00006C02EF007C02FF000C027F001C028F0E6
:10D0D00002C029F003C02AF0E1EC6DF027C014F47F
:10D0E00028C015F429C016F42AC017F47FC92CF003
:10D0F00080C92DF081C92EF082C92FF014C427F009
:10D1000015C428F016C429F017C42AF0F8EC6CF006
:10D1100027C000F028C001F029C002F02AC003F0A7
:10D120000CC42CF00DC42DF00EC42EF00FC42FF043
:10D1300000C027F001C028F002C029F003C02AF087
:10D14000F8EC6CF027C020F428C021F429C022F4A8
:10D150002AC023F40201C70505E1C3C2BFF2C4C25D
:10D16000C0F205D0030EC703F350BF6FC06B210E92
:10D170000301095D12E1C7C209F30201C751EA6A5E
:10D18000700FE96E020EEA22EFCF0AF303010C29B9
:10D190000C6F640E0C5D01E10C6B0AD00CC420F422
:10D1A0000DC421F40EC422F40FC423F4BF6BC06B72
:10D1B000E8D00CC42CF00DC42DF00EC42EF00FC41A
:10D1C0002FF074C427F075C428F076C429F077C412
:10D1D0002AF0F7EC6CF027C010F428C011F429C035
:10D1E00012F42AC013F42C6A2D6A2E6A2F6A10C416
:10D1F00027F011C428F012C429F013C42AF0D2EC8D
:10D200006EF0010A01E1B2D0F00E2C6E850E2D6E8B
:10D21000990E2E6E3E0E2F6E10C427F011C428F00A
:10D2200012C429F013C42AF08EEC6DF027C010F45C
:10D2300028C011F429C012F42AC013F4A40E2C6ED5
:10D24000700E2D6E7D0E2E6E3F0E2F6E10C427F0C9
:10D2500011C428F012C429F013C42AF0F8EC6CF0C1
:10D2600093EC6EF028C0BFF229C0C0F2030E286E06
:10D27000296ABFC22DF0C0C22EF04EEC6EF026C05F
:10D28000BFF227C0C0F20201BF51C01109E10CC4B6
:10D2900020F40DC421F40EC422F40FC423F465D08D
:10D2A000C351BF5DC451C05904E2C3C2BFF2C4C27E
:10D2B000C0F2BFC228F0C0C229F0E2EC6CF027C077
:10D2C00000F028C001F029C002F02AC003F0960E39
:10D2D0002C6EB20E2D6ECC0E2E6E3D0E2F6E00C03B
:10D2E00027F001C028F002C029F003C02AF0E1ECC9
:10D2F0006DF027C010F428C011F429C012F42AC020
:10D3000013F47FC92CF080C92DF081C92EF082C999
:10D310002FF010C427F011C428F012C429F013C450
:10D320002AF0F8EC6CF027C000F028C001F029C00A
:10D3300002F02AC003F00CC42CF00DC42DF00EC472
:10D340002EF00FC42FF000C027F001C028F002C05B
:10D3500029F003C02AF0F8EC6CF027C020F428C0B4
:10D3600021F429C022F42AC023F40BD00CC420F4E9
:10D370000DC421F40EC422F40FC423F40201BF6BC8
:10D38000C06B120005011F051DE1200E0401046F92
:10D39000056B006B0451005D000E055513E2005152
:10D3A000EA6AC80FE96E020EEA22EF50E66E0051FB
:10D3B000EA6A500FE96E020EEA22E552E750EF6E7C
:10D3C000002BE8D7120005011F050EE10401006BD8
:10D3D000200E005D09E20051EA6AC80FE96E020EF4
:10D3E000EA22EF6A002BF4D7120005011F0523E1A2
:10D3F0000201C751EA6AC80FE96E020EEA22EF5035
:10D40000006E016AD890015004E6FF0E005C000E29
:10D41000015811E2C751EA6AC80FE96E020EEA220A
:10D42000EF28E66EC751EA6AC80FE96E020EEA22DB
:10D43000E552E750EF6E120005011F0501E145D0EE
:10D440002C6A2D6A2E6A2F6A2CC427F02DC428F06E
:10D450002EC429F02FC42AF0D2EC6EF0010A1BE191
:10D460007BC92CF07CC92DF07DC92EF07EC92FF030
:10D470002CC427F02DC428F02EC429F02FC42AF084
:10D48000E1EC6DF027C02CF428C02DF429C02EF457
:10D490002AC02FF41AD077C92CF078C92DF079C999
:10D4A0002EF07AC92FF02CC427F02DC428F02EC4FA
:10D4B00029F02FC42AF0E1EC6DF027C02CF428C02D
:10D4C0002DF429C02EF42AC02FF412000001130EEF
:10D4D0008A6F1C0E8B6F976BF50E986F996B9A6B1A
:10D4E000300E9B6F390E9C6F86EF6AF000010C0EB8
:10D4F0008A6F100E8B6F976BE10E986F996B9A6B1A
:10D500002E0E9B6F3E0E9C6F86EF6AF00001906BB3
:10D5100090C0DEFF84820001706B0001875103E13F
:10D520000001010E876F0001865103E10001010E29
:10D53000866F00018B510001D880885502E28BC0B4
:10D5400088F00001875100018825410806E2410E5C
:10D550000001D88087550001886F86C092F00001D5
:10D56000916B00019151912BEA6A600FE96E000EF8
:10D57000EA22EFCF93F05BD80001906B0001010E1F
:10D58000946F0001935152E00001940501E1F1D83C
:10D59000FFD8010E000194190001946F0001940559
:10D5A00008E1CED8400E0001925D02E20001922B0C
:10D5B000A5D90001902B040E0001905D02E2000E3F
:10D5C00001D0010E036E3C0E0001935D02E0000EDF
:10D5D00001D0010E026E3A0E0001935D02E0000ED2
:10D5E00001D0010E016E2E0E0001935D02E0000ECF
:10D5F00001D0010E011002100314006E00018A51C7
:10D600000001905D02E2000E01D0010E00100DE05D
:10D6100000019151912BEA6A600FE96E000EEA2237
:10D62000EFCF93F004D80001906BABD7120000014C
:10D630009C51D880935502E3000E01D0010E006E7C
:10D640009B51935D02E3000E01D0010E001006E035
:10D650008C6B8D6B8E6B8F6B956B71D09B51935DCB
:10D660008C6F8D6B8E6B8F6B8B29FE0BE842006E7F
:10D67000016A026A036A8CC026F08DC027F08EC052
:10D6800028F08FC029F000C02BF001C02CF002C0A0
:10D690002DF003C02EF048EC70F022C08CF023C0B7
:10D6A0008DF024C08EF025C08FF08AC000F0016A92
:10D6B000026A036A8CC026F08DC027F08EC028F065
:10D6C0008FC029F000C02BF001C02CF002C02DF05B
:10D6D00003C02EF048EC70F022C08CF023C08DF017
:10D6E00024C08EF025C08FF0000197518C279851EF
:10D6F0008D2399518E239A518F233C0E935D02E026
:10D70000000E01D0010E016E3A0E935D02E0000E94
:10D7100001D0010E006E2E0E935D02E0000E01D0CE
:10D72000010E001001100BE08B51E824006E000187
:10D73000005000018C27000E8D238E238F231200B2
:10D740000001750E966FF0D800018705966FECD832
:10D7500000013F0E966FE8D80001150E966FE4D8D1
:10D7600000019205966FE0D800019205966F94EF44
:10D770006CF00001956B8851955D09E29551EA6A5C
:10D78000000FE96E080EEA22EF6A952BF4D712001B
:10D7900000018C518D118E118F1101E1AED000016D
:10D7A0008C510001956F95C0F6FF8DC000F08EC0C2
:10D7B00001F08FC002F00001036A00500001956F74
:10D7C00095C0F7FF8EC000F08FC001F00001026A23
:10D7D000036A00500001956F95C0F8FF0001956B3A
:10D7E000000188510001955D01E37AD00900F5CF71
:10D7F00096F0000189511CE000018939F00B006EA0
:10D80000F00E00019615005C07E200018939F00B6B
:10D810000001965D0001966F0F0E00019615000144
:10D82000895D06E2000189510001965D0001966F55
:10D83000000194051EE1F00E00019615E66E000150
:10D840009551EA6A000FE96E080EEA22E552E750A8
:10D85000EF6E00019639F00BF00BE66E0001952992
:10D86000EA6A000FE96E080EEA22E552E750EF6E11
:10D8700033D0000196390F0B0F0B006E000195514C
:10D88000EA6A000FE96E080EEA22EF50F00B001072
:10D89000E66E00019551EA6A000FE96E080EEA2271
:10D8A000E552E750EF6E0F0E00019615006E000175
:10D8B0009529EA6A000FE96E080EEA22EF50F00B94
:10D8C0000010E66E00019529EA6A000FE96E080E65
:10D8D000EA22E552E750EF6E020E0001952780D74D
:10D8E00000018B29FE0BE842006E00010050000190
:10D8F0008C27000E8D238E238F231200848200013B
:10D90000956B000188510001955D0DE20001955174
:10D91000EA6A000FE96E080EEA22EFCF96F007D808
:10D920000001952BEED71200849201D8120001015C
:10D9300084900001839096BF8382839096AF8392F8
:10D94000838096BD8382839096AD8392838096BBBD
:10D950008382839096AB8392838096B983828390EF
:10D9600096A98392838096B78382839096A78392A9
:10D97000838096B58382839096A58392838096B3A5
:10D980008382839096A38392838096B183828390CF
:10D9900096A1839283808480010100010001966B2F
:10D9A0001200219E05D0219E29AE02D0296C218E25
:10D9B00029C023F0226A336A326A860E246E256AF1
:10D9C0004CEF6FF0219E08D0219E29AE05D0286C27
:10D9D000291EE86A2922218E29C023F028C022F0BE
:10D9E000336A326A8E0E246E256A4CEF6FF02F7EFA
:10D9F000216A88EC6FF0A0EC6FF021B630EF6FF089
:10DA000021A20AD021AA03D021BE30EF6FF021A4B9
:10DA10003CEF6FF039EF6FF021AA05D021AC3CEF5D
:10DA20006FF039EF6FF021A00AD021A808D021BEF5
:10DA300004D021A402D045EF6FF049EF6FF0326AB5
:10DA4000256A2F502A5C316E10E327C033F028C0BE
:10DA500022F029C023F02AC030F02CC027F02DC0BE
:10DA600028F02EC029F0213A09D02CC033F02DC067
:10DA700022F02EC023F02FC030F0316C219E21BC4B
:10DA8000218E30C024F021B078EF6FF01A0E316093
:10DA900078EF6FF0246A2A6A21A408D0276C281E28
:10DAA000291E2A1EE86A282229222A2221AC08D00F
:10DAB000336C221E231E241EE86A222223222422E3
:10DAC000266A315207E02A34293228322732263298
:10DAD000312EF9D7275033262850222229502322CD
:10DAE0002A50242226C032F0219E24AE0BD0326C64
:10DAF000331E221E231E241EE86A332222222322E2
:10DB00002422218E24A006D0D88023322232333220
:10DB10003232302A30C024F04CEF6FF0216A88ECAA
:10DB20006FF0A0EC6FF021B630EF6FF021A205D0BE
:10DB300021BA30EF6FF037EF6FF021BA43EF6FF09B
:10DB400021A005D021B830EF6FF043EF6FF021B87E
:10DB500037EF6FF0256A7F0E2A24246EE86A2522AB
:10DB60002F50245EE86A255A1A0E306E2A6A326AED
:10DB7000336A226A236A2C50275E2D50285A2E5071
:10DB8000295A000E2A5A09E72C5027262D50282200
:10DB90002E502922000E2A2201D0328AD890273610
:10DBA000283629362A36D89032363336223623366E
:10DBB000302EE1D7295028102710D8A4328A4CEFF4
:10DBC0006FF0216A88EC6FF0A0EC6FF021B630EFB7
:10DBD0006FF021A205D021B830EF6FF037EF6FF072
:10DBE00021AA05D021B030EF6FF037EF6FF021B0F0
:10DBF00002D021A802D043EF6FF0256A2F502A24CB
:10DC0000246EE86A25227E0E245EE86A255A326A6E
:10DC1000336A226A236A2E502902F4CF23F0F3CF0D
:10DC200022F02D502902F3503326F4502222000E08
:10DC300023222E502802F3503326F4502222000EC5
:10DC400023222C502902F3503226F4503322000EA6
:10DC5000222223222D502802F3503226F450332260
:10DC6000000E222223222E502702F3503226F45097
:10DC70003322000E222223222C502802F450322676
:10DC8000000E3322222223222D502702F450322666
:10DC9000000E3322222223224CEF6FF028C032F0F4
:10DCA00028502D02F4CF27F0F3CF26F029502E0272
:10DCB000F4CF29F0F3CF28F02D02F3502726F450AB
:10DCC0002822E86A292232502E02F3502726F450E7
:10DCD0002822E86A2922000C216A88EC6FF021B61C
:10DCE00076EF6EF021A20AD021B403D07F0E296E08
:10DCF00019D0800E296E16D0296A14D021B0FCD715
:10DD0000870E2A60F1D77E0E2A64F6D7860E2A5C2B
:10DD100004E0D89029322A2AF9D721A403D0296C0B
:10DD200029AEEAD71200216A88EC6FF021B69DEF88
:10DD30006EF021A20ED021B405D07F0E296EFF0E09
:10DD4000286E1FD0800E296E286A1BD0296A286A87
:10DD500018D021B0FBD78F0E2A60EDD77E0E2A6433
:10DD6000F5D78E0E2A5C05E0D890293228322A2A6F
:10DD7000F8D721A406D0286C291EE86A292229AEEA
:10DD8000E5D71200DBEC6EF021B6000C21B0010CDF
:10DD9000000CDBEC6EF021B6000C21B0000C21B4BD
:10DDA000000C010CDBEC6EF021B6000C21B0000C75
:10DDB00021A4000C010C216A88EC6FF0A0EC6FF03C
:10DDC00021B6120021AE08D021A004D021A802D093
:10DDD00021801200219012002F502A5C0BE12E505E
:10DDE000295C08E12D50285C05E12C50275C02E1FC
:10DDF00021801200D8A002D0218E10D02A502FC02E
:10DE00002AF02F6E29502EC029F02E6E28502DC0DA
:10DE100028F02D6E27502CC027F02C6E2F502A5C36
:10DE200010E0FF0F09E0219021B403D021AE21843E
:10DE3000120021AE219412002F2AD8902E322D32BA
:10DE40002C322C50275E2D50285A2E50295A29BE8C
:10DE5000EAD7D8902736283629362A2EF8D7C8D7B9
:10DE60007F0E2A6EFF0E296E286E276E12007F0E1F
:10DE700021BEFF0E2A6E02D07F0E2A6E800E296E02
:10DE8000286A276AF3D721AE04D0800E2A6E296A49
:10DE9000F7D72A6A296AF4D7235022103310321098
:10DEA000F8E025BEF0D723BE0CD024502510EBE0BF
:10DEB000D89032363336223623362406D8A02506AB
:10DEC000F2D72550D4E12428D2E032AE11D07F0E13
:10DED000321402E133A00CD0332AE86A2222232232
:10DEE00007E3D880233222323332242A2428BFE0A9
:10DEF0002450C9E033C027F022C028F02334296E13
:10DF000024302A6E29322A9E21BE2A8E36EF6FF0E7
:10DF100029362A3602E32184217E06E121802A6AFD
:10DF2000296A286A276A12002A2803E0D880293241
:10DF30001200D890293202E12182120021861200BB
:10DF40002E362F3602E3218C217E06E121882F6AAE
:10DF50002E6A2D6A2C6A12002F2803E0D8802E32F8
:10DF60001200D8902E32EAE1218A1200D9CFE6FFC2
:10DF7000DACFE6FFE1CFD9FFE2CFDAFF0C0EE124E2
:10DF800002E3E168E652E16ED950FA0FE96EFF0E46
:10DF9000DA20EA6E010EEECFDBFF020EEECFDBFFE2
:10DFA000030EEECFDBFF040EEECFDBFF63D8D950BC
:10DFB000010FE96E000EDA20EA6EEECFE6FFEECF3B
:10DFC000E6FFEECFE6FFEFCFE6FF72EC80F0006EEB
:10DFD000060EE15C02E2E16AE552E16E0050DF6E9E
:10DFE000850EDF1404E04DD8EE6AED6A23D0090EE9
:10DFF000DBCF00F00A0EDBCF01F0820E0026FF0E11
:10E0000001223FD800C0EEFF01C0EDFF7E0EF36E8F
:10E01000090EF3CFDBFF0A0EDB6AD950010FE66E63
:10E02000000EDA20E66E26D82DEC76F0E552E552A9
:10E03000E552E552010EDBCF00F0020EDBCF01F01E
:10E04000030EDBCF02F0040EDBCF03F000C026F09E
:10E0500001C027F002C028F003C029F00C0EE15CDB
:10E0600002E2E16AE552E16EE552E5CFDAFFE7CF81
:10E07000D9FF1200D950050FE66E000EDA20E66EC9
:10E080001200F80EDBCFE9FFF90EDBCFEAFF12003A
:10E0900026502B02F3CF22F0F4CF23F02C02F350C2
:10E0A0002326000EF420246E26502D02F350242641
:10E0B000000EF420256E26502E02F3502526275000
:10E0C0002B02F3502326F4502422000E2522275041
:10E0D0002C02F3502426F450252227502D02F35011
:10E0E000252628502B02F3502426F45025222850B0
:10E0F0002C02F350252629502B02F350252612001E
:10E10000000000000000000000000000000000000F
:10E1100000000000000000000000000000000000FF
:10E1200000000000000009800000000000006FF007
:10E130000000000000003FE00000000000000000C0
:10E1400000000000000000000000000000000000CF
:10E1500000000000000000000000000000000000BF
:10E16000000000000000000000000000000000208F
:10E170000000000000003AF000000000004BFFA08B
:10E18000000000005CFF91000000006DFE710000C7
:10E1900000017EFD60000000018FFD5000000000C6
:10E1A0009FFB400000000000FA300000000000006B
:10E1B000200000000000000000000000000000003F
:10E1C0000000000000000000000169BCCA720000ED
:10E1D000009FFEDCDFFFB2001DF8200005FDFF30D0
:10E1E000AF3000009F902ED0F800002CF50006F014
:10E1F000F80004ED300005F0AF308FB100000CE006
:10E200001DFDF8000016DF40009FFFDCDEFFC300AD
:10E21000000169BCCA73000000000000000000009B
:10E2200000000000000000000000000000000000EE
:10E2300002900000000001300AB00000000004F06D
:10E240002F600000000004F0AF977777777779F0C0
:10E25000FFFFFFFFFFFFFFF012222222222226F003
:10E2600000000000000004F000000000000003D0E7
:10E27000000000000000000000000000000000009E
:10E28000000000000000000000000000000001404D
:10E2900007D0000000007FF04F800000001CFEF05F
:10E2A000CC00000002EF57F0F70000002EE207F06C
:10E2B000F8000001DE2007F0CE10002DE20007F08C
:10E2C0004FD658FE300007F006FFFFB1000007F000
:10E2D0000014520000000580000000000000000053
:10E2E000000000000000000000000000000002002C
:10E2F0000920000000007F506F40000000002ED079
:10E30000DB000059000007F0F800008E000004F068
:10E31000EA0000CF100006F09F3007FF90001EE0DB
:10E320001EFCDF87FB79EF50019DC6007EFFD50004
:10E3300000000000002100000000000000000000BC
:10E340000000000000000000000000002BB00000F2
:10E3500000000006FFE00000000002CF69E00000BE
:10E3600000007FB109E00000002CE60009E0000099
:10E3700007FB100009E00000CFFCCCCCCEFDDDD0C7
:10E38000DEEEEEEEEFFEEEE00000000009E0000041
:10E390000000000008C000000000000000000000B5
:10E3A000000000000000000000000000000012005B
:10E3B00078ABCDED0000CE20FFEDCCFA00005FB0D1
:10E3C000F90006F0000008F0F9000AB0000004F0BF
:10E3D000F9000AC0000004F0F90008F300000BF097
:10E3E000F90001FE6213BF90F900004EFFFFFB0031
:10E3F000110000016AA940000000000000000000B8
:10E40000000000000000000000000356653000001E
:10E41000004BFFFFFFFFA20008FE968F956AFF30BA
:10E420006F9001F800003ED0EC0008F0000006F00C
:10E43000F6000AE0000004F0F70007F3000009F01E
:10E44000CD1001EF7213AF904D20002DFFFFF900AA
:10E4500000000000478610000000000000000000DF
:10E46000000000000000000011000000000000009B
:10E47000FA00000000000000FA0000000000049014
:10E48000FA0000000039EFF0FA0000017DFFE940DA
:10E49000FA0005BFFF940000FA18EFFB50000000DF
:10E4A000FEFFD71000000000FFB4000000000000D5
:10E4B000520000000000000000000000000000000A
:10E4C0000000000000000000000000000278500082
:10E4D00003ADB4007FFFFC003FFCFF66FA43AFA032
:10E4E000CD101CFE70000BF0F50001FE000005F0E1
:10E4F000F50000BF100004F0EC0007FFB0000AF0C8
:10E500006FD9CF78FB329F9007EFE6009FFFFB00AB
:10E51000000100000388500000000000000000001F
:10E520000000000000000000000355200000000073
:10E5300004DFFFFB10000B604FD7459FD0001CE0AD
:10E54000DD000005F50005F0F7000000F80004F01C
:10E55000F8000000F70008F0BE200006F2005FA0FF
:10E560002EF9547F947CFC0002AFFFFFFFFE700089
:10E570000001467775300000000000000000000038
:10E58000000000000000000000000000000000008B
:10E59000000000000000000000000000000000007B
:10E5A000000006A10000098000001FF900006FF0C4
:10E5B00000000DF500003FE000000010000000002A
:10E5C000000000000000000000000000000000004B
:10E5D000000000000000000000000000000000003B
:10E5E000000000000000000000000000000000002B
:10E5F0000000300000000000BAAEF0000000000093
:10E60000FFE930000000000053000000000000009F
:10E610000000100000000000978CF00000000000D7
:10E62000FFFB50000000000075100000000000001B
:10E6300000000000000000000000000000000000DA
:10E6400000000000000000000000000000000000CA
:10E6500000000000000000000000000000000000BA
:10E660000000000000000000756AE00000000000EB
:10E67000FFFD700000000000A83000000000000056
:10E68000000000000000000000000000000000008A
:10E69000000000000000000000000000000000007A
:10E6A000000000000000000000000000000000006A
:10E6B00000100000000000002CFFA000000000007F
:10E6C000DD78FA0000000000F2005F0000000000AA
:10E6D000F0004F1000000000EA23DC000000000002
:10E6E0004FFFE200000000000154000000000000A5
:10E6F000000000000000000000000000000000001A
:10E7000000001111111111100000FFFFFFFFFFF0B9
:10E7100000009FA7777777700000D6000000000008
:10E720000002F300000000000001FFCBBBBBBBB048
:10E7300000004FFEEEEEEEE00000AB200000000017
:10E740000001F100000000000002FA555555555037
:10E750000000AFFFFFFFFFF00000024444444440CC
:10E76000D9CFE6FFDACFE6FFE1CFD9FFE2CFDAFF7C
:10E77000260EE12402E3E168E652E16ED950050F6E
:10E78000E1D972EC80F0006E060EE15C02E2E16A13
:10E79000E552E16E0050DF6E800EDF5C05E00B0E8F
:10E7A000DB5012E0DF0410E0210E04017C6F7D6B72
:10E7B000010EDB68020EDB68030EDB687F0EF36E72
:10E7C000040EF3CFDBFF8FD1040EDF5C0EE13EDAE7
:10E7D000010EEECFDBFF020EEECFDBFF030EEECF1E
:10E7E000DBFF040EEECFDBFF7ED1DF0410E1210E54
:10E7F00004017C6F7D6B010EDB6A020EDB6A800E0A
:10E80000F36E030EF3CFDBFF040EDB686CD1D9503F
:10E810000C0F98D9B6EC6FF0006E060EE15C02E2C8
:10E82000E16AE552E16E0050FA0E26C0DBFFFB0EF6
:10E8300027C0DBFFFC0E28C0DBFFFD0E29C0DBFF7D
:10E84000A6D9F30E2C6E040E2D6E350E2E6E3F0ED5
:10E8500087D9C9EC6EF0010A09E1B3D984D9F7EC84
:10E860006CF067D9EDD984D9ACD916D00C0EDB0683
:10E870000D0E01E2DB068BD92C6A2D6A2E6A3F0E43
:10E880006FD976D9160EDBCF04F0170EDBCF05F06B
:10E89000180EDBCF06F0190E66D9E1EC6DF049D900
:10E8A000CFD9F8EC6CF01A0E27C0DBFF1B0E28C086
:10E8B000DBFF1C0E29C0DBFF1D0E2AC0DBFF160E7E
:10E8C000DBCF27F0170EDBCF28F0180EDBCF29F0B7
:10E8D000190EDBCF2AF01A0EDBCF2CF01B0EDBCF8C
:10E8E0002DF01C0EDBCF2EF01D0EDBCF2FF08EECAB
:10E8F0006DF01FD9120E27C0DBFF130E28C0DBFFFF
:10E90000140E29C0DBFF150E2AC0DBFF4DD9120EF5
:10E91000DBCF2CF0130EDBCF2DF0140EDBCF2EF05F
:10E92000150E62D90E0E27C0DBFF0F0E28C0DBFFCD
:10E93000100E29C0DBFF110E2AC0DBFF3D0EF36E67
:10E940001E0EF3CFDBFF7E0EF36E1F0EF3CFDBFF49
:10E950000D0EF36E200EF3CFDBFFBF0EF36E210E14
:10E96000F3CFDBFF0E0EDBCF00F00F0EDBCF01F09D
:10E97000100EDBCF02F0110EDBCF03F03A0E2C6E3F
:10E980003F0E2D6ED40E2E6EC00EEAD8F8EC6CF051
:10E99000220E27C0DBFF230E28C0DBFF240E29C078
:10E9A000DBFF250E2AC0DBFF0E0EDBCF27F00F0E9C
:10E9B000DBCF28F0100EDBCF29F0110EDBCF2AF0D1
:10E9C0001E0EDBCF2CF01F0EDBCF2DF0200EDBCF89
:10E9D0002EF0210E09D9220EDBCF2CF0230EDBCF37
:10E9E0002DF0240EDBCF2EF0250EDBCF2FF08EEC9A
:10E9F0006DF007D9120EDBCF00F0130EDBCF01F064
:10EA0000140EDBCF02F0150EDBCF03F0CDD8010ED4
:10EA1000DBCF2CF0020EDBCF2DF0030EDBCF2EF080
:10EA2000040EE2D827C004F028C005F029C006F083
:10EA30002AC007F078D8046A800E056E310E066E83
:10EA40003F0E076EC9D827C008F028C009F029C0BA
:10EA50000AF02AC00BF0CCD8E1D8E1EC6DF069D80F
:10EA6000830E146E800E156E5E0E166EB90E176E46
:10EA7000B3D827C018F028C019F029C01AF02AC04E
:10EA80001BF0B6D814C027F015C028F016C029F026
:10EA900017C02AF0E1EC6DF027C010F028C011F08B
:10EAA00029C012F02AC013F0010EDBCF1CF0020EB9
:10EAB000DBCF1DF0030EDBCF1EF0040EDBCF1FF00B
:10EAC0001CC02CF01DC02DF01EC02EF01FC02FF05A
:10EAD000F8EC6CF027C00CF028C00DF029C00EF047
:10EAE0002AC00FF020D8010EDBCF00F0020EDBCFE2
:10EAF00001F0030EDBCF02F0040EDBCF03F000C009
:10EB000026F001C027F002C028F003C029F0260E2D
:10EB1000E15C02E2E16AE552E16EE552E5CFDAFF3F
:10EB2000E7CFD9FF120064D882D8F8EC6CF001EF7F
:10EB300076F027C000F028C001F029C002F02AC0FA
:10EB400003F01200E66E000EDA20E66E7FD8EECFFC
:10EB5000E6FFEECFE6FFEECFE6FFEFCFE6FF1200D7
:10EB60002F6E17EF76F0DBCF07F06AD80EEF76F056
:10EB7000F7EC6CF0160E27C0DBFF170E28C0DBFF8A
:10EB8000180E29C0DBFF190E2AC0DBFF1200FA0E97
:10EB9000DBCF00F0FB0EDBCF01F0FC0EDBCF02F091
:10EBA000FD0EDBCF03F01200120EDBCF27F0130EA9
:10EBB000DBCF28F0140EDBCF29F0150EDBCF2AF0C7
:10EBC0001200FA0EDBCF04F0FB0EDBCF05F0FC0EDB
:10EBD000DBCF06F0FD0E12000C0EDBCF28F00D0E81
:10EBE000DBCF29F0E4EF6CF0DBCF2FF0E1EF6DF03D
:10EBF00027C02CF028C02DF029C02EF02AC02FF0FD
:10EC00001200010E27C0DBFF020E28C0DBFF030E3F
:10EC100029C0DBFF040E2AC0DBFF120004C027F06E
:10EC200005C028F006C029F007C02AF0120000C075
:10EC300027F001C028F002C029F003C02AF012001A
:10EC40002C6A2D6A2E6A3F0E2F6E1200D950FA0FD1
:10EC5000E96EFF0EDA20EA6E1200D9CFE6FFDACFB6
:10EC6000E6FFE1CFD9FFE2CFDAFF5BD8013411E252
:10EC70000050FE08000E01540CE276D805E06CD876
:10EC8000800EEE6EEE6847D067D8800EEE6E7F0E77
:10EC90000ED047D8D890015004E6010E005C000E5B
:10ECA00001580BE261D805E057D8EE6A800EEE6E8F
:10ECB00032D052D8EE6AEE6A2ED047D8EECF00F0AE
:10ECC000EECF01F0EECF02F0EFCF03F032D800C06C
:10ECD000EEFF01C0EEFF02C0EEFF03C0EEFF21D841
:10ECE0000050010B05E025D8020E3AD8EF8E04D073
:10ECF00020D8020E35D8EF9E14D8D89001320032B9
:10ED000018D8030E2DD800C0EFFF1AD804E011D890
:10ED1000030E26D8EF8EE552E5CFDAFFE7CFD9FF15
:10ED2000120013D8040E1CD8EECF00F0EFCF01F084
:10ED30001200FA0EDBCFE9FFFB0EDBCFEAFF120079
:10ED400004D8060E0DD8EF501200FC0EDBCFE9FF01
:10ED5000FD0EDBCFEAFF1200ECDFEE6AEE6A120076
:10ED6000E926000EEA221200220E04017C6F7D6B60
:10ED7000A0EF76F0FFFFFFFFFFFFFFFFFFFFFFFFAA
:10ED8000FFFFFFFFFFFFFFFFFFFFFFFFFFFFFFFF93
:10ED9000FFFFFFFFFFFFFFFFFFFFFFFFFFFFFFFF83
:10EDA000FFFFFFFFFFFFFFFFFFFFFFFFFFFFFFFF73
:10EDB000FFFFFFFFFFFFFFFFFFFFFFFFFFFFFFFF63
:10F5100000037ACDEEDCA84000000000000018DFF8
:10F52000FFFFFFFFFFFE920000000007EFFFFFDC80
:10F53000BBCEFFFFFF91000000BFFFC76543223332
:10F5400057BFFFFD20000BFFC40000000000002497
:10F550006EFFD1007FFA000000000000000001BF34
:10F56000FA00EFC00000000000000000000DFF20C6
:10F57000FF6000000000000000000005FF60FF4089
:10F5800000000000000000000003FF70FF8000008A
:10F590000000000000000006FF50CFF30000000054
:10F5A00000000000001DFF104FFE300000000000B2
:10F5B000000001CFF80007FFD71000000000000195
:10F5C0007EFFB000005EFFFB9854333458BFFFFA53
:10F5D000000000019FFFFFFFFFFFFFFFFD50000045
:10F5E0000000017BFFFFFFFFFFE94000000000007B
:10F5F00000000246776541000000000000000000A6
:10F6000000000000000000000000000000000000FA
:10F6100000000000000000000000000000000000EA
:10F6200000000000000000010000000000000000D9
:10F6300000000000001FA00000000000000000010A
:10F640004400009F90000000000000000004FF0044
:10F6500002FF50000000000000000004FF000AFF4D
:10F6600010000000000000000004FF003FFC00004C
:10F670000000000000000004FF00BFFC77777777F0
:10F68000777777777779FF00FFFFFFFFFFFFFFFFB7
:10F69000FFFFFFFFFF00FFFFFFFFFFFFFFFFFFFF79
:10F6A000FFFFFF00333333333333333333333336F6
:10F6B000FF00000000000000000000000004FF0048
:10F6C000000000000000000000000004FF00000037
:10F6D00000000000000000000004FF000000000027
:10F6E0000000000000000003CC000000000000004B
:10F6F000000000000000000000000000000000000A
:10F7000000000000000000000000000000000000F9
:10F7100000000000000000000000000000000000E9
:10F7200000000000000000000000000000000000D9
:10F7300000083000000000000000002AFF0000BFA9
:10F74000D10000000000000008FFFF000AFFB30026
:10F75000000000000003DFFFFF004FFA0000000080
:10F760000000006FFFDBFF00CFE0000000000000A2
:10F7700008FFF808FF00FF800000000000009FFE67
:10F780004008FF00FF40000000000009FFD2000811
:10F79000FF00FF4000000000009FFD100008FF0078
:10F7A000FF800000000008FFD1000008FF00FFE01C
:10F7B000000000008FFE20000008FF009FFA0000FC
:10F7C000001AFFE200000008FF002EFFD62138EFEC
:10F7D000FD2000000008FF0004FFFFFFFFFFC10045
:10F7E00000000008FF00003DFFFFFFE700000000F1
:10F7F0000008FF00000059BB950000000000000B4E
:10F80000FF000000000000000000000000000000F9
:10F8100000000000000000000000000000000000E8
:10F8200000000000000000000000000000000000D8
:10F8300000000000000000000000002000000000A8
:10F8400000000000005E300004F80000000000002E
:10F85000000008FFD0001EFE200000000000000095
:10F8600004DFF8007FF50000000000000000002F1A
:10F87000FE00DFC000000007950000000009FF3017
:10F88000FF700000000CF70000000004FF60FF5054
:10F890000000000EF80000000003FF70FF60000091
:10F8A000002FFA0000000004FF60FFB00000007F9E
:10F8B000FE0000000009FF30BFF4000002EFFF70FF
:10F8C0000000002FFE004FFE60005EFDBFF500004F
:10F8D00003EFF70009FFFFDFFFF32FFFB656BFFF6F
:10F8E000C000008FFFFFFE4004FFFFFFFFFC100081
:10F8F00000028CDB7100002BFFFFFE800000000087
:10F90000000000000000156630000000000000004C
:10F9100000000000000000000000000000000000E7
:10F9200000000000000000000000000000000000D7
:10F930000000000000000000000000000004EFC014
:10F940000000000000000000000001AFFFC0000048
:10F9500000000000000000005EFFFFC0000000008B
:10F9600000000000001BFFD4CFC00000000000001A
:10F97000000006EFF800CFC0000000000000000209
:10F98000BFFC3000CFC0000000000000007FFF700F
:10F990000000CFC00000000000002CFFB2000000FB
:10F9A000CFC0000000000007FFE600000000CFC04D
:10F9B0000000000003CFFA1000000000CFC00000DC
:10F9C00000008FFFEAAAAAAAAAAAEFEAAAAAAA0096
:10F9D000FFFFFFFFFFFFFFFFFFFFFFFFFF00FFFF36
:10F9E000FFFFFFFFFFFFFFFFFFFFFF004444444412
:10F9F00044444444DFD44444440000000000000078
:10FA00000000CFC000000000000000000000000067
:10FA1000CFC000000000000000000000000079706E
:10FA200000000000000000000000000000000000D6
:10FA300000000000000000000000000000000000C6
:10FA40000000000000000000000000200000000096
:10FA5000001234567200000003F80000ABCDEFFF37
:10FA6000FFFFF80000001EFF8000FFFFFFFFFFFF09
:10FA7000F900000028FFF300FFDAA98767FFB00054
:10FA80000000007FFB00FF70000006FF1000000078
:10FA9000000CFF10FF7000000BFA000000000005D2
:10FAA000FF50FF7000000DF7000000000002FF7023
:10FAB000FF7000000EF7000000000002FF70FF70F2
:10FAC00000000EFA000000000004FF60FF7000005C
:10FAD0000BFE10000000000AFF30FF70000006FF60
:10FAE000B0000000006FFD00FF70000000DFFD406F
:10FAF000000029FFF500FF700000003FFFFEBABDC7
:10FB0000FFFF9000FF7000000003DFFFFFFFFFF822
:10FB1000000055200000000007DFFFFFEA30000072
:10FB2000000000000000000134420000000000005E
:10FB300000000000000000000000000000000000C5
:10FB400000000000000000000000000000000012A3
:10FB5000333321000000000000000049CEFFFFFF0A
:10FB6000FFEB7100000000007EFFFFFFFFFFFFFFC3
:10FB7000FF900000003DFFFFFCBAFFFBABEFFFFD75
:10FB8000200004FFFE83001CFD2000028EFFD10038
:10FB90001EFF900000BFE100000001CFF900AFF7A9
:10FBA000000005FF50000000001DFF10FFB0000026
:10FBB0000AFE000000000006FF50FF5000000DFB91
:10FBC000000000000002FF70FF2000000DFC00009C
:10FBD00000000003FF60FF3000000AFF200000006B
:10FBE0000008FF30FF70000005FFC1000000004F5B
:10FBF000FD00EFE1000000CFFD50000028FFF40001
:10FC00007FFD0000002DFFFFDBCDFFFF70000CD259
:10FC100000000001BFFFFFFFFFE500000110000032
:10FC20000000039DFFFEB600000000000000000081
:10FC300000000000000000000000000000000000C4
:10FC400000000000000000000000000000000000B4
:10FC500000000000000000000000000000000000A4
:10FC60000000CC7000000000000000000000000058
:10FC7000FF90000000000000000000000000FF9066
:10FC8000000000000000000000000400FF900000E1
:10FC90000000000000000049EF00FF90000000009D
:10FCA000000000049EFFFF00FF9000000000000025
:10FCB00038DFFFFFFE00FF9000000000017DFFFF26
:10FCC000FFD94000FF9000000005BFFFFFFD83004B
:10FCD0000000FF90000039EFFFFFE8300000000057
:10FCE000FF90006CFFFFFE94000000000000FF92F8
:10FCF0008EFFFFFB5000000000000000FFEFFFFF41
:10FD0000D7100000000000000000FFFFFFA400006B
:10FD10000000000000000000FFFD71000000000076
:10FD2000000000000000BA400000000000000000D9
:10FD300000000000000000000000000000000000C3
:10FD400000000000000000000000000000000000B3
:10FD500000000000000000000000000000000000A3
:10FD60000000000000000367620000000000244261
:10FD700000000004DFFFFFB20000003CFFFFC400F2
:10FD8000008FFFFFFFFE300005FFFFFFFF7008FF41
:10FD9000FB77AFFFE1003FFFA78DFFF64FFC200090
:10FDA00002DFF900BFE300008FFEDFB00000002E8D
:10FDB000FF00FF60000008FFFE1000000008FF4089
:10FDC000FF10000000CFF70000000004FF60FF00FC
:10FDD0000000003FF90000000003FF60FF2000006A
:10FDE000005FFF1000000005FF50FF80000003EFE0
:10FDF000FFA00000000AFF20DFF600005EFCCFF845
:10FE00000000004FFD004FFFC89DFFF33FFFA20021
:10FE100006FFF50007FFFFFFFE4006FFFFDCEFFFD8
:10FE2000A000004CFFFF9100005EFFFFFFFA000002
:10FE300000002430000000018EFFFB4000000000A5
:10FE400000000000000000110000000000000000A1
:10FE500000000000000000000000000000000000A2
:10FE6000000000000000000000000002210000006F
:10FE700000000000000000017DFFFFEA30000000EC
:10FE800000044000006EFFFFFFFFFA000000006F5B
:10FE9000E20008FFFFB99BEFFFC0000000BFFA00BF
:10FEA0004FFF70000005EFF80000000CFF10DFF3BB
:10FEB000000000001EFF10000006FF50FF80000041
:10FEC000000006FF50000004FF60FF40000000003B
:10FED00001FF70000004FF60FF300000000001FF20
:10FEE00070000007FF40FF700000000004FF4000AA
:10FEF000000DFE00EFE2000000000BFD0000009F7F
:10FF0000F8007FFD300000007FF400001AFFD100F0
:10FF10000BFFFB520008FF60136AFFFE200000AFDA
:10FF2000FFFFFFFFFFEFFFFFFFC200000004BFFF66
:10FF3000FFFFFFFFFFFFC500000000000269CDEFDB
:10FF4000FFEDB962000000000000000000000000AA
:10FF500000000000000000000000000000000000A1
:10FF600000000000FFFFFFFFFFFFFFFFFFFFFFFF9D
:10FF7000FFFFFFFFFFFFFFFFFFFFFFFFFFFFFFFF91
:10FF8000FFFFFFFFFFFFFFFFFFFFFFFFFFFFFFFF81
:10FF9000FFFFFFFFFFFFFFFFFFFFFFFFFFFFFFFF71
:10FFA000FFFFFFFFFFFFFFFFFFFFFFFFFFFFFFFF61
:10FFB000FFFFFFFFFFFFFFFFFFFFFFFFFFFFFFFF51
:10FFC000FFFFFFFFFFFFFFFFFFFFFFFFFFFFFFFF41
:10FFD000FFFFFFFFFFFFFFFFFFFFFFFFFFFFFFFF31
:10FFE000FFFFFFFFFFFFFFFFFFFFFFFFFFFFFFFF21
:10FFF000FFFFFFFFFFFFFFFFFFFFFFFFFFFFFFFF11
:020000040001F9
:10000000D7EC85F00501206921691200FFFFFFFF91
:10001000FFFFFFFFFFFFFFFFFFFFFFFFFFFFFFFFF0
:10002000EAEC84F057EFA4F0FFFFFFFFFFFFFFFFB4
:10003000C6EFAFF06EEFB5F0BFEFB5F00000FFFF19
:1000400080EC83F005011E6B1200FFFFFFFFFFFF36
:10005000CEEFAFF0FFFFFFFFFFFFFFFFFFFFFFFF50
:1000600057EFA4F0FFFFFFFFFFFFFFFFFFFFFFFFC2
:10007000FFFFFFFFFFFFFFFFFFFFFFFFFFFFFFFF90
:10008000C8ECA8F00501030E236F57EFA4F0FFFFA3
:10009000FFFFFFFFFFFFFFFFFFFFFFFFFFFFFFFF70
:1000A000120000EE00F00D0EEE6AEA62FDD71200BB
:1000B00066EF6AF076EF6AF0FFFFFFFFFFFFFFFFDA
:1000C00013EFA3F01AEFB6F046EFB6F0FFFFFFFF15
:1000D000FFFFFFFFFFFFFFFFFFFFFFFFFFFFFFFF30
:1000E0002FEFAEF0D9CFE6FFDACFE6FFE1CFD9FFB1
:1000F000E2CFDAFFE652006801687F0E026E036A03
:10010000D950FA0FE96EFF0EDA20EA6EEE500016B3
:10011000EE500116EE500216EE5003166AD800C0DB
:10012000EEFF01C0EEFF02C0EEFF03C0EEFFFD0ECA
:10013000DB50800B02E0010E01D0000EE66E59D8B4
:10014000060EE926000EEA22E552E750EF6EFC0E9D
:10015000DBCF00F0FD0EDBCF01F0D890003601368A
:10016000FC0E00C0DBFFFD0E01C0DBFFDB50E66EC6
:1001700040D8040EE926000EEA22E552E750EE6E62
:10018000ED6AFD0EDB50006E016AFF0E001818E1EB
:10019000015016E12ED8EECF00F0EECF01F0EECFF9
:1001A00002F0EFCF03F0005001100210031006E040
:1001B000210E04017C6F7D6B800E0BD0040E09D0E4
:1001C000FD0EDB5008E115D8EE6AEE6AEE6AEE6AC3
:1001D000010EDF6E06D0020EDF6E0BD8EE52EE522D
:1001E000EE8EDF50E552E552E5CFDAFFE7CFD9FFDB
:1001F0001200F80EDBCFE9FFF90EDBCFEAFF1200A9
:10020000BB073BBCFFD03B3C0CF83AF297493AA302
:100210003AE93A6018043A1E099039DF4C01399DD9
:100220003EE5395EED3A39258D333901BAC638CA13
:10023000DC82389E4D8438789D9F3842AC34381823
:10024000C9A33C78BD453BF902CC3BA0443E3B589A
:1002500023623B14FA313AD06DA43A93FBDD3A4F56
:10026000F8033A12718D39DB55AB39AB1277398609
:100270001EEA3952542C3924B2373900DBDA38C936
:1002800044673FA100003F809EED3F5C96533F4195
:10029000B8523F1E19CE3F01CAC13EE1CCCD3ECC83
:1002A00000003EC033333EB3B4393EA8ED913E9CCE
:1002B00026E93E91A1CB3E85F3B63E7D48E93E6EF0
:1002C00006F73FDF06253FB1902E3F98DCC73F85FC
:1002D00008313F6C0C4A3F52020C3F3B73823F2671
:1002E00051EC3F18F3B63F0D86593F08D6A13F04A5
:1002F000A2343F04816F3F0467383F040BE13F03A2
:1003000047AE3F01C2273F26E2193F3851EC3F4834
:10031000068E3F50E9103F578A723F5E18933F6444
:10032000C1553F68154D3F6C91003F6EB7803F70DF
:100330009C783F72538F3F74CFAB3F751DE73F777B
:1003400058103ED91F8A3F1317593F27E8A73F3857
:1003500019653F42B2FF3F4BF1413F53F4F13F5A21
:100360002DE03F60EAB33F6352BD3F6644D03F6833
:1003700085F03F69C7113F6AF4883F6B3C363F6D9B
:10038000AA3BC0B8AA3BC13844FEC19084D4C1D5B1
:10039000CFA2C21B0558C25DAD3BC29C2CCFC2DEB2
:1003A00040F6C31DA22BC352E459C38666EDC3AC0D
:1003B00002D0C3DCA9ABC40C9D93C4330720C46531
:1003C0006C0BC00B6C0BC08BE798C0D959DCC121FA
:1003D000ADBDC16B1F2EC1A7F2BFC1ECFCC7C227C8
:1003E000C193C26D3EA3C29FF7DEC2CB5544C30288
:1003F000540CC326AE9EC354C955C3872522C3AD32
:10040000EC0E3E22F9C93DA9F2A83D5CA08A3D163A
:10041000A1233CCFEC893C92D09A3C4FD3523C1262
:10042000B7263BCF333A3B9B787B3B72CAC03B3D00
:10043000C4D73B14BF583AE84EA53AB6FF0A3A8EE5
:1004400078BE3EBC01903E52DB713E0B57373DC13A
:100450006C183D8674223D3FFBBA3D07C21A3CC072
:10046000AB443C887C103C4CDE0E3C1F74913BFA44
:100470006ABB3BC4B56C3B99E0573B70FA8F3B3C81
:10048000000040800000410000004148000041940D
:10049000000041D833334219333342590000429AA5
:1004A000000042DA000043120000433B0000436FAB
:1004B00080004398000043C3000043F9C000441E7D
:1004C00047AE3FC147AE40410A3D4097AE1440DFC2
:1004D0005C294123AE1441673D7141A4E14841E8E4
:1004E000CCCD4224C28F425C6148428DAE1442B4EE
:1004F000947B42E66B8543133D71433C07AE4370EA
:10050000BEBE3F525D853F14EEEE3ED9FE4C3E9F8F
:10051000D9993E6785273E296EAD3DF54E043DB025
:100520005C8D3D7CEACD3D3D0BB03D152C233CEA76
:1005300012963CB84F6E3C9076823C62DE9F3C3116
:1005400066E03F7D35C63F660D7C3F4507EA3F21AB
:1005500053093EFCC4B53EC2B51C3E92F8A53E58B8
:1005600090BC3E1EB79E3DF148C33DBF42493D97FA
:1005700000D43D6F21693D3C14F53D142E983CE9B3
:10058000FFFFFFFFFFFFFFFFFFFFFFFFFFFFFFFF7B
:10059000FFFFFFFFFFFFFFFFFFFFFFFFFFFFFFFF6B
:1005A000FFFFFFFFFFFFFFFFFFFFFFFFFFFFFFFF5B
:1005B000FFFFFFFFFFFFFFFFFFFFFFFFFFFFFFFF4B
:1005C000FFFFFFFFFFFFFFFFFFFFFFFFFFFFFFFF3B
:1005D000FFFFFFFFFFFFFFFFFFFFFFFFFFFFFFFF2B
:1005E000FFFFFFFFFFFFFFFFFFFFFFFFFFFFFFFF1B
:1005F000FFFFFFFFFFFFFFFFFFFFFFFFFFFFFFFF0B
:100600002E29C943D8A2017C363DA154F0EC130633
:10061000A762F305C7C08C739398D92B4CBCCA82D0
:100620009B1E3C57D4FD16E04267186F178A12E5EF
:100630004EBED6C49EDA49DEFBA08EF52FBB7AEE05
:1006400068A99179B2153F07C2948910220B215FE6
:100650007F809A5D905A27323E35E7CCF7BF0397EB
:1006600019FFB330A548D1B55ED72A9256ACC6AAB9
:10067000B84FD238A496B67DFC76E26B749CF10438
:100680009D455970716420875B8665CF2DE602A871
:10069000601BAD25B0AEF6B9461C696140340F7ED3
:1006A000475523A351DD3AAF5CC3CEF9C5BA26EA5C
:1006B000532C6E0D28850984DFD3F4CD8141524D32
:1006C000DC6AC837C16CFAABE124087BBD0C4AB1C7
:1006D00088788B9563E36DE8CBE9FED5003B391D47
:1006E000EFF20EB75866E4D077A6F87275EB0A4BB6
:1006F0004431B450ED8F1A1F99DB338D119F148351
:100700000901BD6B0901306B316B0901326B336B31
:100710000901346B356B0901366B376B0901386998
:1007200013EE00F0010EF86E04018C0E346F4A0EC9
:10073000356F4A0E366F3F0E376F00C528F001C582
:1007400029F0E2EC6CF027C000F028C001F029C0CD
:1007500002F02AC003F02C6A2D6A7A0E2E6E440E27
:100760002F6E00C027F001C028F002C029F003C09E
:100770002AF08EEC6DF027C008F428C009F429C0D7
:100780000AF42AC00BF40401006B100E0401005D92
:1007900001E3FAD0DC0E2C6E680E2D6E800E2E6EEC
:1007A0003D0E2F6E08C427F009C428F00AC429F0B2
:1007B0000BC42AF0F7EC6CF027C004F028C005F059
:1007C00029C006F02AC007F004C02CF005C02DF0A7
:1007D00006C02EF007C02FF034C427F035C428F02F
:1007E00036C429F037C42AF0E1EC6DF027C000F0E0
:1007F00028C001F029C002F02AC003F00401005112
:10080000040DF3CFE9FFF4CFEAFF800EE926040ED2
:10081000EA2200C0EEFF01C0EEFF02C0EEFF03C0FF
:10082000EEFF020EF76E04010051002500250025A1
:10083000800FF66E0900F5CF41F40900F5CF40F4C2
:100840000900F5CF43F40800F5CF42F4800FF66EAF
:10085000F72A0900F5CF49F40900F5CF48F409005B
:10086000F5CF4BF40800F5CF4AF404010051040D14
:10087000F3CFE9FFF4CFEAFF800EE926040EEA2267
:10088000EECF08F0EECF09F0EECF0AF0EFCF0BF08D
:1008900040C42CF041C42DF042C42EF043C42FF0CC
:1008A00008C027F009C028F00AC029F00BC02AF0C0
:1008B000F7EC6CF027C004F028C005F029C006F062
:1008C0002AC007F048C42CF049C42DF04AC42EF0C9
:1008D0004BC42FF004C027F005C028F006C029F053
:1008E00007C02AF0E1EC6DF027C000F028C001F04D
:1008F00029C002F02AC003F004010051040DF3CF17
:10090000E9FFF4CFEAFF670EE926050EEA2200C0F0
:10091000EEFF01C0EEFF02C0EEFF03C0EEFF0401D8
:100920000051040DF3CFE9FFF4CFEAFF670EE9268B
:10093000050EEA22EECF00F0EECF01F0EECF02F08E
:10094000EFCF03F02C6A2D6A2E6A2F6A00C027F0C1
:1009500001C028F002C029F003C02AF0D2EC6EF0EA
:10096000010A0FE104010051040DF3CFE9FFF4CFB8
:10097000EAFF670EE926050EEA22EE6AEE6AEE6AE3
:10098000EE6A0401002B01D70401100E006F200E47
:100990000401005D12E204010051040DF3CFE9FFF0
:1009A000F4CFEAFF800EE926040EEA22EE6AEE6A30
:1009B000EE6AEE6A0401002BEAD713ECA0F0050101
:1009C000236B0501226B0501316B0501326B0501BB
:1009D000666B120013EE00F004018C0E346F4A0EA9
:1009E000356F4A0E366F3F0E376F00C528F001C5D0
:1009F00029F0E2EC6CF027C000F028C001F029C01B
:100A000002F02AC003F02C6A2D6A7A0E2E6E440E74
:100A10002F6E00C027F001C028F002C029F003C0EB
:100A20002AF08EEC6DF027C008F428C009F429C024
:100A30000AF42AC00BF402C528F003C529F0E2EC41
:100A40006CF027C000F028C001F029C002F02AC0D5
:100A500003F02C6A2D6A7A0E2E6E440E2F6E00C0A3
:100A600027F001C028F002C029F003C02AF08EEC64
:100A70006DF027C00CF428C00DF429C00EF42AC074
:100A80000FF4DC0E2C6E680E2D6E800E2E6E3D0E59
:100A90002F6E08C427F009C428F00AC429F00BC43B
:100AA0002AF0F7EC6CF027C000F028C001F029C054
:100AB00002F02AC003F000C02CF001C02DF002C0EB
:100AC0002EF003C02FF034C427F035C428F036C40C
:100AD00029F037C42AF0E1EC6DF027C024F428C0D7
:100AE00025F429C026F42AC027F40401286B296BB9
:100AF0002A6B2B6B0CC430F40DC431F40EC432F4E9
:100B00000FC433F413C529F0D1EC6CF027C000F00A
:100B100028C001F029C002F02AC003F02C6A2D6A17
:100B2000C80E2E6E420E2F6E00C027F001C028F0B6
:100B300002C029F003C02AF08EEC6DF027C07BF9CB
:100B400028C07CF929C07DF92AC07EF912C529F098
:100B5000D1EC6CF027C000F028C001F029C002F0F1
:100B60002AC003F02C6A2D6AC80E2E6E420E2F6E1C
:100B700000C027F001C028F002C029F003C02AF00D
:100B80008EEC6DF027C077F928C078F929C079F983
:100B90002AC07AF9BCEC8FF013ECA0F00501236BAE
:100BA0000501226B0501316BC0ECA0F012004FD89B
:100BB0000901BD5105E1010EBD6F00EC60F002D0EE
:100BC000F3EC64F04DDBC0ECA0F005012351030A07
:100BD00027E0020A1DE0010A12E093EC96F013EC04
:100BE000A0F0E3EC69F00301010E066F07EC8DF055
:100BF000050123510F0824E2020E236F23D093EC4A
:100C000096F04DEC94F016EC63F0050123691BD0CF
:100C1000030E235D01E117D0236B2DEC8BF013D075
:100C200013ECA0F0E3EC69F0C2EC69F00201C76BD1
:100C3000926B93EC96F0FCEC64F00501236B03D00F
:100C40002DEC8BF000D0E5EC95F0F7EF64F000C5EB
:100C500028F001C529F0E2EC6CF027C000F028C0B4
:100C600001F029C002F02AC003F02C6A2D6A7A0E26
:100C70002E6E440E2F6E00C027F001C028F002C077
:100C800029F003C02AF08EEC6DF027C008F428C0CC
:100C900009F429C00AF42AC00BF402C528F003C5E0
:100CA00029F0E2EC6CF027C000F028C001F029C068
:100CB00002F02AC003F02C6A2D6A7A0E2E6E440EC2
:100CC0002F6E00C027F001C028F002C029F003C039
:100CD0002AF08EEC6DF027C00CF428C00DF429C06A
:100CE0000EF42AC00FF410C529F0D1EC6CF027C027
:100CF00000F028C001F029C002F02AC003F02C6ADD
:100D00002D6AC80E2E6E420E2F6E00C027F001C055
:100D100028F002C029F003C02AF08EEC6DF027C045
:100D200034F428C035F429C036F42AC037F411C58C
:100D300029F0D1EC6CF027C000F028C001F029C0E8
:100D400002F02AC003F02C6A2D6AC80E2E6E420EE5
:100D50002F6E00C027F001C028F002C029F003C0A8
:100D60002AF08EEC6DF027C038F428C039F429C081
:100D70003AF42AC03BF41CC529F0D1EC6CF027C032
:100D800000F028C001F029C002F02AC003F02C6A4C
:100D90002D6AC80E2E6E420E2F6E00C027F001C0C5
:100DA00028F002C029F003C02AF08EEC6DF027C0B5
:100DB0005FF928C060F929C061F92AC062F91DC530
:100DC00029F0D1EC6CF027C000F028C001F029C058
:100DD00002F02AC003F02C6A2D6AC80E2E6E420E55
:100DE0002F6E00C027F001C028F002C029F003C018
:100DF0002AF08EEC6DF027C063F928C064F929C091
:100E000065F92AC066F917C529F0D1EC6CF027C046
:100E100000F028C001F029C002F02AC003F02C6ABB
:100E20002D6AC80E2E6E420E2F6E00C027F001C034
:100E300028F002C029F003C02AF08EEC6DF027C024
:100E40007FF928C080F929C081F92AC082F90501FB
:100E50001B515BE01BC529F0D1EC6CF027C004F0FE
:100E600028C005F029C006F02AC007F0850E2C6EB8
:100E7000EB0E2D6E1F0E2E6E410E2F6E04C027F04E
:100E800005C028F006C029F007C02AF08EEC6DF0EE
:100E900027C000F028C001F029C002F02AC003F0EA
:100EA0000CC42CF00DC42DF00EC42EF00FC42FF086
:100EB00000C027F001C028F002C029F003C02AF0CA
:100EC000F8EC6CF027C06FF928C070F929C071F9EF
:100ED0002AC072F97FC92CF080C92DF081C92EF08B
:100EE00082C92FF06FC927F070C928F071C929F0A5
:100EF00072C92AF0F8EC6CF027C06FF928C070F9BD
:100F000029C071F92AC072F905D009016F6B706BA5
:100F1000716B726B18C529F0D1EC6CF027C000F032
:100F200028C001F029C002F02AC003F02C6A2D6A03
:100F3000C80E2E6E420E2F6E00C027F001C028F0A2
:100F400002C029F003C02AF08EEC6DF027C0EFF547
:100F500028C0F0F529C0F1F52AC0F2F519C529F02D
:100F6000D1EC6CF027C004F028C005F029C006F0D1
:100F70002AC007F0660E2C6EE60E2D6EC70E2E6E82
:100F8000420E2F6E04C027F005C028F006C029F0DD
:100F900007C02AF08EEC6DF027C000F028C001F0E9
:100FA00029C002F02AC003F00CC42CF00DC42DF0AF
:100FB0000EC42EF00FC42FF000C027F001C028F09F
:100FC00002C029F003C02AF0F8EC6CF027C0F3F55A
:100FD00028C0F4F529C0F5F52AC0F6F57FC92CF034
:100FE00080C92DF081C92EF082C92FF0F3C527F0FA
:100FF000F4C528F0F5C529F0F6C52AF0F8EC6CF038
:1010000027C0F3F528C0F4F529C0F5F52AC0F6F598
:101010001AC529F0D1EC6CF027C000F028C001F00F
:1010200029C002F02AC003F02C6A2D6AC80E2E6E69
:10103000420E2F6E00C027F001C028F002C029F038
:1010400003C02AF08EEC6DF027C0F7F528C0F8F544
:1010500029C0F9F52AC0FAF513C529F0D1EC6CF0D6
:1010600027C000F028C001F029C002F02AC003F018
:101070002C6A2D6AC80E2E6E420E2F6E00C027F00D
:1010800001C028F002C029F003C02AF08EEC6DF0F8
:1010900027C07BF928C07CF929C07DF92AC07EF9D8
:1010A00012C529F0D1EC6CF027C000F028C001F087
:1010B00029C002F02AC003F02C6A2D6AC80E2E6ED9
:1010C000420E2F6E00C027F001C028F002C029F0A8
:1010D00003C02AF08EEC6DF027C077F928C078F9AC
:1010E00029C079F92AC07AF915C529F0D1EC6CF03C
:1010F00027C000F028C001F029C002F02AC003F088
:101100002C6A2D6AC80E2E6E420E2F6E00C027F07C
:1011100001C028F002C029F003C02AF08EEC6DF067
:1011200027C097F228C098F229C099F22AC09AF2F3
:1011300014C529F0D1EC6CF027C000F028C001F0F4
:1011400029C002F02AC003F02C6A2D6AC80E2E6E48
:10115000420E2F6E00C027F001C028F002C029F017
:1011600003C02AF08EEC6DF027C09BF228C09CF2E1
:1011700029C09DF22AC09EF297C22CF098C22DF091
:1011800099C22EF09AC22FF09BC227F09CC228F081
:101190009DC229F09EC22AF0F7EC6CF027C09FF2A6
:1011A00028C0A0F229C0A1F22AC0A2F20CC42CF0DF
:1011B0000DC42DF00EC42EF00FC42FF008C427F07C
:1011C00009C428F00AC429F00BC42AF0F7EC6CF02B
:1011D00027C000F028C001F029C002F02AC003F0A7
:1011E000F00E2C6E850E2D6E990E2E6E3E0E2F6E0D
:1011F00000C027F001C028F002C029F003C02AF087
:101200008EEC6DF027C014F428C015F429C016F434
:101210002AC017F414C427F015C428F016C429F006
:1012200017C42AF093EC6EF028C004F429C005F42A
:101230000401000E045D000E055902E2046B056B0B
:10124000FF0ED8800455000E055502E20469056BB7
:1012500004C44FF205011E510201C36FC46B12009A
:10126000010E02019025906F000E9121916F0501F2
:10127000185109E108C4E7F509C4E8F50AC4E9F51D
:101280000BC4EAF54ED0EFC52CF0F0C52DF0F1C53A
:101290002EF0F2C52FF008C427F009C428F00AC4C4
:1012A00029F00BC42AF0F7EC6CF027C000F028C03E
:1012B00001F029C002F02AC003F038C42CF039C470
:1012C0002DF03AC42EF03BC42FF034C427F035C4BF
:1012D00028F036C429F037C42AF0F8EC6CF027C0A7
:1012E00004F028C005F029C006F02AC007F004C0A9
:1012F0002CF005C02DF006C02EF007C02FF000C066
:1013000027F001C028F002C029F003C02AF08EECBB
:101310006DF027C0E7F528C0E8F529C0E9F52AC037
:10132000EAF508C42CF009C42DF00AC42EF00BC451
:101330002FF0E7C527F0E8C528F0E9C529F0EAC590
:101340002AF0C9EC6EF0010A08E108C4E7F509C407
:10135000E8F50AC4E9F50BC4EAF5DC0E2C6E680E5C
:101360002D6E800E2E6E3D0E2F6EE7C527F0E8C560
:1013700028F0E9C529F0EAC52AF0C9EC6EF0010AA7
:1013800001E097D0DC0E2C6E680E2D6E800E2E6E56
:101390003D0E2F6EE7C527F0E8C528F0E9C529F016
:1013A000EAC52AF0F7EC6CF027C000F028C001F085
:1013B00029C002F02AC003F000C02CF001C02DF0BB
:1013C00002C02EF003C02FF034C427F035C428F03B
:1013D00036C429F037C42AF0E1EC6DF027C024F4BC
:1013E00028C025F429C026F42AC027F4DC0E2C6E70
:1013F000680E2D6E800E2E6E3D0E2F6EE7C527F007
:10140000E8C528F0E9C529F0EAC52AF0F7EC6CF048
:1014100027C000F028C001F029C002F02AC003F064
:1014200000C02CF001C02DF002C02EF003C02FF040
:1014300038C427F039C428F03AC429F03BC42AF054
:10144000E1EC6DF027C028F428C029F429C02AF463
:101450002AC02BF408C42CF009C42DF00AC42EF0C5
:101460000BC42FF0E7C527F0E8C528F0E9C529F03F
:10147000EAC52AF08EEC6DF027C000F028C001F01C
:1014800029C002F02AC003F02C6A2D6AC80E2E6E05
:10149000420E2F6E00C027F001C028F002C029F0D4
:1014A00003C02AF0E1EC6DF06CEC6EF029C064F53D
:1014B0000BD00401246B256B266B276B286B296BE3
:1014C0002A6B2B6B0501646B0CC430F40DC431F432
:1014D0000EC432F40FC433F4BCEC8FF00501635139
:1014E000040DF3CFE9FFF4CFEAFF670EE926050EFE
:1014F000EA22EECF00F0EECF01F0EECF02F0EFCF18
:1015000003F02C6A2D6A7A0E2E6E440E2F6E00C0E8
:1015100027F001C028F002C029F003C02AF0E1EC56
:101520006DF093EC6EF028C044F229C045F205013D
:101530006351040DF3CFE9FFF4CFEAFF800EE926F3
:10154000040EEA22EECF04F0EECF05F0EECF06F067
:10155000EFCF07F0100E6325040DF3CFE9FFF4CFB2
:10156000EAFF800EE926040EEA22EECF08F0EECF65
:1015700009F0EECF0AF0EFCF0BF008C02CF009C055
:101580002DF00AC02EF00BC02FF004C027F005C0CC
:1015900028F006C029F007C02AF0F8EC6CF027C04C
:1015A00000F028C001F029C002F02AC003F02C6A24
:1015B0002D6A7A0E2E6E440E2F6E00C027F001C0E9
:1015C00028F002C029F003C02AF0E1EC6DF093ECA2
:1015D0006EF028C046F229C047F205011F051BE145
:1015E0009BC22CF09CC22DF09DC22EF09EC22FF00B
:1015F00010C427F011C428F012C429F013C42AF033
:10160000E1EC6DF027C010F428C011F429C012F4E9
:101610002AC013F408D030C410F431C411F432C419
:1016200012F433C413F410C42CF011C42DF012C4FE
:101630002EF013C42FF070C427F071C428F072C4C8
:1016400029F073C42AF0C9EC6EF0010A05E1050126
:10165000235102E1226B236912000401066B076B20
:10166000FCEC64F00201000ED880BF55000EC0559E
:1016700001E3B8D1050118513EE120C4EBF521C4C6
:10168000ECF522C4EDF523C4EEF56FC92CF070C95A
:101690002DF071C92EF072C92FF020C427F021C49B
:1016A00028F022C429F023C42AF0C9EC6EF0010A04
:1016B00011E134C467F935C468F936C469F937C42F
:1016C0006AF938C46BF939C46CF93AC46DF93BC492
:1016D0006EF910D05FC967F960C968F961C969F925
:1016E00062C96AF963C96BF964C96CF965C96DF9B6
:1016F00066C96EF9C1D034C467F935C468F936C417
:1017000069F937C46AF938C46BF939C46CF93AC459
:101710006DF93BC46EF9F3C52CF0F4C52DF0F5C599
:101720002EF0F6C52FF020C427F021C428F022C4E3
:1017300029F023C42AF0C9EC6EF0010A4FE1EFC58D
:101740002CF0F0C52DF0F1C52EF0F2C52FF020C41D
:1017500027F021C428F022C429F023C42AF0F7EC92
:101760006CF027C000F028C001F029C002F02AC0A8
:1017700003F038C42CF039C42DF03AC42EF03BC429
:101780002FF034C427F035C428F036C429F037C40C
:101790002AF0F8EC6CF027C004F028C005F029C04E
:1017A00006F02AC007F004C02CF005C02DF006C0DA
:1017B0002EF007C02FF000C027F001C028F002C0B3
:1017C00029F003C02AF08EEC6DF027C0EBF528C09D
:1017D000ECF529C0EDF52AC0EEF54ED0F7C52CF09A
:1017E000F8C52DF0F9C52EF0FAC52FF020C427F06A
:1017F00021C428F022C429F023C42AF0F7EC6CF0AD
:1018000027C000F028C001F029C002F02AC003F070
:1018100038C42CF039C42DF03AC42EF03BC42FF05C
:1018200034C427F035C428F036C429F037C42AF070
:10183000F8EC6CF027C004F028C005F029C006F0D1
:101840002AC007F004C02CF005C02DF006C02EF011
:1018500007C02FF000C027F001C028F002C029F017
:1018600003C02AF08EEC6DF027C0EBF528C0ECF534
:1018700029C0EDF52AC0EEF520C42CF021C42DF0CE
:1018800022C42EF023C42FF0EBC527F0ECC528F0BE
:10189000EDC529F0EEC52AF0C9EC6EF0010A08E1A9
:1018A00020C4EBF521C4ECF522C4EDF523C4EEF51C
:1018B000DC0E2C6E680E2D6E800E2E6E3D0E2F6E81
:1018C000EBC527F0ECC528F0EDC529F0EEC52AF0F0
:1018D000C9EC6EF0010A69E1DC0E2C6E680E2D6E0B
:1018E000800E2E6E3D0E2F6EEBC527F0ECC528F056
:1018F000EDC529F0EEC52AF0F7EC6CF027C000F03A
:1019000028C001F029C002F02AC003F000C02CF06A
:1019100001C02DF002C02EF003C02FF067C927F0E0
:1019200068C928F069C929F06AC92AF0E1EC6DF0AC
:1019300027C024F428C025F429C026F42AC027F49F
:10194000DC0E2C6E680E2D6E800E2E6E3D0E2F6EF0
:10195000EBC527F0ECC528F0EDC529F0EEC52AF05F
:10196000F7EC6CF027C000F028C001F029C002F0AD
:101970002AC003F000C02CF001C02DF002C02EF0F0
:1019800003C02FF06BC927F06CC928F06DC929F08E
:101990006EC92AF0E1EC6DF027C028F428C029F4C4
:1019A00029C02AF42AC02BF409D00401246B256B2A
:1019B000266B276B286B296B2A6B2B6BD0EC97F06F
:1019C000F5EC69F00201010EC16F22ECA0F00501F7
:1019D0002329236F100E235D04E2010E0401066F1C
:1019E000076B02D00501236B0401010E061901E10A
:1019F000075101E132D6050123510F0803E2010E20
:101A0000236F04D0C2EC69F00501236B120093EC44
:101A100096F00501236B08C420F409C421F40AC41C
:101A200022F40BC423F40201010E926F0401066B31
:101A3000076B2C6A2D6A800E2E6E3F0E2F6E20C40F
:101A400027F021C428F022C429F023C42AF0F7EC9F
:101A50006CF027C020F428C021F429C022F42AC049
:101A600023F405011F0509E1B7C293F2B8C294F24D
:101A7000B9C295F2BAC296F208D074C493F275C492
:101A800094F276C495F277C496F293C22CF094C285
:101A90002DF095C22EF096C22FF020C427F021C45D
:101AA00028F022C429F023C42AF0C9EC6EF0010A00
:101AB00001E05AD20CC42CF00DC42DF00EC42EF04F
:101AC0000FC42FF020C427F021C428F022C429F02D
:101AD00023C42AF0C9EC6EF0010A01E045D20201EC
:101AE000926B0301066B0501185164E12C6A2D6AA3
:101AF0002E6A3F0E2F6E20C427F021C428F022C486
:101B000029F023C42AF0F8EC6CF027C0EBF528C0CC
:101B1000ECF529C0EDF52AC0EEF52C6A2D6A2E6A87
:101B20003F0E2F6E20C427F021C428F022C429F0D4
:101B300023C42AF0F8EC6CF027C000F028C001F0B4
:101B400029C002F02AC003F06FC92CF070C92DF033
:101B500071C92EF072C92FF000C027F001C028F023
:101B600002C029F003C02AF0C9EC6EF0010A11E1AD
:101B700034C467F935C468F936C469F937C46AF9F9
:101B800038C46BF939C46CF93AC46DF93BC46EF9C9
:101B900010D05FC967F960C968F961C969F962C99C
:101BA0006AF963C96BF964C96CF965C96DF966C9ED
:101BB0006EF948D134C467F935C468F936C469F997
:101BC00037C46AF938C46BF939C46CF93AC46DF991
:101BD0003BC46EF92C6A2D6A2E6A3F0E2F6E20C40C
:101BE00027F021C428F022C429F023C42AF0F8ECFD
:101BF0006CF027C000F028C001F029C002F02AC014
:101C000003F0F3C52CF0F4C52DF0F5C52EF0F6C5A4
:101C10002FF000C027F001C028F002C029F003C057
:101C20002AF0C9EC6EF0010A66E12C6A2D6A2E6A70
:101C30003F0E2F6E20C427F021C428F022C429F0C3
:101C400023C42AF0F8EC6CF027C004F028C005F09B
:101C500029C006F02AC007F0EFC52CF0F0C52DF022
:101C6000F1C52EF0F2C52FF004C027F005C028F012
:101C700006C029F007C02AF0F7EC6CF027C000F08E
:101C800028C001F029C002F02AC003F038C42CF0AB
:101C900039C42DF03AC42EF03BC42FF034C427F0E1
:101CA00035C428F036C429F037C42AF0F8EC6CF0BB
:101CB00027C008F028C009F029C00AF02AC00BF09C
:101CC00008C02CF009C02DF00AC02EF00BC02FF078
:101CD00000C027F001C028F002C029F003C02AF09C
:101CE0008EEC6DF027C0EBF528C0ECF529C0EDF5C2
:101CF0002AC0EEF565D02C6A2D6A2E6A3F0E2F6E33
:101D000020C427F021C428F022C429F023C42AF0DB
:101D1000F8EC6CF027C004F028C005F029C006F0EC
:101D20002AC007F0F7C52CF0F8C52DF0F9C52EF044
:101D3000FAC52FF004C027F005C028F006C029F02E
:101D400007C02AF0F7EC6CF027C000F028C001F0C3
:101D500029C002F02AC003F038C42CF039C42DF099
:101D60003AC42EF03BC42FF034C427F035C428F019
:101D700036C429F037C42AF0F8EC6CF027C008F01C
:101D800028C009F029C00AF02AC00BF008C02CF0C6
:101D900009C02DF00AC02EF00BC02FF000C027F0B4
:101DA00001C028F002C029F003C02AF08EEC6DF0CB
:101DB00027C0EBF528C0ECF529C0EDF52AC0EEF5FB
:101DC0002C6A2D6A2E6A3F0E2F6E20C427F021C484
:101DD00028F022C429F023C42AF0F8EC6CF027C0C4
:101DE00000F028C001F029C002F02AC003F000C0B2
:101DF0002CF001C02DF002C02EF003C02FF0EBC577
:101E000027F0ECC528F0EDC529F0EEC52AF0C9ECA5
:101E10006EF0010A17E12C6A2D6A2E6A3F0E2F6EB2
:101E200020C427F021C428F022C429F023C42AF0BA
:101E3000F8EC6CF027C0EBF528C0ECF529C0EDF507
:101E40002AC0EEF5DC0E2C6E680E2D6E800E2E6E06
:101E50003D0E2F6EEBC527F0ECC528F0EDC529F03F
:101E6000EEC52AF0C9EC6EF0010A69E1DC0E2C6EB9
:101E7000680E2D6E800E2E6E3D0E2F6EEBC527F078
:101E8000ECC528F0EDC529F0EEC52AF0F7EC6CF0B2
:101E900027C000F028C001F029C002F02AC003F0DA
:101EA00000C02CF001C02DF002C02EF003C02FF0B6
:101EB00067C927F068C928F069C929F06AC92AF0FA
:101EC000E1EC6DF027C024F428C025F429C026F4E5
:101ED0002AC027F4DC0E2C6E680E2D6E800E2E6E3E
:101EE0003D0E2F6EEBC527F0ECC528F0EDC529F0AF
:101EF000EEC52AF0F7EC6CF027C000F028C001F026
:101F000029C002F02AC003F000C02CF001C02DF05F
:101F100002C02EF003C02FF06BC927F06CC928F067
:101F20006DC929F06EC92AF0E1EC6DF027C028F4E4
:101F300028C029F429C02AF42AC02BF409D00401AE
:101F4000246B256B266B276B286B296B2A6B2B6BFD
:101F5000D0EC97F005012329236F100E235D04E2D6
:101F6000010E0401066F076B0401010E061901E161
:101F7000075101E15BD5120013EE00F0010EF86E7F
:101F8000050163690401706B716B726B736B040103
:101F9000006B100E0401005D02E34CEF94F0020EA2
:101FA000F76E04010051002500250025F66E09009A
:101FB000F5CF59F40900F5CF58F40900F5CF5BF4DB
:101FC0000800F5CF5AF4400FF66E0900F5CF5DF426
:101FD0000900F5CF5CF40900F5CF5FF40800F5CFF8
:101FE0005EF4400FF66E0900F5CF41F40900F5CF1D
:101FF00040F40900F5CF43F40800F5CF42F4400F58
:10200000F66E0900F5CF45F40900F5CF44F4090058
:10201000F5CF47F40800F5CF46F4400FF66EF72AE7
:102020000900F5CF49F40900F5CF48F40900F5CFD0
:102030004BF40800F5CF4AF4400FF66E0900F5CFD7
:102040004DF40900F5CF4CF40900F5CF4FF408002A
:10205000F5CF4EF4D40E2C6E400E2D6E180E2E6E53
:10206000380E2F6E58C427F059C428F05AC429F0EE
:102070005BC42AF0D2EC6EF0010A01E1DED0450E1D
:102080002C6E120E2D6EBD0E2E6E3B0E2F6E58C492
:1020900027F059C428F05AC429F05BC42AF0C9ECCF
:1020A0006EF0010A01E1C9D04B0E2C6E890E2D6E27
:1020B000C90E2E6E380E2F6E5CC427F05DC428F05A
:1020C0005EC429F05FC42AF0D2EC6EF0010A01E18F
:1020D000B4D09A0E2C6E990E2D6E190E2E6E3E0EE9
:1020E0002F6E5CC427F05DC428F05EC429F05FC485
:1020F0002AF0C9EC6EF0010A01E19FD0440E2C6E6B
:102100008B0E2D6E6C0E2E6E3E0E2F6E40C427F081
:1021100041C428F042C429F043C42AF0D2EC6EF046
:10212000010A01E18AD05C0E2C6E8F0E2D6EA20E7C
:102130002E6E3F0E2F6E40C427F041C428F042C4DB
:1021400029F043C42AF0C9EC6EF0010A76E0250EAE
:102150002C6E060E2D6E010E2E6E3F0E2F6E48C495
:1021600027F049C428F04AC429F04BC42AF0D2EC25
:102170006EF0010A62E0C70E2C6E4B0E2D6E770ECC
:102180002E6E3F0E2F6E48C427F049C428F04AC473
:1021900029F04BC42AF0C9EC6EF0010A4EE05C0E47
:1021A0002C6E8F0E2D6E020E2E6E3F0E2F6E44C4BF
:1021B00027F045C428F046C429F047C42AF0D2ECE1
:1021C0006EF0010A3AE02C6A2D6AE00E2E6E3F0E88
:1021D0002F6E44C427F045C428F046C429F047C4F4
:1021E0002AF0C9EC6EF0010A28E0750E2C6E930EF1
:1021F0002D6ED80E2E6E3E0E2F6E4CC427F04DC4A1
:1022000028F04EC429F04FC42AF0D2EC6EF0010A37
:1022100014E0DF0E2C6E4F0E2D6E6D0E2E6E3F0EE7
:102220002F6E4CC427F04DC428F04EC429F04FC483
:102230002AF0C9EC6EF0010A02E10901358B0401B4
:102240000051040DF3CFE9FFF4CFEAFF800EE92639
:10225000040EEA22EECF04F0EECF05F0EECF06F04A
:10226000EFCF07F004C02CF005C02DF006C02EF013
:1022700007C02FF024C427F025C428F026C429F075
:1022800027C42AF0F7EC6CF027C000F028C001F05A
:1022900029C002F02AC003F058C42CF059C42DF014
:1022A0005AC42EF05BC42FF000C027F001C028F004
:1022B00002C029F003C02AF0E1EC6DF027C02CF435
:1022C00028C02DF429C02EF42AC02FF41CEC6AF08B
:1022D00004010051040DF3CFE9FFF4CFEAFF800EB3
:1022E000E926040EEA22EECF04F0EECF05F0EECFA1
:1022F00006F0EFCF07F02CC42CF02DC42DF02EC427
:102300002EF02FC42FF004C027F005C028F006C01F
:1023100029F007C02AF0F8EC6CF027C000F028C0C4
:1023200001F029C002F02AC003F004010051040D9D
:10233000F3CFE9FFF4CFEAFF800EE926040EEA228C
:1023400000C0EEFF01C0EEFF02C0EEFF03C0EEFFD3
:10235000100E04010025040DF3CFE9FFF4CFEAFFCE
:10236000800EE926040EEA22EECF04F0EECF05F04F
:10237000EECF06F0EFCF07F004C02CF005C02DF033
:1023800006C02EF007C02FF028C427F029C428F07B
:102390002AC429F02BC42AF0F7EC6CF027C000F017
:1023A00028C001F029C002F02AC003F05CC42CF060
:1023B0005DC42DF05EC42EF05FC42FF000C027F086
:1023C00001C028F002C029F003C02AF0E1EC6DF052
:1023D00027C02CF428C02DF429C02EF42AC02FF4D5
:1023E0001CEC6AF0100E04010025040DF3CFE9FF88
:1023F000F4CFEAFF800EE926040EEA22EECF04F0C5
:10240000EECF05F0EECF06F0EFCF07F02CC42CF0A6
:102410002DC42DF02EC42EF02FC42FF004C027F0B1
:1024200005C028F006C029F007C02AF0F8EC6CF0CF
:1024300027C000F028C001F029C002F02AC003F034
:10244000100E04010025040DF3CFE9FFF4CFEAFFDD
:10245000800EE926040EEA2200C0EEFF01C0EEFF66
:1024600002C0EEFF03C0EEFF04010051040DF3CFE4
:10247000E9FFF4CFEAFF800EE926040EEA22EECF50
:1024800000F0EECF01F0EECF02F0EFCF03F0100E30
:1024900004010025040DF3CFE9FFF4CFEAFF800E1D
:1024A000E926040EEA22EECF04F0EECF05F0EECFDF
:1024B00006F0EFCF07F004C02CF005C02DF006C0E9
:1024C0002EF007C02FF000C027F001C028F002C096
:1024D00029F003C02AF0F8EC6CF027C02CF428C0D7
:1024E0002DF429C02EF42AC02FF404010051040D4C
:1024F000F3CFE9FFF4CFEAFF800EE926040EEA22CB
:10250000EECF08F0EECF09F0EECF0AF0EFCF0BF0F0
:1025100008C02CF009C02DF00AC02EF00BC02FF01F
:1025200040C427F041C428F042C429F043C42AF033
:10253000E1EC6DF027C004F028C005F029C006F0DA
:102540002AC007F0100E04010025040DF3CFE9FFA7
:10255000F4CFEAFF800EE926040EEA22EECF10F057
:10256000EECF11F0EECF12F0EFCF13F010C02CF041
:1025700011C02DF012C02EF013C02FF044C427F06C
:1025800045C428F046C429F047C42AF0E1EC6DF0B8
:1025900027C00CF028C00DF029C00EF02AC00FF0A3
:1025A0000CC02CF00DC02DF00EC02EF00FC02FF07F
:1025B00004C027F005C028F006C029F007C02AF0A3
:1025C000F8EC6CF027C000F028C001F029C002F040
:1025D0002AC003F02CC42CF02DC42DF02EC42EF0F4
:1025E0002FC42FF000C027F001C028F002C029F04E
:1025F00003C02AF08EEC6DF027C040F428C041F4EF
:1026000029C042F42AC043F404010051040DF3CF61
:10261000E9FFF4CFEAFF800EE926040EEA22EECFAE
:1026200008F0EECF09F0EECF0AF0EFCF0BF008C0C4
:102630002CF009C02DF00AC02EF00BC02FF048C4BA
:1026400027F049C428F04AC429F04BC42AF0E1EC31
:102650006DF027C004F028C005F029C006F02AC09C
:1026600007F0100E04010025040DF3CFE9FFF4CFAD
:10267000EAFF800EE926040EEA22EECF10F0EECF3C
:1026800011F0EECF12F0EFCF13F010C02CF011C00C
:102690002DF012C02EF013C02FF04CC427F04DC403
:1026A00028F04EC429F04FC42AF0E1EC6DF027C0A9
:1026B0000CF028C00DF029C00EF02AC00FF00CC09D
:1026C0002CF00DC02DF00EC02EF00FC02FF004C066
:1026D00027F005C028F006C029F007C02AF0F8EC62
:1026E0006CF027C000F028C001F029C002F02AC019
:1026F00003F02CC42CF02DC42DF02EC42EF02FC4CA
:102700002FF000C027F001C028F002C029F003C05C
:102710002AF08EEC6DF027C048F428C049F429C097
:102720004AF42AC04BF440C42CF041C42DF042C4FA
:102730002EF043C42FF02CC427F02DC428F02EC453
:1027400029F02FC42AF0F7EC6CF027C004F028C061
:1027500005F029C006F02AC007F048C42CF049C48F
:102760002DF04AC42EF04BC42FF004C027F005C052
:1027700028F006C029F007C02AF0E1EC6DF027C070
:1027800000F028C001F029C002F02AC003F00401C3
:102790000051040DF3CFE9FFF4CFEAFF670EE926FD
:1027A000050EEA2200C0EEFF01C0EEFF02C0EEFF00
:1027B00003C0EEFF04010051040DF3CFE9FFF4CF95
:1027C000EAFF670EE926050EEA22EECF00F0EECF13
:1027D00001F0EECF02F0EFCF03F02C6A2D6A2E6AE3
:1027E0002F6A00C027F001C028F002C029F003C002
:1027F0002AF0D2EC6EF0010A0FE104010051040D41
:10280000F3CFE9FFF4CFEAFF670EE926050EEA22CF
:10281000EE6AEE6AEE6AEE6A04010051040DF3CF2F
:10282000E9FFF4CFEAFF670EE926050EEA22EECFB4
:1028300000F0EECF01F0EECF02F0EFCF03F070C466
:102840002CF071C42DF072C42EF073C42FF000C0B0
:1028500027F001C028F002C029F003C02AF0C9EC1B
:102860006EF0010A15E104010051040DF3CFE9FFF8
:10287000F4CFEAFF670EE926050EEA22EECF70F4E8
:10288000EECF71F4EECF72F4EFCF73F400C463F5C2
:102890000401002BC9EF8FF012000501226B010E1D
:1028A0000401046F056BEDD8F1EC9BF00A0E0501F5
:1028B0002225226F010E04010425046F000E05215C
:1028C000056F05011F0535E1B3C22CF0B4C22DF030
:1028D000B5C22EF0B6C22FF09BC227F09CC228F0E2
:1028E0009DC229F09EC22AF0E1EC6DF027C000F0F5
:1028F00028C001F029C002F02AC003F0AFC22CF0BA
:10290000B0C22DF0B1C22EF0B2C22FF000C027F03D
:1029100001C028F002C029F003C02AF0F8EC6CF0E6
:1029200027C010F428C011F429C012F42AC013F4EF
:1029300008D074C410F475C411F476C412F477C4CA
:1029400013F430C42CF031C42DF032C42EF033C453
:102950002FF010C427F011C428F012C429F013C4BA
:102960002AF0C9EC6EF0010A03E104010469056B69
:102970000401110E045D000E055995E3FF0E0419C4
:1029800001E1055105E1CFD80A0E0501225D226F54
:10299000010E0401046F056B3C0E0501225D70E21F
:1029A000FFDA05012229226F010E04010425046FBC
:1029B000000E0521056F05011F0535E1B3C22CF09E
:1029C000B4C22DF0B5C22EF0B6C22FF09BC227F0D4
:1029D0009CC228F09DC229F09EC22AF0E1EC6DF065
:1029E00027C000F028C001F029C002F02AC003F07F
:1029F000AFC22CF0B0C22DF0B1C22EF0B2C22FF097
:102A000000C027F001C028F002C029F003C02AF05E
:102A1000F8EC6CF027C010F428C011F429C012F4AF
:102A20002AC013F408D074C410F475C411F476C429
:102A300012F477C413F430C42CF031C42DF032C436
:102A40002EF033C42FF010C427F011C428F012C4A4
:102A500029F013C42AF0C9EC6EF0010A03E1040165
:102A60000469056B04010A0E045D000E055998E324
:102A7000FF0E041901E1055103E105012205226F52
:102A800012000401016B100E015D4CE20151040DB6
:102A9000F3CFE9FFF4CFEAFF000EE926060EEA22A3
:102AA000EECF00F0EECF01F0EECF02F0EFCF03F06B
:102AB0000151040DF3CFE9FFF4CFEAFF800EE926C0
:102AC000060EEA2200C0EEFF01C0EEFF02C0EEFFDC
:102AD00003C0EEFF100E0125040DF3CFE9FFF4CF84
:102AE000EAFF000EE926060EEA22EECF00F0EECF56
:102AF00001F0EECF02F0EFCF03F0100E0125040D30
:102B0000F3CFE9FFF4CFEAFF800EE926060EEA22B2
:102B100000C0EEFF01C0EEFF02C0EEFF03C0EEFFFB
:102B2000012BB1D712000401016B100E015D4CE2C4
:102B30000151040DF3CFE9FFF4CFEAFF800EE9263F
:102B4000060EEA22EECF00F0EECF01F0EECF02F05B
:102B5000EFCF03F00151040DF3CFE9FFF4CFEAFF0B
:102B6000000EE926060EEA2200C0EEFF01C0EEFFCD
:102B700002C0EEFF03C0EEFF100E0125040DF3CFDF
:102B8000E9FFF4CFEAFF800EE926060EEA22EECF37
:102B900000F0EECF01F0EECF02F0EFCF03F0100E19
:102BA0000125040DF3CFE9FFF4CFEAFF000EE9267B
:102BB000060EEA2200C0EEFF01C0EEFF02C0EEFFEB
:102BC00003C0EEFF012BB1D712000CC42CF00DC4D2
:102BD0002DF00EC42EF00FC42FF008C427F009C446
:102BE00028F00AC429F00BC42AF0C9EC6EF0010ADF
:102BF00001E096D005012351010A49E0030A45E0AE
:102C00000CC42CF00DC42DF00EC42EF00FC42FF008
:102C100008C427F009C428F00AC429F00BC42AF01C
:102C2000F7EC6CF027C000F028C001F029C002F0DA
:102C30002AC003F09A0E2C6E990E2D6E190E2E6E70
:102C40003F0E2F6E00C027F001C028F002C029F00F
:102C500003C02AF0F8EC6CF027C010F428C011F47F
:102C600029C012F42AC013F42C6A2D6A2E6A2F6A26
:102C700010C427F011C428F012C429F013C42AF09C
:102C8000D2EC6EF0010A09E103D0316948D047D097
:102C90000401106B116B126B136B2C6A2D6A7F0E83
:102CA0002E6E430E2F6E10C427F011C428F012C4EC
:102CB00029F013C42AF0C9EC6EF0010A07E10401FF
:102CC000106B116B7F0E126F430E136F10C427F041
:102CD00011C428F012C429F013C42AF06CEC6EF071
:102CE00029C031F50401006B070E005D18E20051A8
:102CF000EA6A240FE96E050EEA22EF50050131253C
:102D00000401016F050131510401015D03E2050178
:102D1000316902D001C431F50401002BE5D702D09E
:102D20000501316B120070C474F471C475F472C47F
:102D300076F473C477F405016351040DF3CFE9FF12
